:1000000008200300ED6D0200B16C0200B56C020027
:10001000056E0200096E02000D6E02000000000075
:10002000000000000000000000000000116E02004F
:10003000156E02000000000091F10000570C020054
:100040000000000000000000196E0200696C020050
:10005000ED42010000000000000000000000000070
:100060000000000000000000F56D0200000000002C
:100070000000000000000000DD540100000000004E
:10008000E555010027560100D9690200D96902002F
:1000900025680200000000000000000000000000D1
:1000A000F8B500224FF41261DFF8600B02F0E0F9BE
:1000B000DFF85C4B0022102104F1200002F0D8F997
:1000C000DFF8505B0022182105F10C0002F0D0F996
:1000D0000022082104F1300002F0CAF900220821B0
:1000E00004F1380002F0C4F9002020646064A064C8
:1000F000E0646862A862E862DFF81C6B7063B0635A
:10010000F0632863306470646863A863E863012067
:1001100028640020B064F0644FF0FF306864A86485
:100120000020E864306520657065F06530667066B3
:10013000B066B06202462821304602F099F90020EC
:1001400070600220308100203060DFF8D07A0246F3
:100150000C21384602F08CF9DFF8C40A7860DFF829
:10016000C40A386001203872002028702865688031
:10017000A880E8806065F066A060A065F0626865B0
:10018000A8656066A066E066706730676866286686
:10019000E86501202867E866A8660020E867A86788
:1001A0006867062030860020F067B0672067DFF8B8
:1001B000DC0DE065002020660120A081962068818A
:1001C000062070860C20E0810020B06502464021A8
:1001D00007F10C0002F04CF900220621204602F043
:1001E00047F90022102104F1100002F041F900202B
:1001F000E0616067F1BD10B584B0DFF8204A0C22E1
:10020000214600A802F072F9FFF74AFF0C2200A96C
:10021000204602F06BF91FBD2DE9F0472DED0C8B48
:1002200090B00024254600A821460A460B460EC081
:10023000302102F093F99FEDA98ADFF8D46996ED99
:100240001B0AD6ED140AC6ED1B0ADFF8CC7997ED30
:10025000149A86ED149ADFF8BC8998ED131AB8EE5B
:10026000411ADFED9F1AC1EE819AC7ED149AD8F8B2
:100270004420D8F83490A9EB0200FA30FA21B0FB00
:10028000F1F1FA2303FB110080B2002800F0228470
:100290004C2803DAD8F84010012906D12046F8622C
:1002A0000220A8F8080000F015BCD7F84CA0BAF15D
:1002B000040F24D3F4EE490AF1EE10FA1FD5B4EE80
:1002C000699AF1EE10FA1AD59FED861A20EE811A7E
:1002D000B4EE691AF1EE10FA11D59FED831AF4EE1F
:1002E000419AF1EE10FA0ADB87ED149AC6ED140A72
:1002F00086ED1B0A0320A8F8080000F025BC97ED46
:100300000DAA87ED0EAAD7ED10AAC7ED11AA0146D6
:1003100000EE101AB8EE400AD8ED0B8AC8EE800A3B
:1003200098ED0C1A81EE001A21467963396420E0B9
:10033000521C92B2FA2A00D12246DFF8D03803EBE1
:100340008203D3ED231A71EEE01AD3F8743402EE6F
:10035000103A32EE412AD7ED0D2A41EEA12AC7ED1F
:100360000D2AD7ED101A42EE021AC7ED101A491CD9
:1003700089B28142DCDBD7ED0D0A80EE80BA87EDD1
:100380000DBAD7ED100A80EE80CA87ED10CAD6EDFF
:100390001ABA98ED160AD8ED150A70EEC0CAF5EE35
:1003A00040CAF1EE10FA02DDC6ED1ACA03E030EEE3
:1003B000600A86ED1A0A00F0ADFF012802D120463E
:1003C000F86287E3BAF1000F0BD1B88D052802DB84
:1003D00005462046B885F88D052802DB45192046DC
:1003E000F8851AFA85F0002827D1B6EE00DA3CEE3F
:1003F0002A0A20EE0D0ADFEDA10AB4EE600AF1EE42
:1004000010FA11D43BEE0A0A20EE0D0ADFED9C0A29
:10041000B4EE600AF1EE10FA06D4B3EE040AF4EE7C
:1004200040CAF1EE10FA08D5B88D401CB885C8F85E
:1004300048900620A8F808004CE3B88D002802D0A8
:1004400045192046B8851AFA85F000281BD1B7EE69
:10045000000AF4EE409AF1EE10FA03D50720A8F84E
:10046000080037E39FED870AF4EE409AF1EE10FAA8
:1004700006DBF88D401CF8850820A8F8080029E361
:100480002046F88503E0F88D45192046F885284672
:1004900080B200F0E3FF012808D187ED149AC7ED80
:1004A00010AAC6ED1ABA87ED0DAA13E39FED760ADE
:1004B000F4EE409AF1EE10FA02DBDFF8380C386502
:1004C0002046B885BAF1000F10D1386D786587EDF8
:1004D0000FBAB06E706600F0B5FE40E0000000009C
:1004E00000007A446666E63F01004040B6EE00DA5E
:1004F00000F0A8FE012816D197ED140AF0EE000ACC
:1005000020EE200A87ED140A6BEE0D0AC7ED0D0AE6
:100510002CEE0D1A87ED101AC7ED0E0A87ED111A91
:1005200086ED140A6D1C97ED140AD6ED140A30EE10
:10053000200A20EE0D0A87ED150A97ED0D0AD7ED7A
:100540000E0A30EE200A20EE0D0A87ED0F0A96ED16
:100550001A0A3BEE800A20EE0D0A86ED190A98F879
:100560000100012840F0AB82D8F80C00009000A8F0
:10057000D8F810104160D8F814108160214617E0B7
:1005800000AB03EB820393ED010A50F822C000EEAA
:1005900090CAB4EE600AF1EE10FA05D500EB820CB9
:1005A0008CED000AC3ED010A521C022AE8DB491C4B
:1005B000022901DA2246F8E79DED000AB5EE400A6D
:1005C000F1EE10FA2AD5B5EE400AF1EE10FA01DC90
:1005D000B1EE400AD0ED020A30EE800A80ED020A48
:1005E0009DED000AB5EE400AF1EE10FA01DCB1EE25
:1005F000400AD0ED010A30EE800A80ED010A9DED3F
:10060000000AB5EE400AF1EE10FA01DCB1EE400A44
:10061000DDED000A30EE800A8DED000A90ED010A52
:10062000D0ED020A30EEC01ADDED000A30EE600AAD
:10063000B4EE401AF1EE10FA05D5F0EE410AB0EE34
:10064000401AB0EE600AD6ED0C0AC6ED0D0A31EE86
:10065000400A80EE010A9FED0D1A20EE010A86ED98
:100660000C0AB06BF063F4EE400AF1EE10FA0FD50D
:1006700070EE600AC6ED0E0A0EE000BF00001643E1
:100680000000A042666616400100A0400000C8427B
:1006900070EEC00AC6ED0E0A386F796F081800EBCD
:1006A000D070401002EE100A86ED102AC6ED118AB5
:1006B000D7ED100AC6ED120AD7ED141ADFF8500C68
:1006C000C0EDC41A96ED131A31EE611AD6ED132A55
:1006D00072EEE12A21EE221A00F5447181ED011A31
:1006E000C6ED131AD7ED1B1AC1ED021AD8F818106F
:1006F000039103A9C1ED011AC1ED020AC1ED038AFC
:10070000C1ED041AC1ED058AC1ED061AB8EEC22A80
:1007100081ED072AC1ED081A81ED090AC1ED0A1A17
:1007200081ED0B1ADDED032A9FEDD03A62EE832AAC
:100730009FEDCF3A41EE832A9FEDCE3A20EE833AE9
:10074000DFEDCD3A08EEA33ADFEDCC3A61EEA33A05
:100750009FEDCB4A48EE843A9FEDCA4A21EE844A87
:10076000DFEDC94A02EE244ADFEDC84A61EEA44A31
:100770009FEDC75A40EE054A9FEDC65A21EE855AB5
:10078000DFEDC55A01EE255AF8EE085AF4EE652A57
:10079000F1EE10FA00F19381DFEDC05AB4EE653A44
:1007A000F1EE10FA00F18B81DFEDBD5AF4EE653AFF
:1007B000F1EE10FA00F18381DFEDBA5AB4EE654A2A
:1007C000F1EE10FA00F17B819FEDB76AF4EE464A34
:1007D000F1EE10FA00F173819FEDDE6AB4EE465A35
:1007E000F1EE10FA00F16B81DFEDDB6AF4EE662AC0
:1007F000F1EE10FAC0F26381DFEDD82AB4EE623A6E
:10080000F1EE10FAC0F25B81F4EE653AF1EE10FA07
:10081000C0F25581B4EE464AF1EE10FAC0F24F81B3
:10082000F4EE654AF1EE10FAC0F24981DFEDCC2A10
:10083000B4EE625AF1EE10FAC0F24181DFEDC92A3E
:100840009DED033AB4EE623AF1EE10FA01D5CDED2A
:10085000032ADDED032A9FEDC43AF4EE432AF1EEBC
:1008600010FA02DBDFF8E82B0392DFEDD52AF4EE75
:10087000621AF1EE10FA01D5C1ED012A9FEDD13ACD
:10088000DFEDBA3A91ED014AB4EE634AF1EE10FAA7
:1008900001DB81ED013A9FEDB64AF4EE440AF1EE38
:1008A00010FA01D581ED024AD1ED020A9FEDB14A5D
:1008B000F4EE440AF1EE10FA02DBDFF8982B8A60BE
:1008C000DFEDC10AF4EE608AF1EE10FA01D5C1ED58
:1008D000030A9FEDBE4AD1ED034AF4EE444AF1EE1D
:1008E00010FA02DBDFF8702BCA60F4EE621AF1EE48
:1008F00010FA01D5C1ED042AD1ED044AF4EE634AA1
:10090000F1EE10FA01DB81ED043AF4EE608AF1EECB
:1009100010FA01D5C1ED050AD1ED050AF4EE440A3D
:10092000F1EE10FA02DBDFF8302B4A61F4EE621AC6
:10093000F1EE10FA01D5C1ED062AD1ED060AF4EE6A
:10094000630AF1EE10FA01DB81ED063AF1EE000ADE
:10095000B4EE602AF1EE10FA02D54FF08142CA617E
:10096000D1ED070A9FEDA32AF4EE420AF1EE10FA48
:1009700002DBDFF84C2CCA61F4EE621AF1EE10FAD9
:1009800001D5C1ED082AD1ED080AF4EE630AF1EEB3
:1009900010FA01DB81ED083ADFED970AB4EE600A48
:1009A000F1EE10FA01D5C1ED090A91ED090ADFED6A
:1009B000930AB4EE600AF1EE10FA02DBDFF8442C81
:1009C0004A62F4EE621AF1EE10FA01D5C1ED0A2A7C
:1009D00091ED0A0AB4EE630AF1EE10FA01DB81ED43
:1009E0000A3AB5EE401AF1EE10FA01D52246CA6273
:1009F00091ED0B0ADFED820AB4EE600AF1EE10FA17
:100A000002DBDFF8042CCA62214612E01B1FD3ED83
:100A1000000A92ED031AF4EE410AF1EE10FA01D544
:100A20009FED780AB8EEC00AD2ED020A00EE208AE5
:100A3000491C31293ADA9FED740A0B011A18D2F8D1
:100A400004C0BCF1010F0DF10C0C1B580CEB83031F
:100A5000DCD11B1FD3ED000A92ED031AF4EE410A1C
:100A6000F1EE10FADEDB9FED670ADBE7168733BD98
:100A7000B0568DBD03275BB9E23C9CB9983115BED9
:100A8000BF49D3B97061FDBD55C128BC36CB05BE89
:100A90003D7FDABBDDED0ABEE4BE353E6666A6BF2D
:100AA0003333F3BFCDCC4CBFCDCC8CBFB5EE408A39
:100AB000F1EE10FA03DD0F20A8F808000AE097ED28
:100AC000150A284680B200F0AFF800F055F8044649
:100AD000C8F84890C8F844900020C8F84C00C8F8FE
:100AE0002C00C8F83000C8F840000246102106F17A
:100AF000200001F0BDFC00220C2108F10C0001F0E7
:100B000031FDDFF88804F06500203066F8880028A1
:100B10001AD1F86F00280CD0B86CF968401A398ED9
:100B2000B0EB510F02DB002038810DE0012038814D
:100B30000AE0B88DF98D11FA80F0032802DB01205C
:100B4000388101E002203881204610B0BDEC0C8BCA
:100B5000BDE8F087333333BFCDCC0CC09A9919BFB1
:100B6000CDCC4CBE5017C93FC9AC454216E66840D3
:100B70007D90A341A2F2924438B50025DFF81C4CC9
:100B80000120E06700F01EFD2060E06C218E8842AD
:100B900014D3A06CE060208DA080608DE080A06DFB
:100BA0006061E06DA061206EE061606E2062A06E09
:100BB00060620120A0672846E0670125284632BD13
:100BC000A9F56E3E15E66840BA9F17443564EC44BB
:100BD0001148C16881640021C16441600221018122
:100BE00000218162C1690166416A81660021C16795
:100BF00070470000010058427B4D4F3D47FFC74200
:100C0000BEBA984101000000FFFFFFFFF86F03002C
:100C1000986403001863030098630300F0D1030095
:100C200000002F43000070422DE9F84F2DED048B9A
:100C300082B08346002213461046DFF8604BE56C15
:100C400005F10F0101F00F01EE1D06F007060096F9
:100C5000DFF8506B06EB810787ED030ABBF1000F4D
:100C600018D0074614E0A1F1010CACEB070C0CF115
:100C7000100C4FEAEC0E0CEB1E7E4FEA2E1EBCEB66
:100C80000E1C03D406EB8C0C8CED030A7F1C3FB2C8
:100C90005F45E8DB102D02D2294609B200E00F21A2
:100CA0009FEDBB8ADFEDBA0A9FEDBA1A07461BE03B
:100CB00006EB810CDCED031AF5EE401AF1EE10FAAA
:100CC00010DD38EE218AF4EE610AF1EE10FA01D55A
:100CD000F0EE610AF4EE411AF1EE10FA01D5B0EE31
:100CE000611A7F1C491E09B20029E1D53FB239467D
:100CF00003290BDB78EE600A70EEC10A891E01EE53
:100D0000101AB8EEC11A80EE818A07E0012905DBCE
:100D100000EE907AF8EEE00A88EE208AB5EE408A7E
:100D2000F1EE10FA01D0002F01D1B0EE408A84ED2F
:100D3000168A9FED990AB4EE408AF1EE10FA02D5B8
:100D4000B0EE408A08E09FED950AB4EE408AF1EEDD
:100D500010FA01DBB1EE028AB0EE040AB4EE408A6A
:100D6000F1EE10FA08D494ED1B0AF0EE080AB4EE86
:100D7000600AF1EE10FA02D50321218501E0042179
:100D80002185A76C07F00709DFF8208A09EB080E18
:100D9000218D8EF8B818BBF1000F0BD0A7F1010C14
:100DA0000CF0070CC44407F0070AC2449AF8B8A82C
:100DB0008CF8B8A84FF0080C10E0BAF1040F00D17D
:100DC000401CA9F101090FFA89F9B9F1000F01D509
:100DD00009F10809ACF1010C0FFA8CFCBCF1010F10
:100DE00016DB0FFA89F909EB080A9AF9B8A8BAF1E3
:100DF000030F01D15B1C03E0BAF1040F00D1521CB8
:100E0000BCF1060FDDDBBAF1030FD6D1401ED8E7E7
:100E1000B4F82AC092B29BB29A4207D3934202D24C
:100E2000042060850DE000B2002802D50320608513
:100E300007E0012802DB0420608502E09EF9B80883
:100E40006085B4F82A90B9F1040F01D1104600E092
:100E50001846CC4509D000202081E088002820D108
:100E6000042D1ED3012020811BE012FA83F2012AF7
:100E700015DB052A10DB00EE102AB8EEC00AF6EEEC
:100E8000080A20EE200A00EE900AF8EE600AF4EE5E
:100E9000400AF1EE10FA02D50120208101E0022083
:100EA000208149B2B0EE480A304600F025F9DFED66
:100EB000900AB4EE600AF1EE10FA01D5B0EE600AC5
:100EC00084ED170A584600F1010A00EE90AAF8EEE8
:100ED000E08AD4ED180A48EE800AC4ED180A9FEDA6
:100EE000CE9A20EE080A20EE090A009908EB81014B
:100EF00001F65C0181ED000ABBF1000F1AD04FF042
:100F0000000C15E00099491EA1EB0C0108318A1074
:100F100001EB5272D210B1EBC20105D408EB810192
:100F200001F65C0181ED000A0CF1010C0FFA8CFC5A
:100F30008445E7DB082D02D2284600B203E00720F3
:100F400001E0401E00B20028FBD584ED190A494695
:100F500049B2304600F048F968EE090AB7EE001AC7
:100F6000C1EE200A20EE800AD4ED1A0A48EE800A6B
:100F7000C4ED1A0A0AEB0700A0640AEB0500E0645E
:100F800002B0BDEC048BBDE8F18F000000007A4494
:100F9000000000000000C8426666A63F01009040C5
:100FA00049B2032944D1DFED9D0AB4EE600AF1EEA7
:100FB00010FA01DBB0EE600A9FED991ADFED990A95
:100FC00040EE010A90ED011A9FED970AB4EE401A27
:100FD000F1EE10FA43DADFED951AB4EE611AF1EE94
:100FE00010FA74DBB4EE401AF1EE10FA6FD59FEDF3
:100FF000900A31EE000ADFED8F1A60EE211A9FEDA4
:101000008E0A9FED8E2A01EE002A22EE200A20EEA3
:10101000210A9FEDB72ADFEDB72A41EE022A62EEE0
:10102000A00AB7EE001A31EE611A00EE810A56E00E
:10103000DFED830A60EE200A60EE800A9FEDAE1AB3
:1010400040EE410A9FEDAD0A70EE800A90ED011A64
:101050009FED750AB4EE401AF1EE10FA0ADB90ED3E
:10106000010A9FED751ADFED751A40EE011A21EEA7
:10107000A00A34E0DFED6D1AB4EE611AF1EE10FA59
:1010800025DBB4EE401AF1EE10FA20D59FED680A88
:1010900031EE000ADFED671A60EE211A9FED660A55
:1010A0009FED662A01EE002A22EE200A20EE210A98
:1010B0009FED8F2ADFED8F2A41EE022A62EEA00A11
:1010C000B7EE001A31EE611A00EE810A07E090EDEA
:1010D000010A20EE800ADFED8A0A20EE200A007A5B
:1010E000022803D1DFEDD10A20EE200A704700006C
:1010F000CDCC4C3E0000A04010B52DED028BB0EEE3
:10110000408A0C46DFED7F8A49B2FFF749FF64B29F
:10111000042C31D1DFED7C0AB4EE608AF1EE10FAD6
:1011200016DBB1EE021AB4EE418AF1EE10FA0FD5D9
:10113000DFED760A78EE200AB1EE041A60EE810A3D
:10114000FCEEE00A10EE900AC01D08EE900A3DE0A9
:10115000B4EE608AF1EE10FA03D5072008EE900A8B
:1011600034E0F1EE020AB4EE608AF1EE10FA2DDB03
:10117000122008EE900A29E0F7EE080AB4EE608A21
:10118000F1EE10FA11DBDFEDAA0AB4EE608AF1EE9F
:1011900010FA0AD5FFEE080A78EE200AB1EE041A1A
:1011A00060EE810AFCEEE08A10E0F7EE080AB4EE89
:1011B000608AF1EE10FA09D4DFED9D0AB4EE608A80
:1011C000F1EE10FA02DB062008EE900ADFF8FC0CC4
:1011D00018EE901A00EB8100D0ED000A20EE200AF4
:1011E000BDEC028B10BD0000F0EE0C0A49B20429E0
:1011F00004D19FED901A40EE010A03E09FED8E1A94
:1012000040EE010A9FED8D0A20EE800AD0ED000A23
:1012100020EE200A70470000000070429A991940A1
:101220006ADEF13D8638163F00002A43000016436F
:10123000000016C3CDCC4C3D4260E53A6666263FC1
:101240002575C23E0020DFF8541591ED140AF7EE23
:10125000040AB4EE600AF1EE10FA47DADFF8702CF7
:10126000D288042A42DAD1ED150A9FED751A60EE94
:10127000810AB4EE600AF1EE10FA03D5022A01DB0E
:10128000012012E0DFF84C1C91ED0B0ADFED6D0A36
:10129000B4EE600AF1EE10FA07DBDFED6B0AB4EE94
:1012A000600AF1EE10FA00D5012001281ED1DFF806
:1012B000241C91ED170AD1ED180A70EEC00A9FEDBB
:1012C000631AF4EE410AF1EE10FA07DBF7EE080AB2
:1012D000B4EE600AF1EE10FA00D50020DFEDC50A89
:1012E000B4EE600AF1EE10FA00D50020704700005D
:1012F00052491D3BB81E053F7593E83F2497534064
:10130000C1C0C03B0000000066660640666606C0BD
:10131000805803000021DFF88424538D032B1FDA4B
:1013200092ED140ADFEDA50AB4EE600AF1EE10FAB0
:1013300016DB92ED0D0AF2EE040AB4EE600AF1EE4D
:1013400010FA0DD592ED100ADFEDAB0AB4EE600A8B
:10135000F1EE10FA04D50421DFF8743B1981012164
:1013600092ED100AF6EE000A92ED111A30EE011A13
:1013700021EE201AF3EE0E1AB4EE611AF1EE10FA15
:101380001CD492ED0D1AD2ED0E1A71EE211A61EEF7
:10139000A01AB2EE042AF4EE421AF1EE10FA0DD4BD
:1013A000F3EE041AB4EE610AF1EE10FA06D4B1EECF
:1013B000040AB4EE401AF1EE10FA04D50521DFF864
:1013C000103B1981012192ED140A9FED8C1AB4EEA5
:1013D000410AF1EE10FA27DBDFF8F82A92ED0A0A4B
:1013E00092ED0B1A80EE010A9FED851AB4EE410AC8
:1013F000F1EE10FA18DB00EE100AB8EE400A20EE0B
:10140000200AD2ED080AF4EE400AF1EE10FA0BD5EC
:10141000D2ED090AF4EE400AF1EE10FA04D50E20DE
:10142000DFF8AC1A08810121084670473333733F57
:101430009A993940CDCC4C3ECDCCCC3D0AD7A33B7C
:101440003333333F010020420000C8420100C03F57
:10145000C8AC4542A1F292443464EC4401460020F9
:10146000CE4AD36C13FA81F102291AD392ED140AF1
:10147000DFED8F0AB4EE600AF1EE10FA11DB92EDA7
:10148000110AD2ED100A80EE200ADFED8A0AB4EECE
:10149000600AF1EE10FA04DB0920DFF8343A188113
:1014A000012002291CD39FED840AD2ED110A92ED8E
:1014B000101AC0EE810AF4EE400AF1EE10FA0FDBCA
:1014C000D2ED0E0A92ED0D1AC0EE810AF4EE400A3A
:1014D000F1EE10FA04DB0A20DFF8F439188101205C
:1014E000002913D0DFF8EC1991ED190ADFEDA50AF8
:1014F00020EE200AD1ED1A0AF4EE400AF1EE10FABD
:1015000004D50B20DFF8C8190881012092ED140AD8
:10151000DFED9D0AB4EE600AF1EE10FA08DA92ED02
:10152000150ADFED9A0AB4EE600AF1EE10FA1EDB3E
:1015300092ED100ADFED960AB4EE600AF1EE10FAB1
:101540000DD492ED0D0ADFED930AB4EE600AF1EED0
:1015500010FA04D4DFF87819C988022907DB518D05
:10156000032904DB0C20DFF868190881012092EDC3
:101570000F0ADFED870AB4EE600AF1EE10FA08D424
:1015800092ED1B0AF1EE040AB4EE600AF1EE10FAD5
:1015900012D5116F526F511800EE101ABAEEEF0A01
:1015A000DFED7D0AB4EE600AF1EE10FA04DB0D20E7
:1015B000DFF81C190881012070470000010000407D
:1015C00000005842002075498A6C12F1640F0FD256
:1015D0009FED730AD1ED180AF4EE400AF1EE10FA0D
:1015E00006DAD1ED1A0AF4EE400AF1EE10FA00DB49
:1015F0000120704785EB113F000020420100404070
:101600003433333F46FFC742BDBA984110B4014658
:101610000020DFF8C028654BD3F8144900EE104ACB
:10162000D1ED000AB4EE600AF1EE10FA08D1147898
:10163000641C1470E4B2FE2C04DB3224147001E04C
:101640000446147003F6141393ED010AD1ED010A58
:10165000B4EE600AF1EE10FA08D15478641C5470AC
:10166000E4B2FE2C04DB3224547001E004465470D2
:1016700093ED020AD1ED020AB4EE600AF1EE10FA1F
:1016800008D19178491C9170C9B2FE2904DB32213E
:10169000917001E0014691701178322905DA517894
:1016A000322902DA9178322900DB012010BC704720
:1016B000010060400100A04001007041014600208F
:1016C00091ED000AB5EE400AF1EE10FA01DCB1EE40
:1016D000400ADFF80028DFED340AB4EE600AF1EECC
:1016E00010FA08DBD3785B1CD370DBB2FE2B04DB73
:1016F0003223D37001E00346D37091ED010AB5EEB9
:10170000400AF1EE10FA01DCB1EE400AB4EE600AD4
:10171000F1EE10FA08DB13795B1C1371DBB2FE2BC0
:1017200004DB3223137101E00346137191ED020AC9
:10173000B5EE400AF1EE10FA01DCB1EE400AB4EE6B
:10174000600AF1EE10FA08DB5179491C5171C9B2F7
:10175000FE2904DB3221517101E001465171D1783B
:10176000322905DA1179322902DA5179322900DB7E
:1017700001207047DFF89C0CC0697047DFF8940CBB
:10178000006970479A99993E01009040010080409D
:101790000000C8430000164301008C429863030018
:1017A0008096184BF0D1030035336B41F86F03007E
:1017B0002DE9F84F2DED068B86B0814688464FF017
:1017C000000A9FEDD88ADFEDD78A9FEDD69ADFED2C
:1017D000D59ADFF8444CE088ADF81000A088ADF849
:1017E00002002089ADF800005046019005464846A9
:1017F000FFF70CFF03904846FFF760FF0290DFF809
:10180000D06628467065B0653081B06EDFF80C7C1C
:10181000D7F8141900EE101AD9ED000A30EEC01AEC
:1018200001EE900AF8EEE11A21EE211AB5EE401A07
:10183000F1EE10FA1BD596ED1D1A70EE411AF5EE79
:10184000401AF1EE10FA01DC71EE401A9FEDB61A63
:10185000F4EE411AF1EE10FA05DB216F491C216705
:10186000F16D491CF16586ED1D0A4042B06607F630
:10187000141090ED010AF16E99ED011A31EE401A43
:1018800001EE901AF8EEE11A21EE211AB5EE401A97
:10189000F1EE10FA1BD596ED1E1A70EE411AF5EE18
:1018A000401AF1EE10FA01DC71EE401A9FED9E1A1B
:1018B000F4EE411AF1EE10FA05DB226F521C22679A
:1018C000326E521C326686ED1E0A4942F16690ED78
:1018D000020A306F99ED021A31EE401A01EE900AB9
:1018E000F8EEE11A21EE211AB5EE401AF1EE10FAE7
:1018F0001BD596ED1F1A70EE411AF5EE401AF1EE67
:1019000010FA01DC71EE401A9FED871AF4EE411ACD
:10191000F1EE10FA05DB216F491C2167716E491C3D
:10192000716686ED1F0A404230673078052805D180
:1019300001203064284630707080B080F06C4044E4
:10194000F064706B716C884201D101203064B06B1F
:1019500000EB400107EB810B0BF6C000C0ED000A65
:10196000D9F804104160D9F8081081604146484612
:1019700000F0B2FA2061DFF85C850398012802D0FC
:101980000298012836D19FED670ADBF8C00800EE07
:10199000900A60EEA00ADBF8C40801EE100A21EEFE
:1019A000011ADBF8C80801EE900A61EEA11A98F856
:1019B0000000322805DA98F80300322801DA30EE08
:1019C000800A98F80100322805DA98F804003228D5
:1019D00001DA30EE010A98F80200322805DA98F8A8
:1019E0000500322801DA30EE210A00F025FDB0EEC4
:1019F00040AA37E00BF50C60D0ED020A90ED011A19
:101A0000DBF8C00800EE100A20EE000A01EE010A21
:101A100000EEA00A00F010FDB0EE40AAD9ED010AD8
:101A200099ED000A20EE000A00EEA00A00F004FD85
:101A3000F0EE408AD9ED020A99ED010A20EE000A83
:101A400000EEA00A00F0F8FCB0EE409AD9ED020AD0
:101A500099ED000A20EE000A00EEA00A00F0ECFC6E
:101A6000F0EE409AF06B002824D128460CE007EBFA
:101A7000800181ED15AA07EB8002C2ED008A81ED9D
:101A8000079AC1ED0E9A401C0728F0DBF068B061A0
:101A90003069F06170693062B1EE0C0A68EE800A5C
:101AA000C6ED030A69EE000AC6ED040A29EE800AB3
:101AB00086ED050AB06B07EB800181ED15AA07E002
:101AC00007EB8A0090ED150A38EE008A0AF1010A48
:101AD000BAF1070FF4DB86ED098A96ED090A706BFF
:101AE00007EB800080ED230AD6ED0B0A70EE800A2A
:101AF000C6ED0B0AF268B2613269F2617269326254
:101B0000B26B07EB8202C2ED008A81ED079AC1ED4C
:101B10000E9A2A46DFED030A9FED021ADFED011A45
:101B200013E000BF00000000CECC4C3E07EB820368
:101B300093ED002A70EE820A93ED072A31EE021A25
:101B400093ED0E2A71EE821A521C072AEEDBC6EDC7
:101B5000030A86ED041AC6ED051AD1ED1C0A70EED3
:101B6000600A00F27442C2ED000A81ED1C0AD6ED53
:101B70000C0AD0F8742401EE102A70EE810AC6ED2A
:101B80000C0AD9ED000AF5EE400AF1EE10FA01DC7C
:101B9000F1EE600A9FEDCB1AF4EE410AF1EE10FA75
:101BA0001BDAD9ED010AF5EE400AF1EE10FA01DC7C
:101BB000F1EE600AF4EE410AF1EE10FA0DDAD9ED19
:101BC000020AF5EE400AF1EE10FA01DCF1EE600ACD
:101BD000F4EE410AF1EE10FA08DB0122C8F81C20ED
:101BE000D8F8102042F00102C8F81020B4EE41AA43
:101BF000F1EE10FA04DAB5EE40AAF1EE10FA08D5CB
:101C00000122C8F81C20D8F8102042F00202C8F8BF
:101C10001020B5EE400AF1EE10FA08D50122C8F8FE
:101C20001C20D8F8102042F00402C8F810209FEDC4
:101C3000A60AD1ED1C0AF4EE400AF1EE10FA08DB18
:101C40000121C8F81C10D8F8101041F00801C8F89C
:101C50001010D0ED230AF4EE400AF1EE10FA08DB82
:101C60000121C8F81C10D8F8101041F01001C8F874
:101C70001010D0F8741400EE101AD8ED050AF4EE26
:101C8000400AF1EE10FA10D1D8F81810491CC8F823
:101C90001810FB290CDB0121C8F81C10D8F8101013
:101CA00041F02001C8F8101002E02946C8F81810C9
:101CB00088ED050AD8F81C10012901D12846FCE05E
:101CC00007F6141199EC030A81EC030AD8F8701096
:101CD000012906D101203064284630707080B08020
:101CE0007CE0316D491C31653278012A01D0032A2C
:101CF00037D102292AD2628D042A27DAE16C002921
:101D00006CD196ED0A0ADFEDD70AB4EE600AF1EE67
:101D100010FA08D5D0F8741401EE101AB4EE601A57
:101D2000F1EE10FA0FDAF9EE0C0AB4EE600AF1EEF9
:101D300010FA53DBD0F8740400EE100AB4EE600A17
:101D4000F1EE10FA4AD50120306447E0272908D384
:101D50007288002A03D011FA82F14B2901D30121A4
:101D60003164D0F8740400EE900A96ED0A0A00F08F
:101D70007BF9D8F87400401CC8F87400FB2805DB18
:101D80000120307030647080B08030653078012878
:101D900024D17088002821D0B18800291ED00322C8
:101DA00011FA80F03D2801DB01203064608D0428A9
:101DB00000DB0222F088824201D2012030642846F2
:101DC00070663066F065FEF727FA0190206F606755
:101DD00028462067B080F080C8F87400706BB16C42
:101DE000401AFA304FF0FA084146B0FBF1F108FB17
:101DF00011007189884201D100F037FA706BB16C23
:101E0000401AFA304146B0FBF1F108FB110064289A
:101E100001D100F06BFAE088BDF81010814204D1C6
:101E2000BDF80210A288914200D00125002812D0EE
:101E3000706BB16C401AFA304146B0FBF1F108FB0F
:101E40001101322902D10120208114E04B2912D145
:101E5000002020810FE0A08800280CD0706BB16CAE
:101E6000401AFA304146B0FBF1F108FB11007D2821
:101E700001D101202081BDF800002189884200D0D5
:101E80000125706B07EB8001D1F87414B162401C1E
:101E90007063FA2801D100207063B06B401CB063FE
:101EA000072801D10020B063F06B401CF06301985B
:101EB0002843401E8041C043C00F06B0BDEC068BD6
:101EC000BDE8F28FC4F51C430C578944D465030068
:101ED000186303009864030010B4DFF8402590ED08
:101EE000000AD2F8143900EE903A30EE600A02F699
:101EF0001413D0ED010A93ED011A70EEC10A90EDB2
:101F0000021AD3ED021A31EE611AB5EE400AF1EE73
:101F100010FA02DDF0EE401A01E0F1EE401AF5EEA3
:101F2000400AF1EE10FA02DDB0EE602A01E0B1EEF7
:101F3000602AB5EE401AF1EE10FA02DDF0EE412A09
:101F400001E0F1EE412A71EE821A71EEA21AB5EEAD
:101F5000400AF1EE10FA01DCB1EE400ADFF8B404F9
:101F600090ED082A32EE000A80ED080AF5EE400AEC
:101F7000F1EE10FA01DCF1EE600A90ED090A30EEA4
:101F8000200A80ED090AB5EE401AF1EE10FA01DCE4
:101F9000B1EE411A90ED0A0A30EE010A80ED0A0A0C
:101FA00090ED0B0A30EE210A80ED0B0ADFF8703459
:101FB000DB6B002B12D1002306E002EB840404F655
:101FC0007C04C4ED001A5B1C9BB21C460F2CF4DB96
:101FD000B2EE0E0A21EE800A80ED150A038902EBAB
:101FE0008302D2F87C4800EE104A31EEC00AD0EDF0
:101FF000150A30EE200A80ED150A02F67C02C2EDC9
:10200000001AF2EE0E0A80EE200ADFF80C2482EDB0
:102010001B0AD0ED170AB4EE600AF1EE10FA01D5F2
:1020200080ED170AD0ED180AF4EE400AF1EE10FA2E
:1020300001D580ED180ADFEDAB0AB4EE600AF1EECF
:1020400010FA03D5826D8918816501E00021816550
:10205000591C018189B20F2901D100210181806DB4
:1020600010BC70470100E0409FED9F1ADFF8A80305
:10207000408D042801DBB0EE001ADFF8A403B5EEB2
:10208000400AF1EE10FA07DBF5EE400AF1EE10FA25
:1020900002D5C188491CC1800178002905D00229D8
:1020A00060D02DD3032976D0B0E0F1EE0C1A31EEDA
:1020B000211AB4EE401AF1EE10FA0BDBB4EE601AFE
:1020C000F1EE10FA06D5016D1029C0F08F800021C5
:1020D00001658BE0416BDFF8442302EB8101D1F80D
:1020E000741401EE901ADFF83C1391ED010AF4EE3E
:1020F000401AF1EE10FA40F18980C1ED011A85E035
:10210000416BDFF8182302EB8101D1F8741401EE62
:10211000901ADFF8101391ED002AB4EE612AF1EE67
:1021200010FA01D5C1ED001AF7EE001AB4EE610AFB
:10213000F1EE10FA6ADBB7EE000AF4EE400AF1EEB7
:1021400010FA63D5016D418000210165B9EE0C0ADA
:1021500030EE410AF4EE400AF1EE10FA10D40221FA
:10216000017053E0F9EE0C1A31EEC11AB4EE410AD7
:10217000F1EE10FA4ADBF4EE410AF1EE10FA45D521
:1021800003210170A549426B01EB8201D1F874145F
:10219000A44A51603AE0416BA04A02EB8101D1F8B8
:1021A000741401EE901A9F4991ED012AF4EE421A3F
:1021B000F1EE10FA01D5C1ED011ADFED831AB4EE8C
:1021C000610AF1EE10FA21D5F4EE610AF1EE10FA8F
:1021D0001CDB016D818000210165B1EE0C0A31EE3E
:1021E000000AB4EE600AF1EE10FA0ED5012101707A
:1021F0008C490A6842654A688265884A436B02EBEB
:102200008302D2F874240A6000E0017000787047FD
:1022100000280CD0C168804AD160916490ED070A13
:1022200082ED070A406A506282ED180A9066704794
:10223000002803D07849282200F058B970470028B8
:1022400006D0794942684A6002680A60007A0872DA
:10225000704780B5002801D1002002BD54220146FC
:10226000724800F043F9012002BD10B56A4C608D40
:10227000218D002904D0002802D00020208106E012
:10228000084302D00120208101E0022020810020AB
:10229000E06420626061A0802085E0626065A065E6
:1022A00002464021624800F0E3F8E06F012801D1C6
:1022B000FEF78EFC57484189002909D0628E8A4278
:1022C00001D2218600E02286002141810846A067D4
:1022D000A06F012801D1608E20860020A06710BD6C
:1022E00000000000EC51383E0000000010B54A4CE0
:1022F000608D218D002904D0002802D0002020818B
:1023000006E0084302D00120208101E00220208164
:102310000020206260616085E08002460821454817
:1023200000F0A6F80020E062E06F012801D1FEF77E
:102330004FFCA06F012801D1608E208610BD80B5B2
:10234000012034490867FFF7D1FFFFF78EFFBDE892
:10235000014003E000202F49086770472D48C089DD
:102360002D49098E814200D200E070472A49CA6C8B
:102370000B8E9A4203D20886002088677047254951
:10238000488170472448C16C002904D1818DC08DDB
:1023900010FA81F0704700207047014600200029A4
:1023A00002D0012901D0704702E01B48C06C704781
:1023B0001948018EC26C891A828D891AC08D081A3B
:1023C00000D5002070470000FEFF7FBF38B50446EF
:1023D0001348104D1049012C06D106224A860C22C2
:1023E000EA819622428105E007224A860F22EA818D
:1023F00064224281A889A04209D0088E082803DA05
:10240000488EFFF7B3FF02E0E889FFF7AFFFAC812A
:1024100031BD00009864030098630300F86F030067
:102420001863030014D90300F0D10300D46503003E
:10243000FCD10300B078030081B08DED000A009854
:10244000401000F1FE500090DDED000AC0EE200AC1
:102450009DED001A70EE810ACDED000AB5EE001A6E
:10246000DDED001A80EE210A00EE810A01B070470E
:1024700062F30F2262F31F4200B500BF13009646BD
:102480009446103928BFA0E80C50FAD85FEA417C86
:1024900028BF0CC048BF40F8042BC90728BF20F84C
:1024A000022B48BF00F8012B00BD50F8041B61B19E
:1024B00050F8042BD30744BFA9F101039A18002355
:1024C000091F42F8043BFAD1EFE7704762B38B076C
:1024D00008D0521E11F8013B00F8013B00F02480A7
:1024E0008B07F6D1830740F0208000BF103A07D356
:1024F00030B4B1E83810103AA0E83810F9D230BC46
:10250000530724BFB1E80810A0E8081044BF51F8F1
:10251000043B40F8043BD20724BF31F8022B20F8DB
:10252000022B44BF0B7803707047083A07D3B1E819
:102530000810083A40F8043B40F804CBF7D25307A0
:10254000E4E78268521C8260426832B10268531C20
:10255000036011704168491E416070470022FFF717
:102560008BBF000062F30F2262F31F42401810F08D
:10257000030308D0C91A1FD3DB0748BF00F8012D99
:1025800028BF20F8022D130030B414461546103928
:1025900028BF20E93C00FAD8490728BF20E90C00F1
:1025A00048BF40F8042D890028BF20F8022D48BFFD
:1025B00000F8012D30BC7047C91818BF00F8012D74
:1025C000CB0728BF00F8012D7047000038B505463D
:1025D0000C46224629460FF2240001F053FCDFF896
:1025E000482D2046002102EBC503C3E90001108DF0
:1025F0000121A9400843108531BD0000416C617282
:102600006D5F4164642025753A25750A000000005D
:1026100010B5044621460FF21C0001F033FC0120E6
:10262000A040DFF8041D0A8D82430A854A8D1043BD
:10263000488510BD416C61726D5F57616B65757047
:102640002025750A0000000010B5044621460FF24F
:102650002C0001F017FCDFF8D00C0022134600EB31
:10266000C401C1E900230121A140C943028D0A40F0
:102670000285428D1140418510BD0000416C6172A0
:102680006D5F52656D6F76652025750A000000004C
:1026900010B500241AE0DFF8900C018D0122A24051
:1026A000114212D000EBC401D1E90023521E63F1A4
:1026B000000300EBC400C0E90023002B05DC01DBB4
:1026C000012A02D22046FFF7A3FF641C052CE2DB9F
:1026D00010BD10B5DFF8544D606E002801D1002008
:1026E00010BD01F01BFA616E401A4FF47A71B0FB15
:1026F000F1F010BD38B50446DFF8305D28780028C9
:102700000AD1012C15D100220421012000F090FEF5
:1027100001F004FA68660CE001280AD1012C08D007
:10272000FFF7D7FF02460421012000F081FE0020C0
:1027300068662C7031BD10B5DFF8F04C20790007C9
:1027400009D50FF2400001F09DFB0C2001F040FE86
:10275000022000F0A6FE6078012808D10121206A3D
:10276000D4ED030A94ED020ABDE81040CCE2012149
:10277000206CD4ED0B0A94ED0A0ABDE81040C3E2C8
:102780000000000041637469766520474E53532072
:102790004C4F432043420A0010B5DFF8904C20789C
:1027A00001280CD1DFF8800B90F82A00800741D572
:1027B0000020FFF79FFF0120BDE8104044E7E088BC
:1027C000002801D0401CE08004F1480104F1080019
:1027D00000F0E1F900F08EF8E088032802DBBDE8A4
:1027E0001040A8E7DFF8401B91F82A10890721D58F
:1027F0002178022913D1A16C002905D1002803D129
:102800000120BDE81040C5E20120FFF71DFF0A21AD
:102810000120FFF7DBFE0320BDE810406AE7032933
:1028200008D1002802D0BDE8104084E70120BDE8AF
:102830001040AFE210BD38B5054601F06FF9DFF882
:10284000F04C024621780FF23C0001F01BFBA088FF
:102850000121A9400843A0802078022810DA4FF017
:10286000FF30A0640020E08000F077F90220FFF73D
:1028700041FF05210120FFF7A9FE01F04FF9206675
:1028800031BD00004750535F53746172742025645A
:102890002025750A0000000038B5044601F03EF915
:1028A000DFF88C5C024629780FF2380001F0EAFA72
:1028B000002C02D10020A88004E0A8880121A140BA
:1028C0008843A880287802280BDBA888002808D134
:1028D00000F052F90020FFF70DFF0120BDE8324063
:1028E000B2E631BD4750535F53746F7020256420AA
:1028F00025750A00F8B5DFF8344BD4E9062304F156
:102900001805D5E908018B4201D1824238D0002B4D
:1029100001D1002A34D00FF2F80001F0B3FA261DDD
:1029200096ED010ADFEDD20AB4EE600AF1EE10FA7C
:1029300016D4DFEDD00AB4EE600AF1EE10FA0FDA29
:1029400096ED020ADFEDCC0AB4EE600AF1EE10FA61
:1029500006D4DFEDCA0AB4EE600AF1EE10FA11DB1C
:102960000FF2C40001F08EFA287B002804D0042165
:10297000012000F070FC03E00321012000F06BFC5B
:102980000020F2BDA868652805D30521012000F0CC
:1029900062FC0020F2BD671C7A78A1880FF29C00CF
:1029A00001F070FA2079000702D4787800281FD04F
:1029B0000FF2A00001F066FADFF8780B9FEDD10A64
:1029C000D6ED010A60EE800AFDEEE00AC0ED000AD5
:1029D000D6ED020A20EE800ABDEEC00A80ED010AA3
:1029E000A9688160D4E90623C0E90423296B018327
:1029F00004F1280004F108012022FFF777FD708818
:102A0000002801D10120708001206070F2BD00001B
:102A10004750535F4C6F635F4669786564203A2086
:102A2000256C6C750A000000475053204C6F6320E2
:102A300057726F6E6721210A000000004750535FF4
:102A40004C6F635F46697865642025752025750A9B
:102A50000000000055706461746520474E53532098
:102A60006C6F630A000000000FB470B5DFF8BC693A
:102A7000307802284DD003284BD0DDE90E452246A0
:102A80002B460FF2940001F0FDF9DDE9040101F09D
:102A90008FFFB060DDE9060101F08AFFF0600020E1
:102AA00030617061C6E9064510983062012086F8F1
:102AB0002400FFF71FFF00282BD03078002807D113
:102AC00002210120FFF782FD0120FFF713FE06E03F
:102AD0000120FFF7B9FD02210120FFF777FDB07853
:102AE00000280ED04FF0FF30DFF8481A08830FF2AD
:102AF000400001F0C7F90C2001F06AFC022000F050
:102B0000E4FC0321306AD6ED030A96ED020A00F0D8
:102B1000FBF870BC5DF814FB4750535F5061737352
:102B20006976655F434220256C6C750A00000000E1
:102B30005061737369766520474E5353204C4F4361
:102B40002043422025750A00002803D0DFF8E80959
:102B500001F0D5BF002001F0D2BF80B5BF2002F048
:102B60007AFA014600208DF80000002903D000A861
:102B7000C9694968884701BD80B5BF2002F06BFA7A
:102B8000014600208DF80000002903D000A8C96983
:102B9000C968884701BD70B504460D4602F02FF89C
:102BA0000646D6E9000101F003FF2060D6E90201E4
:102BB00001F0FEFE60600020A060E060D6E90A013E
:102BC000C4E90401306BA06100202077002D02D001
:102BD00096F83C0028600020DFF85419487070BD5A
:102BE00080B50FF2300001F04DF9DFF84008002108
:102BF00080F8681000F168019FEDD30A81ED020AA8
:102C000081ED030A00228A61012280F888200020D9
:102C1000887001BD4C4D5F496E69740A0000000068
:102C200038B50C46DFF8085995F86810012901D02D
:102C3000022907D1224601460FF24400BDE8384080
:102C400001F020B92146012807D10FF2580001F008
:102C500019F92046FFF7EFFD06E00FF25C0001F0E6
:102C600011F9204600F031F9012085F8680031BDE6
:102C70000000B4C20100B442000034C30100344378
:102C80004C4D5F5265715F4C6F633A256420616CF7
:102C900072656164792072756E6E696E673A25643B
:102CA0000A0000004C4D5F5265715F4C6F63204716
:102CB00050533A25640A00004C4D5F5265715F4CD9
:102CC0006F63204E4C503A25640A000070B50446EC
:102CD000DFF858572878022802DB2046FFF7DCFD92
:102CE000DFF8B86D307D002802D0204600F00EF9E4
:102CF0002878002805D1307D002802D1002085F8F1
:102D0000680070BD8096184BF8B52DED028B86B02B
:102D1000B0EE408AF0EE608A04460D46DFF80C679C
:102D200006F16807B9690FF2540001F0ABF8EDB293
:102D3000012D07D100220321012000F079FB0020A2
:102D4000FFF7AAFDD6E90E232146F0EE680AB0EEA1
:102D5000480A00A800F0D9FB06F1700000A918226B
:102D6000FFF7C4FB86F888500020B870022086F870
:102D7000680006B0BDEC028BF1BD00004C4D5F4C0D
:102D80006F635F46697865642061725F643A2564A9
:102D90000A00000010B5044621460FF2380001F089
:102DA00071F8DFF88C07012C0BD1032180F8681033
:102DB00000220521012000F03BFB0020BDE810406F
:102DC0006AE5042180F86810002207210120BDE88F
:102DD00010402DE34C4D5F4C6F635F54696D656F20
:102DE00075742025750A00002DE9F0472DED028B42
:102DF00086B008EE100A08EE901A92461F46DFF8D9
:102E00002C8608F16809DDE91045129ED9E9040114
:102E1000A94213D301D8A04210D322462B460FF269
:102E2000780001F02FF8002E30D0324639460720C6
:102E300006B0BDEC028BBDE8F047F9E232463946F8
:102E4000072000F0F5FA22462B465146B8EEE80A74
:102E5000DFEDC70AC0EE200AB8EEC80A9FEDC41A1B
:102E600080EE010A00A800F050FB08F1700000A9F4
:102E70001822FFF73BFB88F88870012089F80200D0
:102E8000002000F043F8022088F8680006B0BDEC8E
:102E9000028BBDE8F08700004C4D5F5365745F4CBA
:102EA0006F6320536B697021210A000080B5DFF841
:102EB000F40B90F82A00400706D5002000F026F811
:102EC0000220BDE8024065E701BD38B504460FF2B7
:102ED000300000F0D7FFDFF8C45BE88A0121A14091
:102EE0000843E882287D002808D1032001F070FA09
:102EF0001E210220FFF76AFB0120287531BD00006A
:102F00004E4C505F5265710A0000000038B505460E
:102F10000FF2380000F0B6FFDFF8804B002D02D131
:102F20000020E08204E0E08A0121A9408843E08299
:102F3000207D002807D0E08A002804D10220FFF776
:102F400083FB0020207531BD000048434E4C505F8C
:102F500053746F700A00000080B50FF6FC4000F05B
:102F600091FFDFF83C0B002101800161416181721A
:102F7000C160C161816101BD30B583B001AA0DF1AD
:102F8000010100A800F0B4F8DFF8144B2069002814
:102F900007D00199884202D2081AE06001E00020BF
:102FA000E0606078002801D1002161619DF8001087
:102FB00088421DD00121A1720A259DF800109DF8BC
:102FC000012015FB0122A17815FB00110FF694409A
:102FD00000F058FF62699DF800009DF8011015FB94
:102FE0000011C9B2032000F023FA0020606105E05F
:102FF0006069E168081860610020A0720198206192
:1030000000F08CFD60609DF80000012803D100F005
:1030100085FDE06107E0042805D1A07A002802D0F0
:1030200000F07CFDA0619DF8000060709DF801003B
:10303000A07037BD38B504460FF63C4000F022FFC3
:10304000DFF85C5A28890121A140084328812878AB
:10305000002805D100F02AF8002802D001202870AD
:1030600031BD0FF62040BDE8324000F00BBF38B54F
:1030700004460FF6244000F005FFDFF8245A2889A3
:103080000121A140884328812978012907D10028FE
:1030900005D100F01CF8002802D00020287031BDB6
:1030A0000FF60040BDE8324000F0ECBE80B50FF6F0
:1030B000084000F0E7FE0022DFF8541A9A2001F0E1
:1030C000A7FE002801D0002002BD012002BD80B56E
:1030D0000FF6F03000F0D6FE0022DFF8341A9A2006
:1030E00001F0F2FE002801D0002002BD012002BD47
:1030F0007CB504460D46164600A802F0B2FE9DF8C7
:10310000000020709DF80100287002F0BBFE3060C6
:1031100073BD10B5DFF888496078042807D100F046
:10312000FDFCA169401A44F6206188420AD2607809
:10313000012809D000F0F2FCE169401A4EF6602146
:10314000884201D3012010BD002010BD80B5DFF8FA
:103150004C09002141620A461021001DFFF702FAC6
:1031600000221521DFF8AC09BDE80840FFF780B95F
:103170008096184B2DE9FF4104460F4615462E4612
:1031800033463A4621460FF6483000F07BFE012CCC
:1031900056D1012F54D1DFF808090769DFF8FC8800
:1031A00098F80400002807D188F8045031460FF63B
:1031B000403000F067FE41E0D8F8242039460FF691
:1031C000543000F05FFED8F82400381AA8F8060042
:1031D000B8F80A00B8F80C100818B8F80E1008185B
:1031E000B8F810100818B8F812100818A8F8080055
:1031F000072001F0EDF8B8F812000390B8F81000BD
:103200000290B8F80E000190B8F80C000090B8F8E1
:103210000A30B8F80820B8F806100FF6203000F091
:1032200031FE0022102108F10400FFF79BF988F815
:10323000045031460FF6543000F024FEC8F82470D4
:10324000DFF85888B8F820000121A1400843A8F809
:103250002000BDE8FF8170B505460E460FF65030E0
:1032600000F010FEDFF8AC4821780A290CDA0FF6DE
:10327000503000F007FE20780019457020780019C2
:10328000C6722078401C207070BD10B5DFF80C08A5
:1032900090F82000800701D500F01BF803F016F825
:1032A000DFF87048227801460FF6203000F0EAFD82
:1032B00003F00CF801280BD12078002808D00FF675
:1032C000243000F0DFFD082001F082F8002020709B
:1032D00010BDDFF8CC074078012805D1DFF8BC0726
:1032E0004189491C41817047022805D1DFF8AC07AC
:1032F0008189491C81817047032805D1DFF89C072B
:10330000C189491CC1817047042805D1DFF88C07A9
:10331000018A491C01827047052804D1DFF87C0727
:10332000418A491C4182704768D5030010B5DFF817
:103330006C47A08B401CA08380B2322818DB002091
:10334000A083FFF7A5F939480078002801D0FFF7DE
:1033500023FA207D002801D0FFF7A8FDDFF8400701
:103360000078002801D0FFF707FEBDE810408CE789
:1033700010BD6F4890F86810022902DB002180F828
:103380006810704738B50FF6742000F07BFD0022FE
:103390003021DFF81007FFF76BF8244C00222821BA
:1033A00004F16800FFF764F8002268212046FFF767
:1033B0005FF8DFF8E8560022062105F11400FFF758
:1033C00057F800222021DFF8D806FFF751F8002037
:1033D0002870014604F12800FFF7DDFBFFF700FC31
:1033E000FFF7BAFD0120FFF7AFFB0022202105F116
:1033F0002000FFF73DF8BDE83140A7E60020FFF7C9
:10340000A3BBDFF8A80600687047DFF89C0670478A
:1034100080B50022C821DFF89006FFF729F80020C8
:10342000DFF88816086001BD0000000000CF03002F
:10343000F8B507460E461446DFF870562868BF28D0
:1034400005D30FF6C410BDE8F24000F01BBD00F03C
:1034500065FB2A68DFF850165754521C2A605654F0
:10346000521C2A60230E5354521C2A60230C5354BE
:10347000521C2A60230A5354521C2A605454521C72
:103480002A60030E5354521C2A60030C5354521CDE
:103490002A60030A5354521C2A605054501C28605E
:1034A000F1BD10B5044621460FF6841000F0EAFC89
:1034B000012C05D103210120BDE81040FFF7B0BB6E
:1034C0000320BDE81040FFF701BC10B504462146BB
:1034D0000FF6741000F0D6FC1548012C02D1012122
:1034E000817010BD0021817010BD10B504462146C9
:1034F0000FF6701000F0C6FC2046401E8041C0430D
:10350000C00FDFF89815087010BD00B587B08DEDBD
:10351000000ACDED010A0591DFF8841509690491CF
:10352000CDE9022300A91822FEF7E0FF07B000BD95
:1035300000CF0300B0D60300693A00002DE9704FB8
:103540002DED108B94B0B0EE418A9FED73AA21EE61
:103550008A1A00EECA1A8DED0B1A00200A9020EE8E
:103560000A0A03F0DFF89FED6D9BF7EE000AF0EE1C
:10357000608A10EE100A03F085F953EC192B03F062
:10358000A9F901F015FA00EE100AF0EE680A03F04E
:1035900073FAF0EE408A28EE0A0A03F0C3F8F7EE59
:1035A000000AB0EE608A10EE100A03F06BF953ECDB
:1035B000192B03F08FF901F0FBF900EE100AF0EE81
:1035C000480A03F059FAB0EE408AB0EE680A03F0F8
:1035D0008AFA8DED090AB0EE480A03F084FA8DEDFF
:1035E000040AB0EE680A03F081FA8DED080AB0EE25
:1035F000480A03F07BFA8DED070A9DED090ADDED1F
:10360000040A20EE200A8DED060A9DED080ADDED84
:10361000070A20EE200A8DED050A9FED3EEA9FED98
:103620003DAA9DED0B8A002600E0761C36B2142ED2
:1036300080F21E828DED0C8AB0EE480A03F053FA38
:10364000F0EE409AB0EE480A03F050FAB0EE409A1D
:103650009DED040A20EE090ADDED090A9DED071A29
:1036600060EE810A9DED081ADDED041A21EE211AA3
:1036700041EE690A20EE000A00EEA00AB5EE400A0B
:10368000F1EE10FA0EDB10EE100A03F0FBF841EC3D
:10369000100B03F02FFA51EC100B01F089F908EE32
:1036A000900A01E0DFED1B8A9DED060A9DED058A7B
:1036B00000EE298AF0EE480AB0EE680A03F0DCF961
:1036C000B0EE40EAF5EE408AF1EE10FA02D1DFEDFD
:1036D00011EA05E09DED060A20EE090AC0EE28EA8F
:1036E000B7EE00AA0EEEEEAA18EE100A03F0CAF822
:1036F000CDE912011AEE100A03F0C4F841EC1B0BDD
:103700009FEDE49BB5EE40AAF1EE10FA0AD19FEDD1
:1037100001CA1CE00000000034FA8E3C000020B515
:1037200088E4EF3F059803F0ADF853EC192B03F054
:10373000D1F853EC1B2B03F05DFA02460B46DDE992
:10374000120103F07BFB01F033F90CEE100A9FED40
:10375000D00A2AEE000A10EE100A03F093F841ECAA
:103760001A0B0022D24B03F0B5F804460D4651EC7B
:103770001A0B0022CF4B03F0ADF802460B46002097
:10378000CD4903F05BFB02460B4651EC1A0B03F0EC
:10379000A1F80022C94B03F011FC02460B4651EC84
:1037A0001A0B03F097F80022C54B03F007FC2246E2
:1037B0002B4603F08FF80022D14B03F0FFFB01F002
:1037C000F7F80A9051EC1A0B0022BE4B03F082F876
:1037D00004460D4651EC1A0B0022BB4B03F07AF85D
:1037E00002460B460020B94903F028FB02460B466F
:1037F00051EC1A0B03F06EF80022B54B03F0DEFB20
:1038000002460B4651EC1A0B03F064F80022B14B50
:1038100003F0D4FB22462B4603F05CF801F0C8F815
:103820000FEE100A9FEDACAB51EC1B0B4FF060425A
:10383000AB4B03F04FF804460D4651EC1B0B002236
:10384000A84B03F047F802460B4651EC1A0B03F065
:10385000F5FA4FF06042AB4B03F03CF853EC1A2BF7
:1038600003F0ACFB22462B4603F034F801F0A0F83D
:103870000FEE900A2CEE0C0A10EE100A03F002F87C
:10388000CDE9100118EE900A02F0FCFFCDE90E011F
:103890001FEE100A02F0F6FFCDE902011CEE100A3D
:1038A00002F0F0FF41EC1B0B9FED8FCB9FED90DB07
:1038B0002FEE280A10EE100A02F0E4FFCDE9000115
:1038C000DDE9020100228C4B03F004F804460D46AA
:1038D000DDE9100153EC192B02F0FCFF53EC1D2B1A
:1038E00003F06CFB02460B46DDE9120102F0F2FF29
:1038F00082468B46DDE902010022804B03F07AF913
:1039000053EC1B2B02F0E6FF80468946DDE90E23CF
:1039100051EC1A0B02F0DEFFDDE90E2302F0DAFFB4
:1039200053EC1C2B03F04AFB42464B4602F0D2FFFD
:1039300080468946DDE9102351EC1A0B02F0CAFFDC
:1039400053EC1C2B03F03AFB42464B4602F0C2FFFD
:1039500002460B465046594603F070FA22462B4663
:1039600002F0B8FF02460B4651EC1B0B03F026FB9E
:10397000DDE9002302F0AEFF01F01AF80AEE100AAA
:103980000B9802F07FFFCDE902011FEE900A02F0D2
:1039900079FF02460B460020594903F04FFA4FF0D9
:1039A0006042584B02F096FF04460D461EEE900A08
:1039B00002F068FF22462B4602F08CFFCDE90001A1
:1039C0001EEE100A02F05EFF804689462FEEA80A1E
:1039D00010EE100A02F056FF04460D462FEE880A3C
:1039E00010EE100A02F04EFF82468B4653EC1B2B62
:1039F00051EC190B02F06EFF53EC1B2B02F06AFF27
:103A000053EC1D2B03F0DAFA52465B4602F062FFDC
:103A100053EC1B2B03F0D2FA22462B4602F05AFF3E
:103A200042464B4603F0CAFADDE9002302F052FF9A
:103A3000DDE9022303F0C2FA00F0BAFF08EE100A33
:103A4000B5EE408AF1EE10FA02D19FED2F0A05E0A3
:103A50009DED0C0A38EE400A80EE080AB0EEC00A6E
:103A6000DFED2A0AB4EE600AF1EE10FA7FF5DDAD63
:103A70009DED0A0ADFED280A20EE200A7EEE4A0AB2
:103A800020EE200A14B0BDEC108BBDE8708F00BF93
:103A900032D6DC3B000000000000004020D40300D0
:103AA00090D6030068D5030038CE030054D9030034
:103AB0000000103F00E0654000007440000088C036
:103AC0000000B0400000503F00804740008052405E
:103AD000000060C0000070400000000000001040C6
:103AE0004A772B3F0000084000000000000008C09B
:103AF000000000000000F0BF0000D03F00001840B0
:103B00000000F03F4A776B3F00000000CDBC8C2BDB
:103B1000886F0300E0D7030021FEC14A00B583B0DF
:103B20000FF25830D0E90023CDE9002300A802F0BD
:103B300035FC9DF900004FF461619DF90120C2EB55
:103B400002139A0011FB00209DF9021040FA81F047
:103B50004FF47A7148430EBD10B40B885C1C0C8086
:103B6000140A1C540B885C1C0C801A5410BC70473F
:103B700010B40B885C1C0C8014161C540B885C1C45
:103B80000C8014141C540B885C1C0C8014121C54E4
:103B90000B885C1C0C801A5410BC70472DE9F04354
:103BA0000546884616461F464FF038090CE0601C53
:103BB000A8F80000304639464A4603F073FA6055CB
:103BC000A9F108091FFA89F9B8F800404846002809
:103BD000EDD1601CA8F800006655BDE8F0830278BE
:103BE00012020A8040781018088070470278120686
:103BF0000A60437802EB03420A60837802EB0322F7
:103C00000A60C0781018086070472DE9F043074635
:103C10000E464FF03809387800214A4603F052FA30
:103C2000C6E900014FF001080EE0A9F10809D6E944
:103C30000045C05D00214A4603F044FA201869415E
:103C4000C6E9000108F101080FFA88F84046082883
:103C5000EBDBBDE8F083000041525F496E69740AF6
:103C60000000000041525F5052203A202564202D70
:103C70003E2025640000000041525F53746172745D
:103C80000A00000045203A4152204F70656E2046E0
:103C900061696C0A0000000041525F53746F700A42
:103CA0000000000045203A415220436C6F736520AC
:103CB0004661696C0A00000041525F4F70656E0AF0
:103CC0000000000041525F436C6F73650A00000002
:103CD0004269675F446174615F436D645F48616E10
:103CE000646C65722025642025642025640A000028
:103CF0004269675F446174615F436D645F48616EF0
:103D0000646C65722053746172742069643A25642E
:103D10000A0000004269675F446174615F436D643B
:103D20005F48616E646C6572206375725F643A25EA
:103D30007520696E695F643A25750A004269675F9C
:103D4000446174615F436D645F48616E646C657269
:103D50002053746F7020646973743A256420746F03
:103D600074616C5F74696D653A25642073743A25DB
:103D7000642077613A25642072753A25642076655F
:103D80003A25642063793A25640A00004269675F36
:103D9000446174615F436D645F48616E646C657219
:103DA0002053746172742069643A256421210A00E9
:103DB0004269675F446174615F45523031000000C1
:103DC000496E736572742025640A00004269675F5A
:103DD000446174615F50726F636573732025642062
:103DE00025640A0053656E642045523031204361DA
:103DF0006C6C6261636B210A00000000534C435FEE
:103E0000496E69740A000000534C435F5365745F48
:103E100044756D705F446174612054656D702064F9
:103E2000756D702069732046756C6C21210A000045
:103E3000534C435F476E73735F526571756573745E
:103E40003A25750A00000000534C435F476E7373B8
:103E50005F506173736976655F546573743A257555
:103E60000A000000534C435F5365745F446F7A65EA
:103E70005F4D6F64653A25750A0000000000000080
:103E8000000000000EB403B0704770B586B0044661
:103E90000D462A4621460FF6B02003F025F9681D8D
:103EA000ADF8000001A80FF6E0211422FEF71EFB7A
:103EB000BDF80000C01CADF80700DFF8586A01200B
:103EC0003070022200A9701CFEF700FB0120F07088
:103ED0003071372070710A2095FBF0F0B071052029
:103EE000F071BDF80000C21EDFF82C0A201800F1A6
:103EF000100106F10800FEF7E9FA314601A803F0C7
:103F0000F1F906B070BDF8B5FFF77BFA0546DFF8AA
:103F1000084A40F2F9402189461A002D33D0FFF7B4
:103F200074FAE06021890B19AE4216D2324601467E
:103F300003F11000FEF7CAFA40F2F9406081002058
:103F40002081AA1BE068311804F11000FEF7BEFAC8
:103F500020892818801B208113E02A46014603F19E
:103F60001000FEF7B3FA208928182081618980B2F9
:103F7000814200D2608140F2F941884201D10020A3
:103F80002081FFF745FA02F0A1F90546012D25D160
:103F900094F90400002821D100266789002F08E049
:103FA000394689B2304680B2FFF76FFFBE1960898B
:103FB000871B08D0FB2FF3D3FA21304680B2FFF7DE
:103FC00064FFFA36F3E7002240F2F94104F11000F1
:103FD000FEF74EFA012060710020A0602571F1BD4E
:103FE0000020704738B5DFF83449257829460FF6A8
:103FF0007810FFF747FF002D14D1012020700FF635
:104000007410FFF73FFFFFF7BDF900F03EF8002006
:10401000FFF710F803F072FE03F0DEFE04F05DF926
:1040200004F056FE002032BD80B50FF65410FFF7A5
:1040300029FF00F02AF80020FFF719F80120FEF709
:1040400045FE03F06FFE03F035FF04F060F904F065
:104050004BFEFFF7D3F90020DFF8C018087002BD4F
:1040600080B50020DFF8B018C880FFF75FF903F0D3
:104070003FFF04F000F904F009FEFFF77AF9FFF7BB
:1040800042FF002002BD0020704780B5DFF888089D
:1040900001214171002181600A4640F2F94110304E
:1040A000FEF7E6F9BDE8014003F036BF70B58AB00F
:1040B000144600221346CDE90823114604910591C8
:1040C0000691ADF80C10102801D008467EE120784A
:1040D000DFF84458287069706980401E322800F269
:1040E0006C81DFE810F03300370068006A01790066
:1040F0009200AD00B800BF006A016A016A016A015E
:104100006A016A01C900EB00FB00110117012001DF
:104110006A016A016A016A016A016A016A016A0147
:104120006A016A01260134013A016A016A016A01E1
:104130006A016A016A016A016A016A016A016A0127
:104140006A016A01400157015D016401012000F02C
:104150003FF932E104A9601CFFF748FD05A9601D85
:10416000FFF744FD06A904F10900FFF73FFD667B58
:1041700008A904F10E00FFF748FDA47D2046029037
:10418000DDE90801CDE900013346069A0599049856
:10419000FEF72AFE0294DDE90801CDE9000133466D
:1041A000069A0599049804F07FF904F011F80220AA
:1041B00000F00EF901E166783046FFF796F904F059
:1041C00053FA03F035FD002231460820FFF730F99D
:1041D000022000F0FDF8F0E0667804A9A01CFFF7CB
:1041E00005FD05A9A01DFFF701FD06A904F10A00C0
:1041F000FFF7FCFC069B059A0499304603F025FD69
:104200006870022000F0E4F8D7E094F9010001287A
:104210002ED10222A11C03A8FEF758F9BDF80C000C
:104220000146090A41EA0020ADF80C00BDF90C0076
:1042300003F0DFFD00206870BDF80C00688017E017
:104240006678E278A1783046FEF794FF6E8002200F
:1042500000F0BEF8B1E06678012E09D13046FFF7D4
:1042600020F905E06678012E02D13046FFF72DF9DE
:10427000022000F0ADF8A0E003A9601CFFF7AFFC3E
:1042800004A9E01CFFF7B2FC05A9E01DFFF7AEFC96
:1042900006A904F10B00FFF7A9FCE07B0090069B48
:1042A000059A0499BDF80C0003F02CFB6870BDF86A
:1042B0000C006880022000F08BF87EE003A9601CEF
:1042C000FFF78DFCBDF80C0003F0B6FB6870BDF87D
:1042D0000C006880022000F07BF86EE003A9601CEF
:1042E000FFF77DFC04A9E01CFFF780FCE27904994C
:1042F000BDF80C0003F028FC6870BDF80C00688065
:10430000022000F065F858E003F06EFC122000F087
:104310005FF852E00120FEF7D9FCFFF7B6FE02205D
:1043200000F056F849E003F05FFC132000F050F86D
:1043300043E003A9601CFFF752FCE178BDF80C00D4
:1043400003F010FF6870022000F042F835E003F03F
:104350001FFF022000F03CF82FE003F025FF0220B1
:1043600000F036F829E004A9601CFFF73FFC05A91E
:10437000601DFFF73BFC03A904F10900FFF72FFCC8
:10438000BDF80C200599049804F05EF8022000F0B6
:104390001FF812E004F07CF8022000F019F80CE09D
:1043A000012004F036F9022000F012F805E06078F0
:1043B00004F047F9022000F00BF86879032801D0D7
:1043C00002206871002004F024F900200AB070BDBA
:1043D0002DE9F04186B00021ADF80010DFF8384536
:1043E000E1880D46012827D0022848D0032868D04C
:1043F000042877D0072800F09780082800F0D080A4
:104400000C2800F0FC80102800F02481112800F016
:104410004B81122800F06B81132800F08F81202837
:1044200000F0C281212800F0CF81302800F0F78110
:10443000312800F01A8227E20820ADF80000DFF8EA
:10444000E06407208A191071491CE180012089B2BB
:104450008A191071481CE080D6F80424A11D301D73
:10446000FFF786FBE088142182191171401CE0805F
:10447000317880B282191171401CE08004E206207C
:10448000ADF80000DFF8986405208A191071491C06
:10449000E180022089B28A191071491CE1802078DC
:1044A00089B28A191071481CE080617880B2821943
:1044B0001171401CE0806288A11D301DFFF74CFB8C
:1044C000E2E10220ADF80000DFF8546401208A190F
:1044D0001071491CE180032089B28A191071481CAF
:1044E000E080D1E10C20ADF80000DFF834640B204F
:1044F0008A191071491CE180042089B28A1910714F
:10450000481CE080DFF81C743A88A11D301DFFF7BD
:1045100023FB7A68A11D301DFFF72AFBBA68A11D95
:10452000301DFFF725FBAFE11120ADF80000DFF8EB
:10453000F06310208A191071491CE180072089B2AC
:104540008A191071491CE180DFF8DC73387889B270
:104550008A191071481CE0807A88A11D301DFFF770
:10456000FBFABA88A11D301DFFF7F6FAFA88A11DE3
:10457000301DFFF7F1FA3A89A11D301DFFF7ECFA63
:104580007A89A11D301DFFF7E7FABA89A11D301DF8
:10459000FFF7E2FAFA89A11D301DFFF7DDFA73E19A
:1045A000E24802785300DE1CADF80060DC4E9B1C34
:1045B0008F193B71491CE180082389B28F193B7127
:1045C000491CE18089B28B191A71491CE1800021D4
:1045D000914280F25981E3880F187F7803EB060C33
:1045E0008CF804705B1CE3800F18FF7A9BB203EB1E
:1045F000060C8CF804705B1CE380491CE8E718206B
:10460000ADF80000C64E17208A191071491CE180D0
:104610000C2089B28A191071481CE080C44F3A6896
:10462000A11D301DFFF7A4FA7A68A11D301DFFF708
:104630009FFABA68A11D301DFFF79AFAD7E9042343
:10464000A11D301DFFF7AAFA3A8BA11D301DFFF7FF
:1046500083FA19E11120ADF80000B14E10208A193B
:104660001071491CE18089B28A191071481CE080E0
:10467000B04F3A88A11D301DFFF76EFAE088B97877
:1046800082191171401CE0807A68A11D301DFFF76E
:104690006FFABA68A11D301DFFF76AFAFA68A11D0A
:1046A000301DFFF765FAEFE00C20ADF800009C4EDE
:1046B0000B208A191071491CE180112089B28A19D6
:1046C0001071491CE1809C4F387889B28A191071A9
:1046D000481CE080797880B282191171401CE0801A
:1046E000D7E90223A11D301DFFF758FACCE0934F04
:1046F00038784200D31CADF80030894E921C8B19DB
:104700001A71491CE180122289B28B191A71491C55
:10471000E18089B28A191071481CE0804FF00008CE
:104720003878804580F2B08007EB48004288A11DB0
:10473000301DFFF711FA08F10108F1E77F4F3878D3
:104740004200D31CADF80030754E921C8B191A71C3
:10475000491CE180132289B28B191A71491CE1802E
:1047600089B28A191071491CE1800021814280F2CE
:104770008B8007EB41025288E3884FEA921C03EBDF
:10478000060E8EF804C05B1CE38001EB070C9CF85E
:104790002AC04CEA82029BB203EB060C8CF8042080
:1047A0005A1CE280491CE1E70220ADF800005C4E93
:1047B00001208A191071491CE180202089B28A19D0
:1047C0001071481CE0805FE01A20ADF80000544EE4
:1047D00019208A191071491CE180212089B28A1997
:1047E0001071481CE080564F3A68A11D301DFFF73C
:1047F000BFF9D7E90223A11D301DFFF7CFF93A69B0
:10480000A11D301DFFF7B4F97A69A11D301DFFF716
:10481000AFF9BA69A11D301DFFF7AAF934E01420E1
:10482000ADF800003E4E13208A191071491CE1803A
:10483000302089B28A191071481CE080414F3A68D3
:10484000A11D301DFFF794F97A68A11D301DFFF7F7
:104850008FF93A89A11D301DFFF77EF9D7E90423AE
:10486000A11D301DFFF79AF90EE00220ADF80000FF
:104870002B4E01208A191071491CE180312089B228
:104880008A191071481CE0806079032801D0022049
:104890006071E088B0F5806F29DCBDF80000C01CB5
:1048A000ADF8000001A80FF2F4011422FDF71EFE7E
:1048B000BDF80000C01CADF80700164C01202070A8
:1048C000022200A9601CFDF701FE0120E0702071AA
:1048D00037206071BDF80000C21E11482818011D64
:1048E000A01DFDF7F3FD214601A802F0FBFC06B078
:1048F000BDE8F081074901F58272C261B7220270FA
:1049000014228260012202730282002242824161EB
:1049100010467047845D03004C4C03006CD90300C3
:1049200058510300ACD4030024D40300E0D70300A3
:10493000B0D603005CD8030078D80300C0AB0300F6
:1049400050D60300C0D10300736C632053656E64BE
:104950004269674D53472073746172743A2564202D
:1049600073697A653A256400534C432B2025640A09
:1049700000000000736C635F73746172740A00005E
:10498000534C432D00000000050000000000000013
:104990000000000000000000000000000500000012
:1049A0000000000000000000000000000000000007
:1049B0004FEAF17CBCF1E04C2CBFBCF5001F11E0CC
:1049C0005FEA4C0C34BFBCF17F5F2EE05FEA9C0CC9
:1049D0004FEA0C1C4FEA3C0CC10071F100414CEB5A
:1049E00050707047C90241EA5051C00218BF41F0EF
:1049F000010141F000414FEA6C50C0F1090021284B
:104A000010D240EACC7CCCF1200C11FA0CF070F101
:104A10000040CCF1200C21FA0CF00CF0004C40EBE3
:104A20000C0070474FEACC707047490011F5001F29
:104A300004D84FEACC10FF30C0057047C817704744
:104A400010B5724C90ED000B84ED000B90ED020B55
:104A500084ED020B90ED040B84ED040B90ED060B3E
:104A600084ED060B00221346C4E90823D0E90A238B
:104A7000C4E90A23006B206301F079FCA06310BD38
:104A80000021624A006882F83C0092F83C3003E062
:104A9000401C9842FCDB491C082901DA0846F8E76B
:104AA000704730B597B0574C90ED000B84ED000B7C
:104AB00090ED020B84ED020B90ED040B84ED040BE2
:104AC00090ED060B84ED060B00221346C4E9082383
:104AD000D0E90A23C4E90A23006B206301F047FCF4
:104AE000A06349484568280007D0214684B068463D
:104AF0006822FDF7FBFC0FBCA84717B030BD38B5E6
:104B00000400414D68680AD1002813D0002004F049
:104B1000C0FB04F08FFB00206860012032BD00283C
:104B200008D13E4804F078FB012004F0B2FB6C6031
:104B3000012032BD002032BD10B5344C0022682166
:104B40002046FDF795FC9FED320B84ED000B84EDC4
:104B5000020B2D48002101704160084610BD000085
:104B600038B5294C94F90000002814D1274D0022B3
:104B700068212846FDF77CFC9FED250B85ED000B99
:104B800085ED020B244804F041FB254804F041FB6D
:104B9000012004F057FB94F90000002803D4401CC6
:104BA0002070002032BD032032BD80B5164890F938
:104BB000001001290CDB491E017049B2002905D102
:104BC00004F05DFB04F02EFB04F030FB002002BD7E
:104BD000032002BD0020704700207047002070476E
:104BE000104901F10C02C261BF22027024228270BE
:104BF000012202820922428241610020704703485B
:104C00007047000038D10300F4D80300D0D003006F
:104C10000000000000006940415A0000A35A000053
:104C2000815A00009C6B03002DE9F04100242546C9
:104C3000DFF898791EE0052004F0BAFC0020F16945
:104C400009688847002804D02046441CC0B20228C6
:104C5000F1DBE4B2032C0BDB0020317847F82100B4
:104C6000307857F82000C8F80400304604F072FE8F
:104C70006D1C0024242D18DA2C2004F053FE064667
:104C800022462C21FDF7F4FBDFF84489304658F822
:104C900035108847307847F8206008EBC508307831
:104CA00057F82000C8F80400C8E72046BDE8F081A6
:104CB000002200E0521C92B28A4204D2135CFF2B05
:104CC000F8D0012070470020704702B51346372105
:104CD00019705870022200A9981CFDF7F7FB01BD5E
:104CE00002B5104601210170022200A9401CFDF707
:104CF000EDFB01BD008A022801DB01207047002086
:104D0000704770B588B0064602A80FF62C11142221
:104D1000FDF7ECFBDFF8B40850F82600458A281DA3
:104D200004F000FE0446224601213046FFF7CDFF85
:104D3000211D304604F017FF281DADF80B00284652
:104D4000A0F1080189B2201DFFF7B2FF00280DD0A5
:104D500001F00DFBCDE90001082200A9281908384F
:104D6000FDF7B4FB214602A802F0BCFA204604F08D
:104D7000F1FD08B070BD10B50C46C17801290ED107
:104D800000216160FFF7B6FF002805D0A068002869
:104D900002D001F03DFB00E00020A06010BD806863
:104DA000002804D001F034FBA060606010BD606892
:104DB00001F02EFB6060A06010BD30B400216FF0E8
:104DC0000042104616E0DFF8084804EBC3035B68B6
:104DD000002B0ED01C6A002C0BD0DD78002D08D1E2
:104DE000E4681B78052B01D1042C02D0A04200DD21
:104DF0002046491C49B20B46242BE4DB082801D08D
:104E0000102800D10420904200D1002030BC70470F
:104E10002DE9F04184B0044615462646DFF8AC077C
:104E200050F8267008788DF800004868019088686E
:104E30000290002F01D1032043E000A93846FFF77C
:104E40009AFF00A907F1200004F0D6FF07F11C0823
:104E500098F80C0001280BD1204604F0B7FE07F1AA
:104E6000100005F043F80020F969496888470DE013
:104E70009DF80000002809D107F1100005F036F870
:104E80003879012802D12046FFF73BFF2A4600214E
:104E90003D20FB691B699847F878002802D1022061
:104EA00005F039F9D8F80800002801D0012300E006
:104EB000002398F80C2031460FF2247002F014F908
:104EC000002004B0BDE8F081FEB506461446DFF8C8
:104ED000FC0650F8265008788DF8000048680190CC
:104EE00088680290002D19D09DF8000000280AD192
:104EF00005F11C07B868002810D0C0680190B86898
:104F00000069029003E000A92846FFF734FF00A9DA
:104F100005F1200004F090FF002801D00320FEBD21
:104F2000EB6905F11C07387B002803D10020D96804
:104F3000884704E0224600213E201B699847022052
:104F400005F0E9F8B868002801D0012300E000234B
:104F50003A7B31460FF2946002F0C6F80020FEBDA5
:104F600030B587B00546DFF8640650F8254008786C
:104F70008DF80C00486804908868059010788DF8CA
:104F800000005068019090680290002C03D00878CF
:104F90001178884201D0032030E003A92046FFF7B2
:104FA000EAFE00A92046FFF7E6FE04980199884230
:104FB00005D105980299884201D100201EE000A980
:104FC00004F1200004F038FF002801D0032015E090
:104FD00003A904F1200004F00FFF002211463F2036
:104FE000E3691B699847022005F095F8049B019A34
:104FF00029460FF2046002F077F8002007B030BDB8
:1050000010B50C4611461A46DFF8C03553F820306B
:10501000002B01D1012010BD2046DB691B69984798
:10502000002010BD10B50C4611461A46DFF89C351D
:1050300053F82030002B01D1012010BD192C04D1D0
:10504000012100F0A7F9002010BD2046DB695B6953
:105050009847002010BD0146CE2901DA002801D171
:1050600000207047DFF8640550F82100704710B544
:1050700082B000218DF80010082804D010281CD020
:10508000202830D013BD00AA01214020DFF83C3594
:105090005B68DB695B6998479DF80000800703D572
:1050A0000021012005F075F89DF80000400732D579
:1050B0000021022005F06DF813BD00AA0121402057
:1050C000DFF808355B68DB695B6998479DF800008D
:1050D000000703D50021032005F05BF80021042020
:1050E00005F057F813BDDFF8E404046A01F03FF956
:1050F000E2699268904700280DD1606A002806D0C6
:105100000069002803D10021082000F043F90021A4
:10511000084605F03EF813BD10B50446206AA268A3
:10512000002A07D1002810D04269521A012A05DB53
:105130004068F7E74069401A012806DA01F017F9DC
:10514000E2699268BDE81040104710BD2DE9F843B0
:1051500004460D4604F1100004F040FF064604F139
:10516000100004F042FF07462078372802DA4FF09B
:10517000040801E04FF00308002F43D040F2012063
:1051800008EB0601814203DB2046BDE8F243C5E09F
:10519000B5F8031016FA81F2DFF8349408EB020137
:1051A00081420DDB0FF25C410FF26C4001F09CFF7D
:1051B00009F59071284602F095F80020A5F8030043
:1051C000B5F80300484400F590722078372803DAD8
:1051D0003946FFF77AFD02E03146FFF781FD3A4696
:1051E00004F11001B5F8030018FA80F0484400F506
:1051F000907004F0ABFEB5F8030008EB0601081848
:10520000A5F80300BDE8F18338B504461546606A89
:1052100000280FD08069401A01280BDA01F052F8FB
:10522000012802D1207B002804D029462046BDE871
:1052300034408BE731BDF0B585B000A80FF20C41CA
:105240001422FDF753F904F05CFF04460025DFF853
:10525000806328E006EBC5004768002F14D097F85C
:105260002800002810D0F87800280DD121463846B3
:10527000FFF752FF00AA21463846FFF7C5FF214637
:1052800007F1200004F0F5FD042D0BD1BDF803005B
:10529000002807D006F5907100A802F023F800203E
:1052A000ADF803006D1C242DD4DBBDF803000028ED
:1052B00003D0C84900A802F015F8002005B0F0BDE1
:1052C00070B5C24951F82050002D26D0C24C20782C
:1052D000401C2070802080F3118800BF00BF6078E0
:1052E000401C60702E6A09E006F108012846FFF7AD
:1052F00042FDF06870613069B0617668002EF3D1CC
:105300006078401E6070C0B2002802D1002080F397
:105310001188BDE8704005F0C9B870BD2DE9F043B3
:1053200085B0044600A80FF238311422FDF7DEF8EC
:1053300025784FF4FE70618A90FBF1F6B6B204F165
:10534000100004F052FE0746DFF8909219E0B846CC
:105350004A4641462846FFF7B8FC424604F1100190
:1053600009F1040004F0F2FD608A00FB08F0001D62
:10537000ADF80300494600A801F0B4FFA7EB080709
:10538000BFB2002F03D0B742E1DBB046E0E705B083
:10539000BDE8F08330B587B004460D468B4850F821
:1053A0002400FFF7BBFF002D13D001A80FF2C4218A
:1053B0001422FDF79BF800A80FF2CC210A680260C6
:1053C0008DF802400320ADF8070000A901A801F004
:1053D00089FF07B030BD30B583B000A80FF250216F
:1053E0000CC90CC000240FE0784800A9615C50F89B
:1053F0002150002D07D02846FFF77CFC002802D062
:105400002846FFF78BFF641C052CEDDB37BD6F4989
:1054100051F82000002804D0406A002801D0012063
:10542000704700207047694951F82000002802D1D8
:105430004FF0FF30704790F82810481E8041C0435D
:10544000C00F40B27047614951F82000002804D0D5
:10545000006A002801D0C0687047002070472DE91D
:10546000F0410446012510E0584850F82500002876
:105470000AD0D4E90067012000212A4601F022FE6B
:1054800030433943C4E900016D1C372DECDB04F1D6
:10549000080681271EE04D4850F82700002818D044
:1054A000A7F18002501102EB90604FEAA0185FFA5A
:1054B00088F806EBC800D0E9004501200021A2EBE6
:1054C000881201F0FFFD2043294306EBC802C2E920
:1054D00000017F1CCE2FDEDBBDE8F0812DE9F0411D
:1054E00086B007460C4600A80FF2A0111422FCF764
:1054F000FDFF4FF4FE7004F015FA050019D121E00C
:105500003E462E2010FB06F81FFA88F808F102002C
:10551000ADF80300412028706E7042462146A81C59
:10552000FCF7D4FF294600A801F0DCFE4444BF1B71
:10553000FFB2002F03D00C2FE2DB0B26E1E7284659
:1055400004F008FA06B0BDE8F08138B5044601253C
:105550000CE01E4850F82530002B06D022460021D2
:105560004820DB695B6998472E346D1C372DF0DBD2
:1055700031BD70B500240120144A00E0401CC0B2C7
:105580000146372906DA52F821100029F6D0641CAA
:10559000E4B2F3E720462E2111FB00F5ADB2284618
:1055A00004F0C0F906000FD000222946FCF7DAFF0C
:1055B0003046FFF7CAFF31462046FFF78FFF3046DF
:1055C000BDE8704004F0C6B970BD00005CAF0300D8
:1055D0006055030080560300C867030038B7030016
:1055E00023612025642C25642C256400237220254A
:1055F000642C25642C25640023632025642C2564F9
:105600003E256400617272616E67655F64617461FA
:105610005F7061636B65740025733A2074785F6412
:105620006174612069732066756C6C28256429009B
:10563000010E061208000000050000000000000036
:105640000000000000000000000000000500000055
:10565000000000000000000000000000000000004A
:105660000500000000000000000000000000000035
:105670000000000005000000000000000000000025
:10568000000000000000000005010000050000000F
:10569000000000000000000000000000000000000A
:1056A00010B500224FF4A871DFF88809FCF7E0FE7E
:1056B000DFF88449002218212046FCF7D9FE00209B
:1056C000606210BD0020704710B5DFF8704900F02F
:1056D0007FFCA060002204F11C018320FFF798FBEF
:1056E000002801D0032010BD002204F11C01BC20C1
:1056F000FFF78EFB002801D0032010BD002204F12B
:105700001C010120FFF784FB002801D0032010BDFD
:10571000002010BD10B5DFF82449002204F11C015F
:105720008320FFF7D1FB002801D0032010BD002209
:1057300004F11C01BC20FFF7C7FB002801D00320A7
:1057400010BD002204F11C010120FFF7BDFB002861
:1057500001D0032010BDFFF7A3FF002010BD000003
:1057600038B52DED028B84B09FEDB68ADFEDB58A9A
:10577000DFF8C848A0693C30A0612068022801D049
:10578000032809D1DFF8B8080069216981420CDAE1
:10579000401A08EE100A08E0042802D1DFEDB78AAB
:1057A00003E0052801D1DFEDB68ADFF8940800692F
:1057B0002061DFF88058B8EE480AD5ED530A30EE84
:1057C000200A30EE280A85ED530ADFEDAE0AB4EE6A
:1057D000600AF1EE10FA09DBDFEDCF0A30EE200AA5
:1057E00085ED530A0FF6700001F07EFCA06947F2C8
:1057F0003051884214DBD5F84C0101F043F8CDE973
:10580000020118EE900A01F03DF8CDE9000118EE12
:10581000102A21680FF6540001F066FC0020A061F8
:1058200004B0BDEC028B31BD70B500F0B1F9FFF7EB
:1058300097FF00F09BF900281BD0DFF8F84704F52C
:10584000C4704568D4F88861701B04F0E3FE034619
:105850002A4631460FF6440001F046FC0020A060C5
:10586000DFF8D807DFF8D8171822FCF73FFE002032
:1058700070BD00F0E9F8002805D0DFF8BC07416AE8
:1058800041F00401416200F0FFF8002805D0DFF884
:10589000A807416A41F00101416200F019F90028AE
:1058A00005D0DFF89407416A41F00201416200F03F
:1058B00035F9002805D0DFF88007416A41F008017A
:1058C000416200F026F800F046F800F0B1F800F070
:1058D0003DFA002070BD80B500F097FA002002BDAF
:1058E0003EB500A900231C461D4638C1002A00D140
:1058F00000AA3D2802D03E2805D008E00621104627
:1059000000F019FB03E00621104600F043FB20469F
:105910003EBD38B5DFF81C47DFF81C0790F82400BF
:1059200000F01B0084F8400100F052FB009004F2EC
:105930004115042200A92846FCF7C8FD0421284689
:1059400000F038FB04F5A070DFF8F4160A68427125
:105950004968817131BDFEB50026DFF8E046DFF809
:10596000E056A868A168401A00F094FA02902068F6
:105970002968884205D0029841F28831884200DBCC
:1059800001260298DFF8BC16884200DB0126DFF80A
:10599000A80690F91210002906D000218174416AEE
:1059A00041F0040141620126002E40D0DFF88466F8
:1059B000B06800EB80018F1D00280BD1042204F198
:1059C000080106F10D00FCF781FD042106F10D0030
:1059D00000F0F0FAB068401CB06070742068B9192B
:1059E0000873781C471C0299DFF85C26914203DBA0
:1059F00002218019017302E0002180190173042241
:105A000002A9B8190C30FCF761FD0321B8190C305C
:105A100000F0D0FA02980190A86800902B68A26864
:105A200021680FF29C6001F05FFBA868A060F7BDE1
:105A3000DFF80806DFF808164A6842600968016066
:105A40007047000000000000DFF8E805DFF8E81507
:105A500091F90010012903DA00218160084670479E
:105A600081683B2905DA012905DB90F984010028CA
:105A700001D0012070470020704700006ABCD43F6D
:105A8000FA7E2A3F4154094BDFF8A80590F98401BA
:105A9000002819D0DFF8A00590F90810012913DBC0
:105AA00090F91310012903D10021C174012070471E
:105AB000DFF88C05DFF884150A6803689A4205D17F
:105AC00049684068814201D1002070470120704739
:105AD000DFF86405DFF86815DFF8602512680B68E9
:105AE0009A4201D00022027490F91020002A01D0BD
:105AF000002070471A46121892F90120012A01DA93
:105B0000002070474968012903DB01210174084620
:105B10007047002070470000405409CB10B5DFF8F3
:105B20001845DFF81C05DFF814150A6803689A4267
:105B300001D00022627494F91120002A01D00020C3
:105B400010BD0A68121992F90920012A01DA002011
:105B500010BD80688968401A00F09CF9616988422C
:105B600002DB0120607410BD002010BD80B5DFF89D
:105B7000C404D0F88C11D0F88801081A04F04AFD4A
:105B800042F21171884201DB012002BD002002BDFA
:105B900030B591B001A804F0BBFE00A806F048FAA9
:105BA00000F094FB012801D1012000E00020DFF883
:105BB000844484F88401D4F85001401C6FF0704193
:105BC00090FBF1F1C1EB0171401AC4F8500100F0F3
:105BD000FFF9DFF86C54A86068619DF800000428A4
:105BE00005D1042028609DF80100686021E0BDF81F
:105BF0000600022810DB042802DB0320286001E0F5
:105C000002202860BDF80A0068609DED0E0ABDEE16
:105C1000C00A85ED040A0CE0D4F85001042806DB24
:105C20000120286001A800F013F8686001E000205E
:105C3000286000F0CDF9D4F8501101EBD172521068
:105C4000A1EB420104EB8101C1F8880111B030BD24
:105C50002DE9F04186B00446DFF8D853D5F85061FD
:105C600000A81421FCF77AFC00A9012003F07BFFB7
:105C70000C20711006EB91718910A6EB810100FBDD
:105C80000151009AC1F8542101F5AA71019A4A60A4
:105C9000029A8A600021324600E0521E331F93426E
:105CA00039DAD31C5F1003EB9777BF10A3EB8703A0
:105CB0005F1C4FEA670C07EB9C7C4FEAAC0CA7EB30
:105CC0008C074FF0000C0BE030EE600ADFEDB00AFD
:105CD000B4EE600AF1EE10FA00DB01210CF1010CC8
:105CE000BCF1030FD9DA00FB075E0EEB8C08D8ED90
:105CF000550A00FB035E0EEB8C0E9EED550A9EEDE1
:105D0000551A31EE601AB5EE401AF1EE10FADBD5F5
:105D100030EEC00ADAE7C948C94A012901D1516900
:105D2000416151694069081A00F0B4F8C6498842D7
:105D300001DB022007E0E088022801D0012801D120
:105D4000012000E0002006B0BDE8F08170B5BA4C3B
:105D5000606A10F01B0F23D0B64E00F01B0086F8CF
:105D6000400106F5A071E161072060839A2020833D
:105D7000B64D0120287068701A20A8700722E81C10
:105D8000FCF7A4FB606A20F01B006062608BC01C03
:105D9000216A488229469A20BDE8704003F0ECBD94
:105DA00010F0240F30D0A34E00F02400307306F121
:105DB0000C00E061B0683B2801DB3B20B060B068BC
:105DC00000EB8000801D60839A2020839F4D01207E
:105DD000287068701A20A870628B06F10C01E81C0C
:105DE000FCF774FBB1680FF2003001F07DF9002080
:105DF0006062B060608BC01C216A488229469A208C
:105E0000BDE8704003F0B8BD70BD10B4012821D1C9
:105E10008A49894890F908200B6814461C41E2071A
:105E200003D5426A42F0010242621A46121892F900
:105E30000120012A03DB426A42F002024262194653
:105E4000091891F90910012909DB416A41F008019B
:105E5000416204E0022802D101207749887410BC15
:105E6000704700B583B076494A688DF801208A688A
:105E7000CDF8022009688DF8001000A90622FCF771
:105E800025FB0EBD6B4890ED530ABCEEC00A10EE28
:105E9000100A7047002801D56D490818002800D560
:105EA0000020704780B5002805D0022825D009D3EE
:105EB000032825D001BD60480272012A3AD1012190
:105EC000C17401BD012007E00B460341DB0702D589
:105ED000594BC3185A70401C0628F5DB564890F9F8
:105EE0000510009190F9043090F9032090F9021008
:105EF0000FF20C2001F0F8F801BD4F48027001BD0F
:105F0000012007E00B460341DB0702D54A4BC318CB
:105F10005A72401C0628F5DB474890F9051000919D
:105F200090F9043090F9032090F902100FF2F0106C
:105F300001F0DAF801BDF8B5044625782679207A13
:105F40008DF80000607A8DF80100A07A8DF80200CB
:105F5000012231462846FFF7A5FF374F032D07D111
:105F6000E079217A083188404FF47A7148437861AA
:105F700000A800F009FA79690FF2C81001F0B4F82E
:105F8000324629460FF2D81001F0AEF8F1BD0000FC
:105F90009B99993E38B50478057900222946204618
:105FA000FFF780FF2A4621460FF2D410BDE83840A3
:105FB00001F09AB810B40022491E05E0135C0C5C95
:105FC00014540B54521C491E8A42F7DB10BC704714
:105FD00000B583B00FF2C410D0E90023CDE900234F
:105FE00000A800F0DBF99DF900001A499DF9012095
:105FF0004EF660235A4301FB00209DF902104FF436
:106000007A7211FB0200BDF9041000FA81F00EBD96
:10601000094908622831C1619A2101703C218160DF
:106020000121017301820021418208494161002060
:106030007047000038C2030008670300F4690300DA
:106040000CD7030000BADB0020BF020048C80300E1
:10605000005C260580EE360041522044697374616D
:106060006E63652052657365740A0000534C6F635C
:1060700041525F547970653A25642C2064697374C9
:10608000312025642064697374322025662C2073C6
:106090002D446973742025660A0000002C203236D6
:1060A0002041542057726F6E672054696D65737478
:1060B000616D7020256420256420256400000000A7
:1060C0002C203236204154204348474D4F44205B1A
:1060D00025645D3A2564202D3E205B25645D3A25CC
:1060E00064202564000000002C203236204154201A
:1060F000626174636873697A65202564000000003A
:106100002C20323620415420616464496E744D6FF6
:106110006465202564202564202564202564000012
:106120002C203236204154206164644578496E74D5
:106130004D6F646520256420256420256420256436
:10614000000000002C203236204154206578496E32
:10615000744475726174696F6E202564202000009C
:106160002C20323620415420726563656976655370
:10617000746172744D7367202564202564000000EB
:106180002C2032362041542072656365697665455E
:106190006E644D73672025642025640000000000B4
:1061A0000000000000B585B000A80FF23C51142299
:1061B000FCF79CF900A806F0B2F8002803D00FF213
:1061C000F04000F091FF05B000BD80B50020DFF881
:1061D000B41448718DF8000000A9082003F0D9FF1D
:1061E0000FF2D84000F080FF01BD10B5DFF89444F5
:1061F0004FF47A72DFF8901404F1240006F0F1F8FD
:106200004FF42F72DFF88C1404F1380006F0E9F82F
:10621000002010BD7047DFF88004704710B586B0CD
:10622000044601A81421FCF799F9FFF7F4FF009048
:106230000D22214601A8FCF749F90420ADF807001A
:1062400000A901A801F04EF806B010BD10B58CB041
:10625000044606A81421FCF781F900A81821FCF7D0
:106260007DF90D22214606A8FCF730F900A8FFF7BA
:10627000F6F81820ADF81B0000A906A801F032F8C6
:106280000CB010BD10B5DFF8FC4360702078012819
:1062900008D16078082805D1FFF79DF80FF2284053
:1062A00006F008F96078042802D10120207003E08C
:1062B000082801D100202070611C0720BDE8104093
:1062C00003F067BFDFF8BC0300787047DFF8B40362
:1062D000C0787047DFF8AC034079704770B50400B0
:1062E0003AD0DFF8A053D5E90401002901D10028F4
:1062F0000ED0D4F80520D4F80930101A63EB010150
:10630000DFF888230123994202D825D3904223D372
:10631000DFF888633078401C3070802080F311886B
:1063200000BF00BF7078401C707003F0DFFAD4F833
:106330000520D4F80930C5E90423C5E906017078C1
:10634000401E7070C0B2002802D1002080F3118876
:10635000BDE8704004F0AAB870BDCA49D1E9042371
:10636000C0E90023D1E90623C0E90223704738B50C
:1063700003F0BCFAC34AD2E9044520186941D2E9C6
:106380000645001BA94134BDBE4902780A72427815
:106390004A72807888720020888170470622C0493E
:1063A000FCF794B810B5044603F0ABFEB5490A6A91
:1063B000002A01D0A21A00E00246B2F57A7F00D38B
:1063C000024688891018888100B2B0F57A7F05DB13
:1063D000A0F57A708881887A401C887291F90A0049
:1063E0003C2804DB3C388872487A401C487291F99A
:1063F00009003C2804DB3C384872087A401C0872CB
:1064000091F90800182801DB002008720C6210BD09
:1064100010B5142801DA022400E00A24042801DA65
:10642000022010BDA12801DBA02010BD90FBF4F0DC
:1064300006F052F841EC100B06F066F851EC100B28
:1064400006F06CF806F048F841EC110B9FED950B47
:1064500006F0D3FA51EC100B06F060F8604310BD63
:1064600000B587B002A80FF294211422FCF73EF881
:1064700000A800210A4606C003F096F801788DF8BE
:10648000001000A9C2784A7042798DF80220807904
:10649000C87001208DF804000520ADF80B0002A89B
:1064A00000F020FF07B000BD30B59FB005A8642103
:1064B000FCF754F800A80FF258211422FCF716F844
:1064C0000024FF22642105A8FBF7D2FF012517E075
:1064D0002846C0B2FEF7BFFD002810D02946491E4D
:1064E000012906D9C91E022903D9091F01D01A3969
:1064F00005D105A964B26554408A401C04196D1C7D
:10650000092DE5DB64B2ADF8034005A900A800F051
:10651000E9FE00201FB030BD38B50446A078014622
:10652000491F1CD0491E1DD0491E012927D9891E8B
:1065300001292CD9203907D00F390AD0491E4AD059
:10654000491E01292CD94BE0D4F80D00FFF71CFFA0
:1065500046E0B4F80300C0B2FFF794FE40E04C48B8
:1065600005F04BFFA078052801D1012000E00020B4
:10657000444DE870E91C062003F00BFE30E00728CC
:1065800001D1012000E000203E49087128E03D4D86
:10659000092802D10020A87022E00120A8701FE085
:1065A000384D3A280ED141A000F09EFD01206871BF
:1065B00005F1380005F04CFFD4F80D10082003F069
:1065C000E8FD0DE00FF2181000F08EFD05F1380027
:1065D00005F013FF04E0D4F80D10012006F0D5FCFF
:1065E000A0781438032801D915380FD18320FEF77D
:1065F00032FD03000AD0D4F80D20B4F80310A078BF
:10660000DB691B6901B0BDE83040184731BD80B57A
:1066100081780C2908D018290FD01B2907D02C29E4
:106620000ED031290FD001BDBDE80240F6E5FFF7DD
:106630000DFEBDE80140FEF79CBFBDE801400FE73D
:10664000BDE8014030E70F480078002803D1BDE8DD
:10665000014000F0B1BD01BD80B500208DF8000003
:10666000481E042802D201208DF8000005489DF83C
:1066700000108279914204D0817100A9052003F0B5
:1066800088FD01BD88D20300A571000000F2052A33
:10669000ACD20300CB7100009C9E5001C867030080
:1066A00090D2030000000000000000404D4F4E005B
:1066B000736B697020524349000000004D4F4646FD
:1066C000204342210000000023212120617020731B
:1066D00074617465206368616E6765210A0000005B
:1066E0004D4F46460000000004FF3100000000004E
:1066F00000000000000000000000000004FF18007F
:106700000000000000000000000000000000000089
:1067100004FF2C000000000000000000000000004A
:1067200000000000DFED4A0A60EE200AB0EEE01A39
:10673000DFED481A00B5B4EE611AF1EE10FA83B03D
:1067400036D5F5EE400AF1EE10FAACBFB6EE001AFF
:10675000BEEE001A70EE810AFDEEE00A10EE900A1D
:10676000A8B1FAEEC90A9FED3C1A00EEC10A9FEDEE
:106770003B1A00EEC10A9FED3A1A00EEC10A9FEDE6
:10678000391A00EEC10A9FED381A00EEC10ADFED9A
:10679000370AB4EE600AF1EE10FA00F003003ADBBB
:1067A000DFED330AB4EE600AF1EE10FA33D51FE0E4
:1067B0008DED000A0098C0F3C750FF2820D010B913
:1067C0000098400241D08DED010A01A806F008FCB6
:1067D0009DED010ADFED250AB4EE600AF1EE10FA34
:1067E00019DBDFED230AB4EE600AF1EE10FA12D5E0
:1067F000C0072AD5FFEE000A80EE800A03B000BD74
:106800000098400221D106F061FC212101609FED3A
:10681000190A03B000BD60EE000A9FED171ADFED04
:10682000171A40EE811AB7EE001A01EEA01A60EEB8
:10683000200ADFED131A00EEA10AC00746BF81EE61
:10684000000AB1EE400A80EE010A03B000BD00006C
:1068500083F9223F0000004F0000C94600A0FD4020
:106860000020A23A000034330030C22EFEFF7FB970
:1068700000008039FFFFFF7F6D161F3C1EB5DBBE99
:106880008329C4BD5FF0FF0C1CEAD05114BF6145E1
:1068900006E0C110400721F0E04101F1605170476E
:1068A00079B900F0004100020AD0B0FA80FC00FA89
:1068B0000CF001F16051A1EB0C5101EBD02140052E
:1068C000704741020CBF40F4E0016FF0000100206E
:1068D00070470000B0B581EA030C0CF0004C40F2A8
:1068E000FF7515EA11541DBF15EA1357AC42AF42AC
:1068F00039E0E41923EA455343F48013C90241F017
:10690000004141EA505EC7021100A7FB02020028C5
:106910004FF00000EEFB01204FF00001E3FB0721E8
:1069200018BF42F00102401800214941E3FB0E016B
:10693000A4F580640F0302D252004041494154F152
:1069400001046CDD470872F1004250F1000051EB88
:106950000451A1F580115CBF41EA0C01B0BD4CEAC5
:1069600005510020B0BD05EA1357AC4214BFAF4239
:1069700041E050EA410E1CBF52EA430E02E061467C
:106980000020B0BD24423C441BD15FEA070EF6D084
:10699000090302BF01460020AEF1140EB1FA81F7DF
:1069A000AEEB070401FA07FE0C37C7F1200100FA2D
:1069B00007F7C8404EEA000E23EA455343F480131C
:1069C000A2E733F00043B3FA83F704BFB2FA82FEC2
:1069D00077440B3FE41BB7F1200E2FBF02FA0EF3F2
:1069E000BB40C7F1200E22FA0EFE38BF43EA0E0369
:1069F000BA40641C82E750EA410E14BF52EA430ECB
:106A00006FF000014FF4001717EB430F8ABF1946D0
:106A100017EB410FB5E74CEA05510020B0BDD4F1AA
:106A20000104B4F120070FDAC4F12007520828BF8F
:106A300042F0010210FA07F501FA07F7E1BF2A4315
:106A4000E0403843E1400FE0352C98DCC7F12004EA
:106A500052EA400220FA07F218BF42F0010231FA6E
:106A600007F0A1400A43002172F1004250F10000FA
:106A700051EB0C01B0BD000010EE101A10EE902A80
:106A8000B0EEC00AC80F49005200F0EEE00A28BF7D
:106A90000C3011F1807F38BF12F1807F0CD28A4216
:106AA00038BF80F00400124214D034BF80EE800A58
:106AB00080EE200A06F010BB11F1807F08BF80F045
:106AC000040098BF12F1807F08D88A4214BF0022C8
:106AD0004FF07E5200EE102A06F0FEBA6FF0004131
:106AE00000EE101A7047012006F048BB002006F0A7
:106AF00045BB000051EC100B00B500F003F841EC71
:106B0000100B00BD40F2FF7C0B0D4DD0634566D2EB
:106B100030B421EA035141F4801103F2FD3C5FEAF5
:106B20005C0C01D300184941890041EA9071800052
:106B30004FF440140023E202D50AB1F5100107D446
:106B40006D081DD2091B641900184941491BF7D56E
:106B50006D080AD20919641B00184941491BEFD579
:106B60006D08F7D301E0520817D0C01861419B1A95
:106B7000AC4100184941801AA941F4D452080AD006
:106B8000C01AA1419B186C4100184941801AA941C3
:106B9000E9D45208F4D15B1C6C4161084FEA330020
:106BA00001EB0C5130BC704750EA0103FBD030B40C
:106BB000B1FA81F311B9B0FA80F41B190B3BB3F1B0
:106BC00020042FBF00FA04F19940C3F1200420FAF9
:106BD00004F438BF21439840D3F101039DE7634596
:106BE000E1D011F5801FDED850EA4101DBD0D94356
:106BF00006F07ABBF0B540F2FF7581EA030C0CF0A9
:106C0000004C15EA11541DBF15EA1357AC42AF42B0
:106C1000E5E0BC41C1F31301C3F31303801A9941AA
:106C200043F4801304D2641E400049418018594146
:106C3000C90241EA5051B1FBF3F603FB1611A2FB66
:106C40000675D7EBC020A94102D2761E80185941A3
:106C5000C90241EA5051B1FBF3FE03FB1E11A2FB36
:106C60000E75D7EBC020A94103D2AEF1010E8018FA
:106C70005941890241EA9051760546EA8E2EB1FBD0
:106C8000F3F603FB1611A2FB0675D7EB8020A94192
:106C900002D2761E80185941C90241EA50514EEA8B
:106CA000060EB1FBF3F603FB1611A2FB0675D7EB3C
:106CB000C020A94102D2761E80185941C90241EA7A
:106CC0005051B1FBF3F703FB1711A2FB0735D3EBD0
:106CD000C020A94167F100070CBF004247F001073F
:106CE00066F3D5274FEA1E31B80814F5806412DD2B
:106CF000BD0775F1004250EB0E5051EB045111F5F8
:106D0000801F5CBF41EA0C01F0BD4CF07F6141F097
:106D1000E0410020F0BDBD076D0840EA0E5041F48F
:106D20008011D4F10104B4F120060ADAC4F120067E
:106D30000200E04001FA06F3E1401843B240154377
:106D40000EE0342C13DCC6F1200445EA40056D0842
:106D500020FA06F2154321FA06F0A1400D43002166
:106D600075F1004250F1000051EB0C01F0BD002024
:106D70005FEA0C01F0BDCFB992185B41B3FA83F71B
:106D800004BFB2FA82F6BF190B3FB7F120062FBF3E
:106D900002FA06F3BB40C7F1200622FA06F638BF16
:106DA0003343BA401CB1E419641E33E77F4231F02B
:106DB0000041B1FA81F404BFB0FA80F6A4190B3C8B
:106DC000B4F120062FBF00FA06F1A140C4F120065D
:106DD00020FA06F638BF3143A0403C1B1AE7AC420C
:106DE0001ABF05EA1357AF4212E050EA41061CBF32
:106DF00052EA4306BFE750EA4107304661461CBFEE
:106E000041EA0551F0BD52EA430C08BFC143F0BD51
:106E100000204FF4001616EB410F98BF16EB430FFE
:106E200008BF16EB410F24BFC14305E016EB430F2B
:106E30000CBF61464CEA0551F0BD000070B44FF044
:106E4000004591EA030F44BF6B4000F0C1B800BF9A
:106E5000841A71EB030604D26E40001BB141121973
:106E600073414FF4001C1CEB410F34BF7CEB430615
:106E700084E00C0DA4EB1356362E7DDC012E43DC92
:106E800045EAC32343EA525312BFD20292025B087F
:106E9000240545EAC12141EA5051D2EBC020994175
:106EA00025D407D1B0FA80F610FA06F164D000209C
:106EB000203608E0B1FA81F6B140C6F1200220FA8E
:106EC00002F21143B0404FEAF474B4EB465434F08C
:106ED00001064FEA74040AD8D6F50016760D04F0C0
:106EE0000044F04061FA06F25040F1404840C00AC8
:106EF00040EA415021F0004128BF5FEA500550F1BF
:106F0000000044EBD12137E045EAC323DB0A45EA20
:106F1000C121C90AB6F120050EDD42EA0242120C77
:106F2000C5F1200603FA06F6EB4042EA06056D427B
:106F3000984161F100010DE062FA06F5F24055401A
:106F400063FA06FC82EA0C02F3405A406D4290411B
:106F500061EB030111F4801F05D1641E620502D0AC
:106F60006D004041494121F48011430875F100430F
:106F700050F1000041EB045170BC70471CEB410F15
:106F800015D223F0004352EA43060BD04FEA4C0CD3
:106F9000BCEB410F04D80C0D661E342EB7DDEBE7B9
:106FA000801A994150EA410608BF0021E4E708BF72
:106FB0001CEB430F28BF6FF00001DDE770B44FF00A
:106FC000004591EA030C44BF6B40FFF741BF00BF8F
:106FD000841A71EB030603D2001BB14112197341ED
:106FE0004FF4001C1CEB410F34BF7CEB430443E027
:106FF0000C0DA4EB1356352E50DC45EAC323DB0AF7
:1070000045EAC121C912B6F120050DDD63FA05F686
:10701000EB4086EA0305124218BF45F00105C0188F
:1070200051F100010CD213E062FA06F5F24055402E
:10703000F3415A40B340F3405A408018594107D3B6
:1070400049085FEA30005FEA350528BF45F00105D1
:1070500001F58011420875F1004250F1000041EB4A
:10706000045170BC4FF4001C1CEB410F38BF70473B
:107070000020090D090570471CEB410F10D252EAA0
:1070800043060BD0BCEB410F05D80C0DAB43661E7D
:10709000342EB5DD02E0AB438018594170BC704717
:1070A00070BC7047D2B2203A22BF21FA02F0002110
:1070B00070472032D141D04048409140D1404840B3
:1070C00070470000D2B2203A22BF00FA02F100203D
:1070D00070475242D041D2F1200291404140D0400D
:1070E00090404140704700000EB470B5C1B00446F6
:1070F00000A84FF48071FBF731FA45AB22464FF4FC
:10710000807100A806F0F6F800A806F011F9441CFA
:10711000002000A9611801F8010C644D2878401C7A
:107120002870802080F3118800BF00BF6878401C61
:1071300068705F4E317808462218F22A0DDA5D4AEF
:107140008018002902D00A2100F8011C224600A95B
:10715000FBF7BCF93078201830706878401E6870F2
:10716000C0B2002802D1002080F3118803F09EF9FC
:1071700041B070BC5DF810FB4D480078002801D08C
:10718000801C00E00020C0B2704738B5484C22781F
:10719000002A10D000280ED0032101704270454D06
:1071A0002946801CFBF792F90022F2212846FBF7C2
:1071B0005FF90020207031BDF0B595B004A80FF242
:1071C000FC010CC90CC0922002F0ACFB040004D1FD
:1071D0000FF2F000FFF788FF65E000229221FBF735
:1071E000C1F9002517E000208DF802009DF802008B
:1071F000002803D0C868019008690290306A00280E
:1072000001D0C0680390102200A904EB0510801C77
:10721000FBF75CF96D1C072D16DA04A82F5C3846C5
:10722000FDF719FF0600F5D000A81021FBF796F92D
:107230008DF8007006F12000017A8DF80110416888
:107240000029D0D00120CFE70CA82021FBF786F938
:10725000194800680C9002F054FF0D90FFF732F8C7
:107260008DF838000DF13A00FFF798F810A8FFF7F5
:1072700074F820220CA904F17200FBF727F906A884
:107280000FF24C011422FBF731F99220ADF81B00EC
:107290003120207007206070214606A800F022F8F7
:1072A000204602F057FB15B0F0BD0000C867030090
:1072B00069D90300ACCA0300006E02000102040594
:1072C00008108300524349206661696C0000000089
:1072D00005000000000000000000000000000000A9
:1072E000000000002DE9F04705460E46B5F8037092
:1072F000334C2078401C2070802080F3118800BF20
:1073000000BF6078401C60702878052803D1FFF723
:1073100033FF804601E04FF0000808EB070000F162
:107320000D0A504602F0FEFA8146B9F1000F11D164
:1073300051460FF2940005F0BDF86078401E607071
:10734000C0B2002802D1002080F31188BDE8F047C8
:1073500003F0ACB8B5F803004044A5F803000D22D3
:1073600029464846FBF7B2F83A46314609F10D0086
:10737000FBF7ACF8B8F1000F04D007EB09000D30B3
:10738000FFF703FFB5F8030000F10D0189B248468D
:1073900002F0FBF96078401E6070C0B2002802D194
:1073A000002080F3118803F081F8B9F1000F04D0B8
:1073B0004846BDE8F04702F0CDBABDE8F0870000CE
:1073C000C867030002F0DBB974786275666665729F
:1073D000206973206E6F7420616C6C6F63617465DB
:1073E000642825642921210A0000000080B50FF6D9
:1073F0008430FCF747FDDFF8480B00210170017471
:10740000C1603C21416000218160012101754FF084
:10741000FF31C1610121417501BD38B5DFF8204B55
:10742000DFF83C5B2878022801D104202070207806
:10743000012807D0C0F08A8003284AD01BD3042833
:1074400067D031BDDFF8F00A90F82810C9070AD5D7
:1074500090F82A00C00779D500F036F90020BDE881
:107460003240FBF7F1B800F03CFA61680020BDE85B
:107470003440FBF7ABB8287803281CD1207D0028C6
:107480000AD0002020753C20606001460020FBF7F8
:107490009DF80120207031BD022060750121FBF7AD
:1074A000BFFB607800F10A0206210120FBF7C0FF54
:1074B0000220207031BD042848D14FF496706060DE
:1074C0000020A0604FF49671FBF780F80120207037
:1074D00031BDDFF8845A2888401C288080B23228C9
:1074E00034DB00F041F8607D022801D100F0C5F8DE
:1074F000606801280ADAA068012802DBE069002838
:1075000004D14FF0FF30E06100F0DEF80020288069
:1075100031BD95F82000012801D0032817D10120A2
:10752000607500F0DEF904F1280105F1080000F0B3
:10753000FCF80120207584F8200060683C2190FB55
:10754000F1F1C9B2A068BDE83440BBE231BD062804
:1075500001D00528E5D160780128E2D10521E06855
:10756000BDE83440AEE20000F8B5DFF8D069F56858
:10757000DFF8CC497078012834D1B07802281EDABF
:10758000DFF8C0793878002830D0607801282DD015
:1075900097ED010ADFEDBB0A30EE200A87ED010A04
:1075A000F7EE000AB4EE600AF1EE10FA1EDB6D1C75
:1075B000FFEE000A30EE200A87ED010A16E015D131
:1075C000DFF880793878002809D06078012806D063
:1075D0000FF6AC10FCF756FC0020A06060600020A5
:1075E000387003E00120DFF85C19087094F820007F
:1075F000002824D0707804280FD194ED020AB8EE48
:10760000C00ADFEDBE0A80EE200ABDEEC00A84ED9E
:10761000070A002084F8200016E0052814D194ED14
:10762000020AB8EEC00ADFEDB60A80EE200ABDEE0F
:10763000C00A84ED070A002084F8200004E0E06915
:10764000012801DB401EE061A068012808DB012D54
:1076500002DB401BA06003E0002D01D50020A060EC
:107660006068012801DB401E6060A26861680FF657
:107670003410BDE8F840FCF705BCDFF8C4088169A8
:10768000002920D0012902D1002181608161DFF829
:10769000AC184A78012A12D18978022908DADFF871
:1076A000BC18097800290ED08169491E8161704794
:1076B00009D10021DFF8A4281170816170470120F1
:1076C000DFF898180870704710B50FF6F400FCF753
:1076D000D9FBDFF874080078002805D00FF6EC001D
:1076E000BDE81040FCF7CEBBDFF85448607D0128B0
:1076F00003D0FBF70EFD002809D001210846FBF757
:107700008FFA0A2201210846FBF792FE0AE00121C6
:107710000220FBF785FA607800F10A0206210120B9
:10772000FBF786FE0220207010BD2DE9F8432DEDF9
:10773000028B82B004460D46DFF804686FF000400B
:10774000B060002712E030EE480AD6ED020AF8EEEB
:10775000E00AB4EE600AF1EE10FA06D5BDEEC00AFA
:1077600086ED020A38F8050070827F1C142F3BDA80
:10777000282000FB07F808EB050999F8020000280B
:10778000F3D099F803000028EFD1D9ED031A99ED51
:10779000021AD4ED010A94ED000AFBF7CFFEB0EE19
:1077A000408ADFF8BC078078002803D1384680B2D1
:1077B00000F032F818EE100AFFF764F8CDE9000186
:1077C000D9F8202038F805100FF61800FCF75AFBFE
:1077D00099ED080AB8EE400AB4EE480AF1EE10FA44
:1077E000B1D538EE400AB0E70220707000210CE0FD
:1077F000282000FB01508278002A05D090F8240050
:10780000012801D101207070491C1429F0DB02B05D
:10781000BDEC028BBDE8F183DFF8241700EB80029A
:1078200001EBC201088DD1ED120AF8EE600A91F861
:107830004C20002A03D0022A19D006D37047F4EE58
:10784000400AF1EE10FA17D50CE0DFF8142792ED9C
:10785000071AB8EE411A71EE200AF4EE400AF1EE72
:1078600010FA0ED5022281F84C2011460CE0B4EE3D
:10787000600AF1EE10FA04D5012281F84C2011467D
:1078800002E070471F852B3F38B504460D462A4657
:1078900021460FF27070FCF7F5FADFF8B0060480AD
:1078A00085709FEDA80ADFF8B816D1ED020A60EEE8
:1078B000800AFDEEE00AC0ED010AD1ED030A20EED8
:1078C000800ABDEEC00A80ED020AC969C1601020BD
:1078D000FCF77EFD224629460420BDE83840FBF730
:1078E000A7BDDFF85C06417D012902D13C21416042
:1078F00070474FF49671416070470000CDCC5C41F9
:10790000CDCCDC402DE9F8432DED028B054608EE89
:10791000101A08EE902A1E464FF0FF370A9CA04628
:107920004346324629460FF2F460FCF7ABFA0020DA
:10793000DFF80C9605E017F1010F0BD107463FB2B7
:10794000401C14280BDA282101FB009191F82A2011
:10795000002AF0D0098DA942F2D1102068E099F8F0
:107960001000142801D1122062E017F1010F01D19B
:1079700002205DE0282101FB0790058500F1280128
:10798000B8EEC80ADFED6F0A80EE200A81ED020A28
:10799000B8EEE80A80EE200A81ED030A0E6280F854
:1079A0004C400120887099F81000401C89F81000A4
:1079B00099F80000002802D1012089F80000002C6D
:1079C0002BD1002089F8010099F8000002282ED060
:1079D00099F8150001282AD10020FAF735FEDFF8C2
:1079E00068050078002808D00020C9F80400C9F80C
:1079F0000800032089F8000019E001210846FBF780
:107A00000FF90A2201210846FBF712FD022089F82E
:107A10000000012089F8140009E0B8F1010F06D137
:107A200099F80100002802D0012089F80100002007
:107A3000BDEC028BBDE8F28338B5054629460FF24E
:107A4000FC50FCF71FFA4FF0FF30DFF8F44402213E
:107A5000617000210AE092F82A30002B05D092F8DC
:107A60004C20012A01D101226270491C142907DA35
:107A7000282202FB0142138DAB42ECD10846F4E709
:107A800000B210F1010F1BD0217C491E2174282265
:107A900012FB0040002180F82A100A4628212830D5
:107AA000FAF760FD207C002808D100202070FAF74A
:107AB000CBFD0120FBF70AF9FFF798FC002032BD4F
:107AC000112032BDF8B504460D462F4622460FF26E
:107AD0008050FCF7D7F9DFF868643078002801D1CE
:107AE0001320F2BD022802D10120FBF7EFF800209D
:107AF000FAF7AAFD03203070B460707D022815D11A
:107B0000C7EB07108000706040F2DC50844202D264
:107B10000020B0610FE00A20B4FBF0F0B061B0F5D6
:107B2000967F08D24FF49670B06104E03C207060FC
:107B3000012086F82000224629460520FBF778FC24
:107B40000020F2BD8096184BF8B507460C46154646
:107B50002E463346224639460FF21450FCF792F96E
:107B60004FF0FF3200200AE0DFF8D41300EB80036F
:107B700001EBC301098DB94200D10246401C142813
:107B8000F2DB12B212F1010F17D02820DFF8B01388
:107B900012FB0012946402F148030A2E05D101245D
:107BA0001C71234682F82B3003E01D71002382F8FC
:107BB0002B3002224A70002212E00FF2D840FCF76C
:107BC00061F91120F2BD00FB021393F82A40002C4A
:107BD00005D093F84C30012B01D101234B70521C7E
:107BE000142AF0DB0020F2BD30B40020014614E07E
:107BF00001EB810203EBC20292F82A40002C0BD069
:107C000000B2148D03EB4005A5F84A4392F84C20CE
:107C1000C31883F87223401C491CC94B1429E7DBA5
:107C2000187C83F848030FF2804030BCFCF72AB977
:107C300010B5C34C2078002806D0022802D10120BC
:107C4000FBF744F80320207010BDF8B52DED048B30
:107C5000044608EE101A08EE902A09EE103AFF25A5
:107C6000B6480669FBF75AFFB8EEC88AF8EEE88A0C
:107C7000BB4FF0EE681AB0EE481AD7ED030A97ED45
:107C8000020AFBF75BFC022C21D119EE100AB0F5B9
:107C9000FA7F14D9F8EE490A30EE800AF8693018F4
:107CA000B969401A00EE900AF8EE600AF4EE400A54
:107CB000F1EE10FA01DB002509E0012507E087ED70
:107CC000028AC7ED038ABE6187ED079A022528461E
:107CD000BDEC048BF2BD10B50FF2E030FCF7D2F82A
:107CE0009C4C207A002808D10FF2E030FCF7CAF84B
:107CF000FBF714FFE0600120207210BD10B50FF2F9
:107D0000E430FCF7BFF8934C00220C2104F108008A
:107D1000FAF7AEFB00202072E06020610120BDE890
:107D2000104047E080B50FF2C830FCF7ABF80020F8
:107D300000F040F88748017A012901D10021017241
:107D400001BD38B5834CA08A401CA08280B2322885
:107D500022DB0020A082794D6A6829690FF29C30ED
:107D6000FCF790F82069002805D1296921610FF2FC
:107D7000B030FCF787F86868E168401A2969226921
:107D8000891AC92902D37249884202D275498842A8
:107D900002D3BDE8314000E031BD80B50FF29C3028
:107DA000FCF770F800F015F86A480021C160016125
:107DB000017201BD80B5002804D06B48BDE80240C7
:107DC00001F02DBA002001F073FABDE8014001F086
:107DD00035BA012001F07EBA10B55E4C00220821B0
:107DE0002046FAF745FB002020706080A080A0713B
:107DF00010BD014601290BDB564A012313700129EE
:107E000003DA00F262205080704740F2592050801F
:107E10007047000038B52DED028B82B04D4CE08AE2
:107E2000401CE08280B2322840DB0020E082A08843
:107E3000411CA1806288904202D300F03BF835E0FB
:107E400089B20A2932DBA079002812D1BF20FDF7C0
:107E500002F9014600208DF80000002903D000A897
:107E6000C969496888470120A07162880146FBF70B
:107E7000DFFAFCF7C4FE054695F83C0020839FED31
:107E80003B8BD5E9002351EC180BFEF723FD04F0E2
:107E90005BFBE061D5E9022351EC180BFEF71AFDFC
:107EA00004F052FB20620420FCF792FA02B0BDEC11
:107EB000028B31BD10B582B0264C2078012816D136
:107EC000002020706080A080A071BF20FDF7C3F863
:107ED000014600208DF80000002903D000A8C969E0
:107EE000C9688847628802210120FBF7A1FA13BD07
:107EF00010B5184C2078002801D0FFF78BFF1048F0
:107F00000078002801D0FFF788FA207A002802D0F4
:107F1000BDE8104015E710BD80B50FF23820FBF723
:107F2000B1FF00224FF452710548FAF7A1FABDE8FB
:107F30000140FFF75BBA000068D5030090D603004C
:107F400078A80300D06F030020D403005CD803009E
:107F5000E193040094D40300C6D503006AD903005A
:107F600068CF030041771B00D78C000000000000A1
:107F7000D012634147465F496E69740A00000000F1
:107F800047465F41525F5420537420486967682018
:107F90006D696E5F74206D696E5F642052657365F4
:107FA00074210A0047465F41525F54206D696E5F3D
:107FB000743A25642C206D696E5F643A25640A006A
:107FC00047465F5265715F4C6F630A0047465F52D8
:107FD00065715F4C6F6320446F7A654D6F646521F6
:107FE0000A00000047465F5570646174655F442075
:107FF00069643A2564207261643A256420643A25F4
:10800000660A000047465F4465746563745F4342D7
:108010002069642025643A25640A000047465F41D0
:1080200064642049443A25642C207261643A2564D2
:108030002C206469723A25640A00000047465F52AA
:10804000656D6F76652049442025640A00000000B4
:1080500047465F53746172745F4152206D696E5F71
:10806000743A2564206D696E5F643A25640A0000E5
:1080700047465F5570646174652049443A25642021
:108080005261643A2564205374617475733A2564AF
:108090000A00000047435F5570646174655F455294
:1080A000524F520A0000000047465F5570646174E9
:1080B000655F496E666F5F43620A00004F44445F2C
:1080C0004F6E496E646F6F7243420A0068616E645E
:1080D0006C696E67204F6E496E646F6F7243420A1F
:1080E000000000004F44445F496E69740A000000BC
:1080F0004F44445F4465696E69740A004F44445FAD
:108100005052206375725F61726420256420746927
:108110006D657374616D70202564200A0000000095
:108120004F44445F505220736574207374617274BD
:108130005F6172642025640A000000004F44445FC0
:108140004F6E4465746563744F7574646F6F720A23
:1081500000000000534C435F47465F496E69740A54
:108160000000000038B504460D460FF2D810FBF7AA
:1081700089FE002C01D0002D01D1012032BD6C48B8
:1081800002210170846085818482C582002032BD15
:1081900080B50FF2C410FBF775FE65480121017030
:1081A00000218160818101BD80B50FF2C010FBF715
:1081B00069FE9FED5D0A00200090F0EE400A024645
:1081C00003465B48D0F8040000F020F8BDE8014009
:1081D00080B50FF2A810FBF755FE5548002141600D
:1081E000817301610178022903D1816881828189CB
:1081F000C18201BD80B50FF29010FBF743FE4C48E1
:10820000002141600121817301BD000038B52DEDD1
:10821000048B09EE100A14461D46B0EE408AF0EEBB
:10822000608A19EE101A0FF27010FBF72BFE41480E
:10823000B8EE490AF2EE040A20EE200ABCEEC00AAB
:1082400080ED000AC0E902459FED380A68EE000A99
:10825000FDEEE00AC0ED040A28EE800ABDEEC00A79
:1082600080ED050A089981612120BDEC048BBDE8F1
:108270003240FCF7ADB810B52F490878022806D176
:108280002E4808311822FAF731F9FFF7B3FF284CCE
:10829000208B401C208380B2322817DB00202083F3
:1082A0002748016921616168C268511861602178BD
:1082B00002290BD1A18A002909D0491EA182B4F953
:1082C0001610012903DB1046081AE08210BD202099
:1082D000FCF77EF80120207010BD10B50FF2CC0025
:1082E000FBF7D0FD124C002214212046FAF7C0F80B
:1082F0000120207000206060A073024618210F4802
:10830000FAF7B6F80120BDE81040FAF793BE80B541
:108310000FF2A800FBF7B6FD012005490870BDE883
:108320000240FAF7A4BE0000000048438096184BB4
:10833000F0D6030050D6030068CF030038D70300FF
:1083400090D60300434C5F4152445F416C61726DB3
:108350005F53746172740A00434C5F4152445F4141
:108360006C61726D5F53746F700A0000434C5F5212
:1083700065715F446973740A00000000434C5F52EA
:10838000657365740A000000434C5F4C6F635F5572
:108390007064617465640A00434C5F446973745F80
:1083A0004342203A2025640A00000000534C435FFA
:1083B000434C5F496E69740A00000000534C435FF0
:1083C000434C5F4465696E69740A000010B5DFF8BC
:1083D000D048002218212046FAF74AF800202070E1
:1083E0000120A074002060756420208200200146D6
:1083F000C4E910012083E064A06402461821DFF87C
:10840000A408FAF735F800221821DFF89C08FAF7DB
:108410002FF800221821DFF89408FAF729F8002233
:108420001821DFF88C08FAF723F800224FF4966140
:10843000DFF88008FAF71CF800221821DFF8780826
:10844000BDE81040FAF714B870B582B004460D4686
:108450001646DFF868080078009033462A46214621
:108460000FF69800FBF70EFDDFF8340844608560D6
:10847000068202210120FAF7D3FB022000F04CF91A
:108480001E220121084602B0BDE87040FAF7D0BFB5
:1084900080B50FF68C00FBF7F5FC0220FAF716FC0E
:1084A000BDE8014092E700002DE9F0478CB000EEF6
:1084B000100A00EE901A11461F46DFF8E4472078B4
:1084C000002800F0A380DDE9148942464B46F8EE0F
:1084D000E00A9FEDC71AC0EE810AB8EEC00A80EE2E
:1084E000010A06A8FBF711F8DFF8B857D5E9020131
:1084F000CDE9000142464B460FF63800FBF7C2FCBF
:10850000D5E90201894520D180451ED1207E002871
:108510001BD0401E20762846DFF88C171822F9F76A
:10852000E5FFD5E90201CDE90401686902906868B8
:10853000FEF7A8F9CDE900012868FEF7A3F9024685
:108540000B460FF61800FBF79DFC169E3346DFF82E
:108550005CA7DAE9020149450AD301D8404507D3AF
:1085600019460FF628000CB0BDE8F047FBF78ABCAF
:108570003A4619460FF63800FBF784FC052F2ED13A
:10858000DFF83457DDED071A9DED061AD5ED010A27
:1085900095ED000AFAF7D2FF0A982969461ABDEE4E
:1085A000C00A10EE107A324639460FF61800FBF773
:1085B00069FCD5E90201002901D1002809D0B81BC6
:1085C000B0F5FA7F05DD0020E0640FF61800FBF738
:1085D00059FC284606A91822F9F788FF16E006A9D3
:1085E00084B068461822F9F781FF0FBC00F07FFACB
:1085F000002E06D0284651461822F9F777FFA068CA
:10860000E06401200CB0BDE8F04785E00CB0BDE8A7
:10861000F08738B50446DFF88856287800280FD050
:108620002246297E0FF2C870FBF72CFC012028752A
:108630006C75687E297E884202D3BDE83140C8E26D
:1086400031BD38B50446DFF85856287800280AD0DE
:1086500021460FF2C870FBF715FC2046401E8041F2
:10866000C043C00FA87431BD80B5DFF83406007870
:10867000002808D0022802D10220FAF727FB0120A7
:10868000BDE8024048E001BD38B5DFF83446207847
:10869000022808D194F82000062804D0052802D02A
:1086A000032000F039F8DFF8F855287D002801D0C4
:1086B00000F042FA2878012804D02CD3032827D0D0
:1086C00003D331BDBDE8314094E020780146032951
:1086D00001DA00281FD1A87C00280AD0032908D17C
:1086E00002210846FAF79CFA1E2206210120FAF719
:1086F0009FFE2078002803D10FF23870FBF7C2FBF1
:108700006868A864A868E8640120BDE8324003E016
:10871000BDE831406AE131BDF8B52DED028B82B084
:108720000446DFF8A00590F82800000702D50320D2
:10873000F9F78AFFDFF86855012C4FD1DFF86C6537
:10874000D6E90201002901D100283BD0DFF860758D
:10875000D7E90201002901D1002833D0D7ED011A51
:1087600097ED001AD6ED010A96ED000AFAF7E6FE3B
:10877000B0EE408A30693969401A00EE100AB8EE4E
:10878000400AF2EE040A60EE200AF4EE480AF1EE26
:1087900010FA03D54FF41670E86002E04FF4E16080
:1087A000E86010EE100AFEF76DF8CDE9000118EE52
:1087B000100AFEF767F802460B460FF29060FBF7CF
:1087C00061FB06E04FF4E160E8600FF2A460FBF7A4
:1087D00059FBE9680320F9F7F9FE03E00FF2AC60FA
:1087E000FBF750FB2C7002B0BDEC028BF1BD00001A
:1087F0008096184B38B5DFF8CC04408DDFF8A044E4
:10880000010728D50320F9F71FFFA07E002805D017
:108810000FF29060BDE83240FBF734BB0FF2BC6052
:10882000FBF730FBDFF8A0040078002805D00FF23A
:10883000D460BDE83240FBF725BB02210120FAF7E6
:10884000EFF90220FFF768FF1E2201210846BDE86C
:108850003840FAF7EDBDC00605D50420F9F7F4FE5F
:108860000020FFF7D6FE208F401C208780B23228E0
:108870006DDB00202087DFF84454687801280ED192
:10888000A87802280DD1A07E00280AD10020E0643B
:108890000120A0760FF28860FBF7F4FA01E00020D7
:1088A000A076A06C411EA164E06CEA68821AE264C2
:1088B0000FF28460FBF7E6FAA06C012847DADFF8D4
:1088C00008140978002942D1002810D1E0683C2121
:1088D00090FBF1F1E26C002A05D50022C9B2062016
:1088E000FAF7A6FD03E0C9B20620FAF7A1FDDFF80A
:1088F000BC03D0E90223002B01D1002A07D0DFF806
:10890000B003D0E90223002B10D1002A0ED16068F9
:10891000B0F5167F04DAA16CA0F51670814205DA75
:108920000020E0640FF22C60FBF7ACFAE06C012849
:108930000DDA02210120FAF773F90220FFF7ECFEAD
:108940001E2201210846BDE83840FAF771BD31BD4D
:10895000F0B587B0DA4CD24D287E002803D1D4E997
:108960000401C5E9100104F1080100A800F04EF966
:10897000287ED04900EB400201EB820100AAC8CA60
:10898000C8C1401C2876C74EC74831461822F9F79F
:10899000ADFD304604F108011822F9F7A7FDA868DB
:1089A000E864D6E90201CDE90401706902907068BB
:1089B000FDF768FFCDE900013068FDF763FF02466F
:1089C0000B460FF2A850FBF75DFABE4890F828005E
:1089D000C00602D50420F9F737FE48F6A04104206E
:1089E00007B0BDE8F040F9F7F1BD000070B52DED1E
:1089F000028B82B0B24DAD48D0E90223D5E9040123
:108A00008B420DD301D882420AD30FF29850FBF764
:108A100039FA012002B0BDEC028BBDE870407BE664
:108A200005F1080184B068461822F9F75FFD0FBC14
:108A300000F05DF80120FFF76FFE994C217E0FF2E8
:108A40008850FBF71FFA974ED6E90201002901D1A1
:108A500000283BD0D5ED031A95ED021AD6ED010A98
:108A600096ED000AFAF76AFDB0EE408AD5E90401F6
:108A7000D6E90223801A994104F076FC00EE100A30
:108A8000DFED850A80EE200ABCEEC00A10EE105A17
:108A900018EE100AFDF7F6FE02460B460FF24C5098
:108AA000FBF7F0F9A06800EE100AB8EEC00AB4EEC9
:108AB000480AF1EE10FA02D561688D4206D2BDEE89
:108AC000C80A10EE101A401AE06401E0FFF740FFF8
:108AD000207E218A884206D1002002B0BDEC028BA4
:108AE000BDE8704095E502B0BDEC028B70BD0FB4DF
:108AF000D0B56B48416881646D486C4CDDE9062354
:108B0000D4E90267921BBB41704E0027BB4207D3DA
:108B100001D8B24204D321461822F9F7E7FC03E05A
:108B20003A461346C0E90223204604A91822F9F761
:108B3000DDFCD0BC5DF814FB2DE97043584C227E5F
:108B4000617E0FF2B840FBF79DF90C25594E607E0F
:108B5000002808D1D4E91023C4E90C230FF2CC403B
:108B6000FBF790F919E0D4E90C230FF2D440FBF79E
:108B700089F9607E15FB006040894FF47A714143AA
:108B8000D4E90C890A4618EB020249EBE173C4E907
:108B90000C230FF2BC40FBF775F9607E15FB00F06B
:108BA00081592162801941686162008920853020E5
:108BB000FBF70EFC607E401C6076217EC0B28842CE
:108BC00005D100F006F80120BDE87043A4E5BDE83A
:108BD000708310B5324C00200146C4E91001208397
:108BE00002464FF496613348F9F742FC00202075A5
:108BF000607D002808D00FF27C40FBF743F931205C
:108C0000FBF7E6FB0020607510BD0000FEB50446D2
:108C10009FED220AD1ED000A60EE800AFDEEE00A27
:108C2000CDED000AD1ED010A20EE800ABDEEC00AAA
:108C30008DED010A4869ADF808001948057E002D40
:108C400003D10020ADF80A001BE0D1E9022315484A
:108C5000D0E90267901B63EB070104F085FB00EE8F
:108C6000100ADFED0D0A80EE200ABDEEC00A10EEFC
:108C7000101AADF80A102A4689B20FF21040FBF71D
:108C800001F900A80EC80EC40C38FEBD04480078D7
:108C9000002800D0F8E4704700007A448096184B12
:108CA000A0D1030050D7030068D7030080D703008A
:108CB00098D7030088970300B0D7030090D603002D
:108CC00068CF030068D5030020D40300E0930400BC
:108CD00080B50FF2EC30FBF7D5F8FFF777FB0120FA
:108CE000BDE80240FAF7A6B980B50FF2E430FBF711
:108CF000C9F80120BDE80240FAF7B9B95265715FC1
:108D00004261746368696E6720743A256420643A2E
:108D1000256420733A25642061723A25640A0000B4
:108D200052656D6F76655F4261746368696E670A4C
:108D3000000000004261746368696E675F53657488
:108D40005F4C6F6320743A256C6C75206C61737492
:108D50005F743A256C6C750A00000000524543565A
:108D6000206C61743A2566206C6F6E3A256620612E
:108D7000636375726163793A25752074696D6573F3
:108D800074616D703A256C6C750A00004261746301
:108D900068696E675F5365745F4C6F632056616CE2
:108DA00069643A257520536B697021210A0000001F
:108DB00056616C69643A25752070726F3A25750AA0
:108DC0000000000053502064697374616E63653A5B
:108DD0002564206172645F646966663A25642021B7
:108DE000210A00005350204D4F56452021210A00F2
:108DF0004261746368696E675F466C7573685F543F
:108E00007269676765722062617463685F6964781C
:108E10003A2575206578743A25640A0042617463C6
:108E200068696E675F4E4C505F5374617475733A36
:108E300025750A004261746368696E67204C4D5F56
:108E400049444C452121210A00000000426174631D
:108E500068696E675F5365745F50725F53746174C5
:108E6000652041525F54203A2025662025660A007D
:108E70004261746368696E675F5365745F50725FC7
:108E800053746174652041525F540A0042617463F7
:108E900068696E675F5365745F50725F5374617485
:108EA000650A00004261746368696E675F41525FE2
:108EB00054204261746368696E672054696D6572FD
:108EC0002052696E67696E6720535420486967684D
:108ED00020636865636B6564210A00004261746306
:108EE00068696E675F41525F5420426174636869CC
:108EF0006E672054696D65722052696E67696E678E
:108F0000210A00004261746368696E675F41525FC5
:108F10005420446F7A654D6F6465210A000000009B
:108F20004261746368696E675F41525F54205354B5
:108F30002048696768210A004261746368696E6746
:108F40005F41525F54206D743A2564206D643A2568
:108F5000640A00004261746368696E675F41525F32
:108F60005420326E6420547279210A004261746385
:108F700068696E675F416363755F4C6F63206C6106
:108F8000743A2566206C6F6E3A2566206163633AF9
:108F900025752074696D657374616D703A256C6C0C
:108FA000750A00004261746368696E675F4F6E5FA7
:108FB0004C6F635F48616E646C696E6720536B69C8
:108FC0007021210A000000004261746368696E67C5
:108FD0005F4F6E5F4C6F635F48616E646C696E6774
:108FE000206964783A25750A00000000646973748A
:108FF000616E63653A25660A000000004261746391
:1090000068696E675F466C7573685F496E5F507222
:109010006F677265737320665F6964783A2575209F
:10902000625F6964783A25750A0000003173742024
:1090300074696D657374616D703A256C6C750A00A6
:1090400074696D657374616D703A256C6C750A0096
:10905000646966665F74696D657374616D703A25E5
:10906000752C2074696D657374616D703A256C6C34
:10907000750A00004261746368696E675F466C75CB
:1090800073685F446F6E650A000000004765745F97
:10909000426174636865645F4C6F632064696666EF
:1090A0005F74696D657374616D703A257520675FD3
:1090B00062617463685F6964783A25750A0000002C
:1090C000534C435F4C425F496E69740A00000000D4
:1090D000534C435F4C425F4465696E69740A0000FB
:1090E00000B5ADF2D47D00A84FF4FA61F9F736FA75
:1090F00006E04FF4FA6300AADFF8640300F04FF9CA
:109100004FF4FA6100A804F041FC01281BDB40F297
:1091100045318842EDD040F2454188420BD047F2BC
:109120000A118842ECD14FF4FA6300AADFF8300349
:1091300000F0ACF9E4E74FF4FA6300AADFF820038B
:1091400000F0FAF9DCE70DF2D47D00BD2DE9D00383
:109150000446DFF81083DFF81093A8FB046709FBCF
:109160000477DFF80803E0FB0167DFF80403DFF8AA
:10917000041330187941DFF80033A3FB0223801A6F
:109180009941BDE8D00370472DE9F04186B004460F
:109190000D4616461F4600208DF8150001208DF85B
:1091A00014000020ADF81000002F06D01820ADF8F4
:1091B0000E0000208DF80C0005E00220ADF80E0036
:1091C00001208DF80C004FF47A70684302908DF8FE
:1091D000124070008DF81300102202A940F2654081
:1091E00004F063FB8046019700962B4622460FF25F
:1091F00064310FF2703003F05DF9B8F1010F01DB5B
:10920000012000E0002006B0BDE8F08194494860EC
:10921000704793498860704791490860704790494A
:10922000C860704700208E494860704700208C4914
:109230008860704700208A4908607047002088498C
:10924000C860704786494A68002A01D0002801D5C5
:10925000002070470246521E9241D20F8A750122A9
:109260000A750861887D002804D000231A46012170
:10927000104689E700231A460969104684E77848B2
:109280000021817501750161417D00230A46184660
:109290007AE701460020724A1368002B07D0517507
:1092A000117D002903D1517D03460A466CE77047C2
:1092B00038B504466A4DE868002801D1002032BD67
:1092C0002346224621460120FFF75EFF002800D0FA
:1092D000EC7532BD38B50446614DE87D044202D0DC
:1092E0000120FFF7E5FF2046401E8041C00F8DF8AA
:1092F0000000012200A94FF4A26004F0D6FA012870
:1093000000DB2C76012801DB012032BD002032BDBC
:1093100053480021016041608160C16081754175E1
:10932000012101760021C17504F0E1BB70B4002277
:109330009FED4A0A134690F9044002E041F82220CA
:10934000521CA242FADB012C27DB1A461FE051F81F
:10935000245005EB850600EB8605D5ED030AB4EE37
:10936000600AF1EE10FA02D5B0EE600A2346641CE2
:1093700090F90450AC42EADB51F8224051F82350F6
:1093800041F8225041F823409FED340A521C90F9D5
:109390000440A24201DA1446EAE770BC704730B5D7
:1093A0008FB004461546002C54D0002D52D0287999
:1093B00000F03F003F284DD1E86803F08DF84FF4EE
:1093C00003722E4BFDF786FACDE90001286903F000
:1093D00083F86FF0E7022A4BFDF77CFACDE9020132
:1093E000686903F079F80022264BFDF703FCCDE90C
:1093F0000401688B03F07AF80022234BFDF7FAFB97
:10940000CDE90601A88B03F071F800221D4BFDF792
:10941000F1FBCDE90801288B0C906A79A968E888EE
:10942000FFF794FECDE90A01207D002805D0616890
:1094300008000AD000A8884707E0607D002804D013
:109440002168080001D000A88847A07D002801D02D
:10945000FFF715FF0FB030BD000000000000000056
:109460004CD50300000029F90F26020040420F00EE
:10947000000087C14F88620400CA9A3B0080663EA4
:10948000FF7F763E000024400000594070B5ADF5E6
:10949000A16D04461546A06800284AD0002D48D08A
:1094A0000026FFA908312846FFF740FF304600900C
:1094B00036E0FFA8083050F8260000EB800105EBED
:1094C000810090ED030AB5EE400AF1EE10FA26DDB8
:1094D00000A9009A01EB021181ED020A017A00AAAB
:1094E000009B02EB03121171417A00AA009B02EB70
:1094F0000312517100A9009A01EB021102690A617D
:1095000000A9009A01EB02114269CA60807A00A9A1
:10951000009A01EB021188710098401C0090761CA3
:1095200095F904008642C4DBA168080001D000A8B8
:1095300088470DF5A16D70BDC168080009D0002AEB
:1095400007D0080005D01278501E8041C043C00FDC
:109550000847704773656E644C6F636174696F6E22
:10956000526571005B495D5B202573205D20696455
:109570003A257520726174653A256C6920706173B3
:10958000736976653A257520617661696C3A25754F
:109590000A00000010B5DFF8284300220821204609
:1095A000F8F766FF204610BDDFF81403704700008F
:1095B00038B5044604F0E4FC4FF47A726243841830
:1095C00051EBE27500BF00BF00BF00BF00BF04F059
:1095D000D7FCA942F6D301D8A042F3D331BD38B5A8
:1095E0000446FCF7C4FEB74AC2E90801002C24D0A7
:1095F000B5480078002820D0B44C2078401C20705A
:10960000B34D2878401C2870102000F084FD802085
:1096100080F3118800BF00BF2078401E207028789A
:10962000012804D16868002801D004F00FFE2878D2
:10963000401E2870002080F311881E20BDE83240B3
:1096400004F0F4BE38B50446FCF791FE9D4AC2E929
:109650000601002C24D09C480078002820D09B4C88
:109660002078401C20709A4D2878401C28700820D3
:1096700000F051FD802080F3118800BF00BF2078EA
:10968000401E20702878012804D16868002801D085
:1096900004F0DCFD2878401E2870002080F311883B
:1096A0001F20BDE8324004F0C1BE38B50446FCF7C7
:1096B0005EFE844AC2E90001002C24D18248007871
:1096C000002820D0814C2078401C2070804D2878C4
:1096D000401C2870202000F01EFD802080F311889F
:1096E00000BF00BF2078401E20702878012804D1D8
:1096F0006868002801D004F0A9FD2878401E287071
:10970000002080F311882120BDE8324004F08EBE95
:1097100080B5002812D0032818D16E48009000238D
:109720001A4603211F2004F04DFE6B4800900023D1
:109730001A4603211E2004F045FE01BD6748009033
:1097400000231A460221212004F03CFE01BD80B511
:10975000FFF720FF04F0CEFEBDE80140C8E080B571
:109760000846FCF7BBFD5E4802F0D9FD002805D095
:109770000FF29010BDE80240FDF7B6BC01BD00231A
:10978000584A4021564804F01DBFFB230FF28412B3
:1097900004F0E3BEF8B50C4615461E4605274C48B6
:1097A0000178491C0170002005F012F8002806D14C
:1097B00033462A462146002005F00DF8074600F002
:1097C00075FE3846C0B2F2BDF8B50C4615461E46C9
:1097D00005273F480178491C0170002004F0F8FF7C
:1097E000002806D133462A462146002004F0F5FF22
:1097F000074600F05BFE3846C0B2F2BD02280ED02C
:1098000005280CD006280ED008280AD00E2806D02D
:109810001D2806D0222802D0C02802D005E004204E
:1098200070470720704709207047002070472DE9D6
:10983000F8430C4615461E46052740B2FFF7DEFFEB
:10984000804615F8019B22480178491C0170264981
:10985000404605F08CF8002808D10095731EDBB255
:109860004A466108404605F098F8074600F01EFE9B
:109870003846C0B2BDE8F2832DE9F04182B00C4613
:1098800015461E46052740B2FFF7B8FF8046104830
:109890000178491C01701449404605F068F8002819
:1098A00007D10096089B2A466108404605F060F8FB
:1098B000074600F0FBFD3846C0B2BDE8F681000067
:1098C000FCD8030008D6030070D9030072D9030046
:1098D000C867030045A60000DFA50000ABA6000096
:1098E00060D303005FA70000801A060004F030BBBD
:1098F00080B5FFF759FE01210170C170417181717E
:1099000001BD00004D534720426F782046756C6CB6
:109910000000000073746172745F74785F73747216
:1099200065616D0030B5134D0446287881B020B9CB
:10993000281D05F0C7F801202870281D05F0DBF868
:10994000204605F0BAFF0446281D05F0FAF8204627
:1099500001B030BD30B50446064D81B0281D05F07C
:10996000CAF8204606F009F9281D01B0BDE83040CC
:1099700005F0E7B838D803002DE9F04180460C46E1
:10998000FBF769FB0546002700F0BBFB0646B8F174
:10999000010F1ED0B8F1040F4BD0B8F1050F78D0ED
:1099A000B8F1080F00F08480B8F1250F00F0A9800D
:1099B000B8F1870F00F0BE80B8F1A10F00F09480DD
:1099C000B8F1A40F00F09680B8F1BB0F00F0AD80A5
:1099D000B5E006F058FCDFF85882B4F9000000EE5C
:1099E000900AF8EEE00A20EE800A88ED000A06F000
:1099F0004AFCB4F9020000EE900AF8EEE00A20EE0C
:109A0000800A88ED010A06F03EFCB4F9040000EE7D
:109A1000900AF8EEE00A20EE800A88ED020A20881B
:109A2000A8F80C006088A8F80E00A088A8F810001C
:109A300085E006F055FDDFF8F881B4F9000000EE8E
:109A4000900AF8EEE00A20EE800A88ED050A06F09A
:109A500047FDB4F9020000EE900AF8EEE00A20EEAD
:109A6000800A88ED060A06F03BFDB4F9040000EE1A
:109A7000900AF8EEE00A20EE800A88ED070A2088B6
:109A8000A8F820006088A8F82200A088A8F8240080
:109A900055E0DFF89C81D8F834002168884200D175
:109AA00001271C22214608F13400F8F70FFD46E09B
:109AB000DFF87C8198F850002178884200D1012796
:109AC0000122214608F15000F8F700FD0222611C36
:109AD00008F15200F8F7FAFC022204F10B0108F138
:109AE0005400F8F7F3FC2AE00C2221465148F8F71D
:109AF000EDFC24E001270C2221464F48F8F7E6FC54
:109B00001DE0DFF82C81D8F858002168884205D183
:109B1000D8F85C006168884200D1012708222146FC
:109B200008F15800F8F7D2FC09E0E078404981F8E4
:109B30006C0004E094F903003D4981F86D00002DAC
:109B40000FD0002F0DD1686A00280AD04069801B11
:109B5000012806DA214605F11000BDE8F04100F0C9
:109B6000C9B9BDE8F08102460846012A0ED0042A90
:109B700010D0052A12D0082A14D0872A22D0A12A70
:109B800014D0A42A16D0BB2A18D070471422284912
:109B9000F8F79CBC14222949F8F798BC1C222849E4
:109BA000F8F794BC06222749F8F790BC0C2221490B
:109BB000F8F78CBC0C222049F8F788BC0122224916
:109BC000F8F784BC01222149F8F780BC01280CD0A9
:109BD00004280FD0052812D008281AD0252813D021
:109BE000872820D0BB2819D07047FF2214211048A5
:109BF000F8F73EBCFF2214211048F8F739BCFF22C9
:109C00001C210F48F8F734BCFF2208211048F8F750
:109C10002FBCFF2206210B48F8F72ABCFF220121A6
:109C20000948F8F725BC0420014981F86D00704708
:109C300090CF0300B8CF0300F0CF0300A4CF030000
:109C4000C4CF0300E0CF0300FCCF0300FDCF03002F
:109C5000E8CF030038B50446002500E06468002C16
:109C60000CD0207A0A789042F8D1E0684A68904295
:109C7000F4D120698A689042F0D1012529460FF27B
:109C80006420FDF731FA002D00D10024204632BDBA
:109C900038B504462020FFF745FE05460022202166
:109CA000F8F7E6FB0C22214605F10800F8F71EFC48
:109CB00060686861A068A86101202877284632BDE5
:109CC000F8B500231C4601F10805854A1678761C74
:109CD0001670802686F3118800BF00BF5678761C68
:109CE000567006686F6801E034467668002E04D02E
:109CF000D6F80CC06745F7DA0123002B0AD0336889
:109D00000B604E603368002B01D0596000E00160A9
:109D1000316005E0002C02D061600C6000E0016061
:109D20005078401E5070C0B2002802D1002080F34D
:109D3000118800F0BBFB0020F2BD10B5684C227802
:109D4000521C2270802282F3118800BF00BF62780B
:109D5000521C62704A680B68002B01D05A6000E008
:109D600002604868002801D00A6802600846FFF7D0
:109D7000F1FD6078401E6070C0B2002802D1002062
:109D800080F3118800F092FB002010BD30B402680F
:109D9000002A03D0C168D368994200D04268002AE3
:109DA00028D04F490B785B1C0B70802383F31188FC
:109DB00000BF00BF4B785B1C4B70D36852699A1A86
:109DC000C3689C1A92FBF3F503FB054343610369E7
:109DD0009C1A92FBF3F203FB024282614878401E18
:109DE0004870C0B2002802D1002080F3118830BC36
:109DF00000F05CBB30BC704770B504460D4620686F
:109E0000FFF728FF06000BD12846FFF741FF064663
:109E100031462046FFF754FF3046FFF7B7FF02E018
:109E2000307F401C3077207A401C2072307A002826
:109E300000D16660002070BD10B504462068FFF7B1
:109E400009FF002801D1032010BD017F491E0177C1
:109E5000217A491E2172017A002901D10021616015
:109E6000017F002903D101462046FFF766FF00204D
:109E700010BD70B51A4A13785B1C1370802383F3EE
:109E8000118800BF00BF53785B1C5370006801E06D
:109E900083614068002815D043695C1A83695B1AA6
:109EA000012C05DAC568661994FBF5F405FB14640A
:109EB0004461012BECDA04691D1993FBF4F304FBF4
:109EC0001353E5E75078401E5070C0B2002802D10D
:109ED000002080F3118800F0E9FA002070BD000036
:109EE000C8670300236663202564000000214181C8
:109EF0000181704738B50446002926D0002C24D0B3
:109F0000B4F90800B4F90A201018228890FBF2F383
:109F100002FB13036088024665689BB200FB035096
:109F2000F8F7D4FAB4F90A002188884202DA401C12
:109F3000608131BD09D12089401C208100B2218877
:109F400090FBF1F201FB1200208131BD2DE9F041BF
:109F500004460D461646002D3ED0002C3CD0B5F9E7
:109F6000081008462A881346374607EB000C63455D
:109F700009DB698801FB07F26B6801FB00312046B1
:109F8000F8F7A4FA1CE01B1ABB4201DBB04603E061
:109F9000A2EB01081FFA88F8698801FB08F26B68D8
:109FA00001FB00312046F8F791FA6888A6EB08011A
:109FB00089B200FB01F2696800FB0840F8F786FAF5
:109FC000B5F908003818298890FBF1F201FB12005E
:109FD00028816889801B6881BDE8F081B0F90A108A
:109FE000408811FB00F080B27047B0F90A0080B2DF
:109FF0007047000080B5FFF779FC009000A800F0E2
:10A0000083F8042000F087F8444802F0F6F901BD17
:10A0100070B5424C2046C068C0460546FAF7CDFEF2
:10A020000646B54212D031462846FCF715FB3146AC
:10A03000204606F08FFA002E204603D0BDE870407F
:10A0400002F0DBB9BDE8704002F002BA70BD10B595
:10A0500082B000200090FCF7DDF80021022002F021
:10A0600094FF23E00098FCF79DF92D480178491CE6
:10A070000170FBF7E0F800F019FA00A9294806F092
:10A0800077FA0028EED0200702D50820FAF7EFFF74
:10A09000E00602D51020FAF7EAFFA00602D520203C
:10A0A000FAF7E5FFA00701D5FFF7B2FF3E2006F063
:10A0B0007DFA04466007E0D4E5E710B584B0174C9C
:10A0C00004F114030822042104F1680006F090FA58
:10A0D000022002904FF40060019004F18000009093
:10A0E000114B50220FF24C0104F1340006F08CFAAF
:10A0F0004FF47A720D49204604B0BDE8104002F0DA
:10A1000070B90648C068704780B50146054806F03A
:10A11000ADFA40B202BD064906F0C6BA1482030089
:10A12000C86703007C8203004FB00000F5AF000059
:10A130004882030073656E736F725F7461736B00A6
:10A14000506002604160086070470A68F8E7486044
:10A150000160704701684068F9E7002007E0364970
:10A1600001EBC00241F8302011464960401C09282B
:10A17000F5DB704710B402680B4600E012688242BB
:10A1800004D09468A342F9D1104600E0002010BC2E
:10A1900070472DE9F04104460D462646264F57F8F4
:10A1A000368008E0D8F80820100002D02946204662
:10A1B0009047D8F8008007EBC6008045F2D1002018
:10A1C000BDE8F08138B50C46092801DA210007D135
:10A1D000224601460FF2640002F06CF9032032BD02
:10A1E000154901EBC00521462846FFF7C3FF0028AB
:10A1F00006D10C20FFF796FB84602946FFF7A5FFE8
:10A20000002032BD70B504460D460B4800EBC4007B
:10A21000FFF7B0FF060007D12A4621460FF23400AF
:10A2200002F048F9032070BDFFF794FF3046FFF7B6
:10A2300091FB002070BD0000D4D2030061626E6FFC
:10A24000726D616C2072656769202825642025780D
:10A250002900000061626E6F726D616C20756E7214
:10A260006567692825642C257829000030B4802092
:10A2700080F3118800BF00BFDFF8941388680022C4
:10A280000A7182F3118800281CBF0268002A33D0AB
:10A29000436954699C422FD100E022461468A4B15E
:10A2A00065699D4211D12246146874B165699D4269
:10A2B0000BD12246146844B165699D4205D12246FE
:10A2C000146814B165699D42E7D0802383F3118837
:10A2D00000BF00BF03680C69844208BF0B61016ABC
:10A2E0000B60196202621168016001B108621060BE
:10A2F00092F8290082F82800002080F3118830BCF1
:10A30000704730B5DFF808430020607181B0206AE3
:10A31000E16900F18040606208001CBF2046884768
:10A32000002080F31188E56808E0E868616A411A56
:10A3300048BF6062002080F311882D6805B380203B
:10A3400080F3118800BF00BF206920B168692169CE
:10A350004969884219D3287C4007EBD5E868216A0F
:10A36000401A0128E1DA284600F0BCF8802080F38A
:10A37000118800BF00BF287C0028D6D101B030BDB5
:10A38000802080F3118800BF00BF01B030BD000005
:10A3900070B5DFF87C420020607001202070E06B17
:10A3A00068B1802080F3118800BF00BFE06B804758
:10A3B000002080F31188E063606384F83800A068AF
:10A3C00000281CBFC16A002904D009680A001CBF0C
:10A3D0004068884794F8310040B1A06894F8301084
:10A3E00080F82810207908B1FFF740FF206948B3B2
:10A3F00004E028682061002080F31188802080F329
:10A40000118800BF00BF25690DB32E7CFEB1700717
:10A410000ED5E868216A411A012905DA284600F0BC
:10A4200061F8287C20B90DE0616A411A48BF60627A
:10A4300006F0FB001028DCD1A86880684068007C2A
:10A440000028D6D1802080F3118800BF00BF60793A
:10A4500050B9206900B32069007C0028206909D028
:10A4600080688068406805E0FFF74BFF607900284E
:10A47000FAD1EEE7A060A068C16A21B149680A007C
:10A480001CBF40688847A06890F8280084F8300016
:10A4900084F83100204670BD84F8310084F8300023
:10A4A000A060207080F31188204670BD10B5584C14
:10A4B0002078401E2070C0B298B9606888B18020B2
:10A4C00080F3118800BF00BF606830B101202070A8
:10A4D000204603F0A8FE00202070607808B980F3C1
:10A4E000118810BD30B581B08168494C41B1226AF4
:10A4F000C2600A68496802B151600A600021816047
:10A50000017C11F00301017426D1216991B9206108
:10A51000207838B901202070204603F084FE002006
:10A52000207001E0012060716078A8B980F3118883
:10A5300001B030BD42694B699342E8D38142E7D014
:10A540009A4209D103461B68002BEDD05D69AA42EF
:10A55000EAD18B42F7D1DAE701B030BD30B52C4CEF
:10A56000227881B04169521C227004F10C0200E093
:10A570001A461368A3B15D69A94211D21A4613683D
:10A5800073B15D69A9420BD21A46136843B15D6984
:10A59000A94205D21A46136813B15D69A942E7D3EF
:10A5A00003600262106043B118625A698A420CBFAC
:10A5B00090F82910002180F82810017C51B98021E1
:10A5C00081F3118800BF00BFFFF78CFF607808B9E6
:10A5D00080F3118801B0BDE8304067E730B50C4C1E
:10A5E0002578681C207081B0204603F01CFE60783E
:10A5F000257008B980F3118801B030BD00B581B075
:10A6000006F070F802480121017001B000BD0000A1
:10A61000C8670300002848BF4042704738B5DFF8DC
:10A62000A80A00880146102908DA002806D0DFF8B9
:10A630009C4A04EB81004168491C4160DFF88C4A68
:10A640002068401C2060B0F5617F15DB01250AE021
:10A6500004EB85004268002A04D029460FF68C20BE
:10A66000FCF742FD6D1C102DF2DB00224021201D65
:10A67000F7F7FEFE0020206031BD0FB42DE9F04752
:10A680002DED028B88B0DFF8484AB4F876A004F1CB
:10A6900008050A27B5F91E0010FB07F0B5F92010D0
:10A6A000A0EB010804F5BA76304601F0C1FC94F83D
:10A6B000740117FB00F7BFB22A2F18D10FFA88F8E0
:10A6C000B8F1000F13D5B06800280DD10120F7F7BD
:10A6D00064FE8046F7F733FE0120B06042463946FB
:10A6E0000FF61420FCF700FD0120706023E0B06835
:10A6F000012807D1F7F72EFE0020B0600FF61020DA
:10A70000FCF7F2FC7068282F0DDB002806D1D4F886
:10A71000802039460FF60420FCF7E6FC012070602B
:10A72000F7F71CFE07E0012803D10FF61020FCF715
:10A73000DBFC00207060129804909DED138A8DED73
:10A74000058ADDED148ACDED068ADDF85C8004A86B
:10A7500090EC030A404600F08AFCDFF8787995ED2A
:10A76000030ADDED120AB4EE600AF1EE10FA30D100
:10A7700095ED040AB4EE480AF1EE10FA29D195EDF0
:10A78000050AB4EE680AF1EE10FA22D1F86900F178
:10A790000109C7F81C90B9F1150F02D30020F86128
:10A7A0001FE0B9F1020F1CD36869FCF76BF8CDE923
:10A7B00002012869FCF766F8CDE90001E868FCF7BA
:10A7C00061F802460B4649460FF67C10FCF78CFCFC
:10A7D00007E00498E8600598286106986861002001
:10A7E000F861414604A8F6F7E3FF804604F1200033
:10A7F000F7F71EFDA869012814D1F868401CF8601D
:10A80000F5F7F9FC04F12000F7F712FD282204F116
:10A81000200104F14800F7F769FE0FF64010FCF73D
:10A8200063FC18E0F6F7A6FF012812D13869401C36
:10A830003861F6F7A3FF7861F5F7DDFC04F120003D
:10A84000F7F7E6FC7A6939690FF61810FCF74CFC4B
:10A8500001E000F021F9B869401CB861B0F5617FF2
:10A8600008DBFB687A6939690FF60810FCF73CFCD5
:10A870000020B861FFF7D2FEBAF1000F40D0B4F863
:10A88000760000283CD1287ADFF84C1894ED020AB3
:10A89000BDEEC00A10EE102A4FF47A735A4301FB42
:10A8A000002095ED010ABDEEC00A10EE101A08183E
:10A8B00041007A68BA603B687B60D4F880003860F9
:10A8C0007869029038690190386800900FF6B800F6
:10A8D000FCF70AFC04F18005B068039070680290F0
:10A8E000286AFBF7CFFFCDE90001A86AFBF7CAFF92
:10A8F00002460B46D4F880100FF6AC00FCF7F4FBD0
:10A90000404608B0BDEC028BBDE8F0075DF814FBD3
:10A91000002805D0DFF8B817096F4022F7F7E6BD29
:10A92000704738B50C4605000BD1DFF8A40700EEE0
:10A93000104AB8EE400A80ED030A0830F7F77FFCB2
:10A9400015E0012D0BD1DFF8880700EE104AB8EEB4
:10A95000400A80ED020A0830F7F771FC07E0022D8B
:10A9600005D1DFF86C0704740830F7F768FC0D2098
:10A9700010FB04F229460FF65000FCF7B5FB42F23B
:10A980007470044640F2EF70224601460FF648000C
:10A99000BDE83840FCF7A8BB2DE9F8432DED028B4C
:10A9A00084B00746884691460FF63C00FCF79CFBB6
:10A9B00042F27470044640F2EF70224601460FF6F0
:10A9C0001800FCF791FBDFF8084700224FF4C07134
:10A9D0002046F7F74DFD04F1080504F1B406AE6614
:10A9E00000EE107AB8EE408A85ED018A00EE108AFA
:10A9F000B8EE400A84ED020A85F80890F2EE0A8A61
:10AA000048460D2111FB00F0029020EE280A10EEBE
:10AA1000100AFBF737FFCDE9000128EE280A10EEF7
:10AA2000100AFBF72FFF02460B460FF2C870FCF727
:10AA30005BFBF5F735FB2846F7F701FC0020606764
:10AA400004F174010220C88028223046F7F74EFD39
:10AA50000120607104F5BA7001F0EAFA0020C4F830
:10AA60007C01C4F8780102463C2104F5C07004B0B2
:10AA7000BDEC028BBDE8F843F7F7FABC10B590B017
:10AA8000F7F780FC044600A8FFF742FF039800197F
:10AA900010B010BD000000002DE9F041DFF8304695
:10AAA000251DA86A616D884204D16A8CB4F84E30C5
:10AAB0009A4279D0B0EB010802D5DFF82006804435
:10AAC00004F1540695ED100AD6ED060A30EE600A40
:10AAD000B5EE400AF1EE10FA03D5DFED940A30EE40
:10AAE000200AD5ED0E0A96ED041A70EEC10AF5EEB5
:10AAF000400AF1EE10FA03D59FED8C1A70EE810A30
:10AB00006878012802D0022827D02DE004F1F4074C
:10AB100039469FEDCA1A404600F052F82079404469
:10AB20002071C0B206281FDB04F5807004F17401A7
:10AB30009FEDC21AD0ED0A0A90ED080AD4F8000180
:10AB400000F03EF82079401C207100224021384658
:10AB5000F7F78EFC0220687006E004F174019FEDA7
:10AB6000B71A404600F02CF8688C002809D1002262
:10AB7000402104F1F400F7F77BFC00202071012054
:10AB80006870282204F1200104F14800F7F7AEFCB8
:10AB900004F17400F06104F1B407402204F174017F
:10ABA0003846F7F7A3FCF761A88CB4F8BA108842CE
:10ABB00004D004F15406F084A4F8BA00BDE8F08192
:10ABC000F8B52DED028BF0EE408AB0EE608AB0EE63
:10ABD000410A0C46DFF8F854EE8CAF8CA68000F0EA
:10ABE00038F894ED0B0A30EE280A84ED0B0A00F0D9
:10ABF00075F884ED0B0A66802780A86B206394EDBE
:10AC00000D0A30EE080A84ED0D0A00F047F884EDD5
:10AC10000D0A95ED100ADFED8A0A20EE200A84ED78
:10AC20000E0ADFED880AB4EE600AF1EE10FA02DBDC
:10AC3000DFF8AC04A063686BE0636088002801D192
:10AC40000020E063286BA060288DE080BDEC028BC3
:10AC5000F1BD38B505460C46E0682818E06000F004
:10AC60005CF8E0606088032802D0042807D00DE07B
:10AC700020692818206100F050F8206131BD60691A
:10AC80002818606100F049F8606131BD206928181A
:10AC9000206100F042F8206131BD000080B52DED4B
:10ACA000028BB0EE408A9FEDB10AB4EE408AF1EE1D
:10ACB00010FA0DDB9FEDAE0A38EE008A18EE100A8E
:10ACC000FBF7E0FD02460B460FF23450FCF70CFA9E
:10ACD000B0EE480ABDEC028B01BD000080B52DED41
:10ACE000028BB0EE408A9FEDA10AB4EE408AF1EEED
:10ACF00010FA0DDB18EE100AFBF7C4FD02460B46F6
:10AD00000FF20850FCF7F0F99FED990A38EE008A2F
:10AD1000B0EE480ABDEC028B01BDDFF8C0138842DB
:10AD200002D3DFF8C01308187047000000247449EC
:10AD3000F7F74CBBF7F78DBA2DE9F8432DED048BEF
:10AD40008AB00446B0EE408AF0EE608AB0EE419AD6
:10AD5000DF4D05F5C27696ED0B0AF0EE480AB4EE2B
:10AD6000600AF1EE10FA05D1D5F884012018C5F873
:10AD7000840102E00020C5F88401F0EE689A96EDA7
:10AD80000C0AB4EE690AF1EE10FA03D170682018CB
:10AD9000706001E000207060B0EE490AD6ED0D0A47
:10ADA000F4EE400AF1EE10FA03D1B0682018B0605A
:10ADB00001E00020B060D6F80480D5F8849140F618
:10ADC000B837B94504DAB84502DAB068B8422EDBC4
:10ADD00010EE100AFBF756FDCDE90801B0680690A9
:10ADE00019EE900AFBF74EFDCDE90401CDF808807D
:10ADF000B0EE480A10EE100AFBF744FDCDE9000161
:10AE00004A4621460FF21040FCF76EF9D5F884014E
:10AE1000B84202DB0020C5F884017068B84201DB4B
:10AE200000207060B068B84201DB0020B0600AB05A
:10AE3000BDEC048BBDE8F1830000000000000000C1
:10AE40008FC2753D0100C8412DE9F8432DED048BFB
:10AE50008AB00446B0EE408AF0EE608AB0EE419AC5
:10AE6000B5EE400AF1EE10FA01DCB1EE400A984D61
:10AE7000DFED940AB4EE600AF1EE10FA05DBD5F8C6
:10AE800090012018C5F8900102E00020C5F890015B
:10AE9000F0EE689AF5EE409AF1EE10FA02DDB0EEAF
:10AEA000690A01E0B1EE690A05F5C876B4EE600AF8
:10AEB000F1EE10FA03DB70682018706001E00020EA
:10AEC0007060B0EE490AB5EE400AF1EE10FA01DC0E
:10AED000B1EE401AB4EE601AF1EE10FA03DBB0687E
:10AEE0002018B06001E00020B060D6F80480D5F8EA
:10AEF000909140F6B837B94504DAB84502DAB0683F
:10AF0000B8422EDB10EE100AFBF7BCFCCDE90801BD
:10AF1000B068069019EE900AFBF7B4FCCDE9040185
:10AF2000CDF80880B0EE480A10EE100AFBF7AAFC34
:10AF3000CDE900014A4621460FF20030FCF7D4F873
:10AF4000D5F89001B84202DB0020C5F89001706886
:10AF5000B84201DB00207060B068B84201DB00201D
:10AF6000B0600AB0BDEC048BBDE8F18301247449E4
:10AF7000002474C970B52DED088B8AB00646B0EE7A
:10AF8000408AF0EE608AB0EE419AF0EE499AB0EE57
:10AF900068AA20EE000A0AEE0A0A09EEA90AF7F7E3
:10AFA0004BFA4B4CD4F89C0104F5CE75002805D122
:10AFB0000021E9604C49A96000212961D5ED030A0F
:10AFC000F4EE400AF1EE10FA01D585ED030AD5ED55
:10AFD000020AB4EE600AF1EE10FA01D585ED020A1C
:10AFE000D5ED040A70EE80AAC5ED04AA6968491C73
:10AFF0000BEE101A85ED01BA3018C4F89C0147F227
:10B00000315188422FDB19EE900AFBF73BFCCDE96A
:10B0100008011AEE100AFBF735FCCDE90601B0EE87
:10B02000480A10EE100AFBF72DFCCDE90401E86890
:10B03000FBF728FCCDE90201A868FBF723FCCDE96A
:10B040000001B8EECB0A8AEE800A10EE100AFBF778
:10B0500019FC02460B460FF20820FCF745F80020C9
:10B060006860C4F89C010AB0BDEC088B70BD70B577
:10B070002DED048B0446B0EE408AF0EE608AB0EE0F
:10B08000419A134DB5F87660FFF756FEB0EE491AB7
:10B09000F0EE680AB0EE480A2046FFF7D5FEB0EEA3
:10B0A000491AF0EE680AB0EE480A2046FFF762FF40
:10B0B00005F5D87080EC038AA5F88061BDEC048B9F
:10B0C00070BD000035336B41206303001CD30300C7
:10B0D0007CC0030070D6030040420F0081969800A8
:10B0E0000000C841806967FF00007A4450443A4636
:10B0F000256428256429000050443A42504F4E20D0
:10B100005648282564292053746570282564290031
:10B1100050443A42504F46460000000050443A53D3
:10B12000746570436E745570205648282564292034
:10B1300053544550282564290000000050443A45E6
:10B14000584954564800000050443A4E41435B254C
:10B15000645D2025662025662025660050443A4F10
:10B160004652000050443A52432825642C25642955
:10B170000000000050443A52432825642C256429DD
:10B180002C4F46282564290050443A5353282564FF
:10B190002C25643E25643E2564292C5243282564D1
:10B1A0002C2564290A00000050443A532825642CB9
:10B1B000252E32662C252E3266292C562825642C05
:10B1C0002564290A0000000050443A5055542825AF
:10B1D000642025642900000050443A5052497625E5
:10B1E000642C4D762564000050443A313453455068
:10B1F0003230000050443A25662025662025640040
:10B2000050443A446973744F6625660050443A438B
:10B21000616C4F462566000050443A45532825642A
:10B220003A25642C252E32662F25642C252E326675
:10B230002F25642C252E32662900000050443A4503
:10B24000462825643A25642C252E32662F25642C49
:10B25000252E32662F25642C252E3266290000000B
:10B2600050443A4E43252E32662C252E32662C252C
:10B270002E32662F78252E32662C79252E32662CBA
:10B280007A252E32660A00002DE9F043002300E003
:10B290005B1C032B4ADA002433E005F1070EAEEB0A
:10B2A000060E4FF007089EFBF8F8C8EBC808AEEB97
:10B2B000080E5FFA8EFE0FF66468C3EBC30908EB55
:10B2C000C90808EB8609D9ED070A07EB000909EB65
:10B2D0008E0999ED3F1A60EE810A08EB860898ED19
:10B2E000001A0CEB8E0EDEED001A41EE610A30EE14
:10B2F000800A761C072ED0DB0CEB850585ED000A55
:10B30000641C032CC4DAC4EBC405AF00542515FB40
:10B31000030507EB050C0D46002A03D100264CF867
:10B320002560EDE79FED440A0026E3E7BDE8F083E2
:10B33000D2B218B400230CE094ED031A21EE001AE7
:10B34000F7EE001A71EEC01A01EEA01A84ED001A91
:10B350005B1C032B0ADA51F8234000EE904A002AC6
:10B3600000EB8304E8D1C4ED000AF1E70C220146AA
:10B370000C3018BCF7F7BAB838B504460D460020B3
:10B380000AE0C0EBC00204EB820202EB810155F837
:10B390002020C1F8FC20401C04F5F27292F9021042
:10B3A0000328EEDB5278C9B22046FFF76DFF94F810
:10B3B000E4219FED220A294604F5A870BDE8384033
:10B3C000B6E70000F8B5044694F9E651EDB2002660
:10B3D00017E0542212FB064211FB002151F8251000
:10B3E00000EE901A00EEA00A401C1C210328F0DB9E
:10B3F00011FB064000EB850705F090F987ED5D0A2B
:10B40000761C032E03DA9FED0C0A0020EDE704EB17
:10B41000850000F5C87191ED070AB5EE400AF1EE1E
:10B4200010FA06D0D0ED640A80EE800A81ED0E0A93
:10B43000F1BD00208863F1BD00000000A4707D3FD5
:10B4400010B5044604F5A870D0ED020A90ED011A7B
:10B4500094ED540A20EE000A01EE010A00EEA00A63
:10B4600005F05CF9002002E000228A61401C0328FC
:10B470000FDA04EB800202F5A871B5EE400AF1EE96
:10B4800010FAF1D0D2ED540AC0EE800AC1ED060ADE
:10B49000ECE710BDD0ED000A70EE800AC0ED000AA6
:10B4A000D0ED010A40EE000AC0ED010A89B2531E38
:10B4B000994215D100EE102AB8EE400AD0ED000AEC
:10B4C000C0EE800AC0ED000AD0ED010A80EE800ACD
:10B4D00080ED010AD0ED000A00EEE00A80ED020ADC
:10B4E00070472DE9F84F04460D4694F9E601C0B2C5
:10B4F00000902E88322096FBF0F0322101FB10677D
:10B50000B5F878804FF000092AE004EB890A09EBCE
:10B51000490005EB800B4FF4FA7231460BF1400005
:10B520009AED5A0AFFF7B6FF40F2DC5241460BF1A2
:10B5300090009AED5A0AFFF7ADFF3222394689B2E0
:10B540000BF11C00C9EBC90304EB8303DDF800C059
:10B5500003EB8C0393ED3F0AFFF79CFF09F1010910
:10B56000B9F1030FD1DBBDE8F18F8A1D072392FBF0
:10B57000F3F3C3EBC303D21A50F8222000EE102AD3
:10B5800000EB8100D0ED000A30EEC00AB0EEC00A38
:10B59000704730B40A460021931D072493FBF4F44E
:10B5A000C4EBC4041B1BDBB2541D072594FBF5F54B
:10B5B000C5EBC505641BE4B250F8233000EE103A29
:10B5C00050F8222000EE902AF4EE400AF1EE10FA34
:10B5D0000AD500EB840292ED001AB4EE401AF1EEA7
:10B5E00010FA01D501210EE0B4EE600AF1EE10FA76
:10B5F00009D500EB8400D0ED000AB4EE600AF1EE4C
:10B6000010FA00D50121084630BC70472DE9FE43F1
:10B6100006460C4696F8E6512088002800F08A80FD
:10B6200000273CE0C7EBC70006EB8009294609F17B
:10B630005400FFF79AFF08EB870080ED000AD4ED75
:10B64000030A30EE800A84ED030A09F1A8082946AE
:10B650004046FFF78AFFD4ED050A30EE800A84EDFC
:10B66000050A294609F15400FFF793FF00EE100A7E
:10B67000B8EE400AD4ED040A30EE200A84ED040A44
:10B6800029464046FFF785FF00EE100AB8EE400A53
:10B69000D4ED060A30EE200A84ED060A7F1C0DF177
:10B6A0000008032FBEDB00200AE094ED010A08EB3E
:10B6B0008001D1ED000A30EE200A84ED010A401C21
:10B6C0000228F2DB94ED020AD8ED020A30EE200ADD
:10B6D00084ED020A294606F5C870FFF746FFD4ED4F
:10B6E000030A30EE800A84ED030A294606F5D67077
:10B6F000FFF73BFFD4ED050A30EE800A84ED050A22
:10B7000006F5E47629463046FFF72FFFD4ED1B0AF5
:10B7100030EE800A84ED1B0A29463046FFF739FFD8
:10B7200000EE100AB8EE400AD4ED1A0A30EE200AF4
:10B7300084ED1A0ABDE8F7830A8890F9E631DBB296
:10B7400000EB830090ED5D0A3220034692FBF3F399
:10B7500000FB1323002B04D181ED020A81ED030AC3
:10B760007047D1ED020AF4EE400AF1EE10FA02D56C
:10B7700081ED020A08E0D1ED030AB4EE600AF1EEB1
:10B7800010FA01D581ED030A521C034692FBF3F334
:10B7900000FB132000281BD191ED020AD1ED030A12
:10B7A00030EE600AD1ED040A70EE800AC1ED040AA1
:10B7B000022B0BDBD1ED010A70EE600AF0EEE00A1D
:10B7C00091ED051A71EE200AC1ED050A81ED010A1D
:10B7D000088840F2DB52904209D191ED040AF3EE61
:10B7E0000E0A80EE200A81ED040A0120887070475D
:10B7F000F8B52DED048B84B00C460021642749E098
:10B80000C1EBC10200EB820290F9E63152F823202D
:10B8100000EE102A00AA02EB810282ED000A04EB7E
:10B82000810202F2B445D5ED030A70EE800AC5ED3F
:10B83000030A4FF4C87313FB014394F8B06403EB9D
:10B84000860696ED001A70EEC10AC5ED030AD2F81D
:10B85000B45400EE905A70EE800A02F2B445C5ED81
:10B86000000A94F8B05432353E4695FBF6F607FBD5
:10B87000165503EB850595ED001A70EEC10A02F22C
:10B88000B442C2ED000A94F8B02403EB820282EDC8
:10B89000000A491C0329B3DB94F8D804002816D108
:10B8A00000200EE004EB8001D1F8B42400EE102A51
:10B8B000DFED850A80EE200A01F2CC4181ED000A1D
:10B8C000401C0328EEDB012084F8D80458E004F57E
:10B8D000966090ED040ADFED7D0A80EE200A8DED82
:10B8E000000A90ED050A80EE200A8DED010A90ED28
:10B8F000060A80EE200A8DED020A9FED758A9FED03
:10B90000740ADFED738A002011E004EB8001D1F8A6
:10B91000CC1400EE901A00A951F8201001EE101A74
:10B9200000EE818A00EEA00A41EE018A401C032845
:10B93000EBDB04F0F3FEB0EE409AB0EE680A04F0E0
:10B94000EDFE29EE000AB5EE400AF1EE10FA01D044
:10B9500088EE008AB0EE480A04F0EEFEDFEDC80A79
:10B9600020EE200AF3EE0E0AB4EE600AF1EE10FAB1
:10B9700003DB002084F8D80402E0012084F8D80416
:10B9800094F8B004401C84F8B004C0B2642802D11A
:10B99000002084F8B00404B0BDEC048BF1BD0000BD
:10B9A00070B52DED048B0646301D90ED018A706850
:10B9B000FAF768FF41EC190B18EE100AFAF762FF6C
:10B9C00002460B4614461D4653EC192BDFF8F406CD
:10B9D000DFF8F416FAF77EFF22462B4604F0DEFE6F
:10B9E0001CD253EC192BDFF8E406DFF8E416FAF763
:10B9F00071FF02460B4614461D469FEDDD0A38EEE8
:10BA0000000A10EE100AFAF73DFF22462B4604F01A
:10BA1000C5FE03D2012086F8740002E0002086F8FB
:10BA20007400BDEC048B70BD70B504460D4616461F
:10BA3000FFF7C8FC2046FFF703FD29462046FFF725
:10BA400050FD29462046FFF7E1FD05F1780120462B
:10BA5000FFF772FE31462046BDE87040C8E60000A0
:10BA600038B52DED028B90ED050A90ED038AFBEEC3
:10BA7000040A9FED841A08EE201AB4EE401AF1EE83
:10BA800010FA1DD510EE100AFAF7FCFE02460B461E
:10BA900014461D4618EE100AFAF7F4FEDFF83426B5
:10BAA000DFF83436FAF716FF0022DFF83036FBF7FE
:10BAB00085FA22462B4604F071FE01D2012000E0F7
:10BAC0000020BDEC028B32BD000048420000C8429D
:10BAD000000000002DE9F0412DED028B8046002092
:10BAE0000CE098ED190A01EB410208EB8201D1ED5F
:10BAF000120A30EE200A88ED190A401CC0B2014635
:10BB00000329EEDB98ED1A0AD8ED1B0A9FED8F1A78
:10BB1000DFED8F1A40EE011AF4EE610AF1EE10FA31
:10BB200015DB9FED8C1ADFED8C1A40EE011AF4EE56
:10BB3000610AF1EE10FA0ADB9FED881ADFED881A30
:10BB400040EE011AF4EE610AF1EE10FA4DDA9FEDC3
:10BB5000850AF4EE400AF1EE10FA46D49FED828B8E
:10BB6000D8F81400FAF78EFE04460D46D8F80C00FB
:10BB7000FAF788FE53EC182BFBF720FA02460B4627
:10BB800020462946FBF736F80022DFF85435FAF74D
:10BB9000A1FEDFF85025DFF85035FBF70FFA02461B
:10BBA0000B4616461F46D8F81800FAF76BFE0446F7
:10BBB0000D46D8F81000FAF765FE53EC182BFBF78A
:10BBC000FDF902460B4620462946FBF713F832469C
:10BBD0003B4604F0E3FD08D398ED190ADFEDCC0AEB
:10BBE000B4EE600AF1EE10FA01DB002000E0012063
:10BBF000BDEC028BBDE8F0812DE9F041804698ED67
:10BC00001A0ADFEDA10A80EE200AD8ED1B0A9FED8B
:10BC10009E1AC0EE810A20EE200A10EE100AFAF7F2
:10BC200031FE02460B4616461F46D8F80C00FAF7BE
:10BC300029FE0022DFF8B434FAF74CFE04460D4624
:10BC4000D8F81400FAF71EFEDFF8A424DFF8A434B5
:10BC5000FBF7B4F902460B4620462946FAF7CAFF1D
:10BC6000DFF86824DFF89034FBF7A8F932463B464A
:10BC700004F0ACFD01D8012000E00020BDE8F08117
:10BC8000ED2E65420000FA4338B52DED048B0546D4
:10BC90000C4600200CE095ED0F0A01EB410205EB8C
:10BCA0008201D1ED080A30EE200A85ED0F0A401C12
:10BCB000C0B201460329EEDB6869FAF7E3FD41EC07
:10BCC000180B2869FAF7DEFD41EC190B53EC182B21
:10BCD000DFF82804DFF82814FAF7FCFD02460B46CB
:10BCE00051EC190B04F05AFD2CD253EC182BDFF851
:10BCF0001404DFF81414FAF7EDFD53EC192B04F0DB
:10BD00004DFD1FD253EC182BDFF80004DFF80014B0
:10BD1000FAF7E0FDDFF8CC23DFF8F833FBF74EF954
:10BD200053EC192B04F03AFD0CD295ED0F0ADFED20
:10BD3000C40AB4EE600AF1EE10FA03D5002C01D16A
:10BD4000012000E00020BDEC048B32BD00C028C5FE
:10BD500000854F49000048C400E87D480000C8C283
:10BD600000C82F4701806D458DEDB5A0F7C6B03EE8
:10BD70000000CDC338B505460C460020A0706070A9
:10BD800095F87A00002806D095F8741005F178002F
:10BD9000FFF77AFFA07095F87400002813D12846A9
:10BDA000FFF75EFE00280CD12846FFF793FE00281F
:10BDB00007D12846FFF720FF401E8041C043C00F37
:10BDC00000E0012060706078002805D1A178481E4D
:10BDD0008041C043C00F00E00120207031BD70B42D
:10BDE00000220378447B2418E370437B144610E060
:10BDF0005B1CDBB20A2593FBF5F505EB8506A3EB8F
:10BE00004603DBB21D18ED78661C16FB052292B2C4
:10BE1000641C0A2CECDB042008702D2A02DB0220B3
:10BE200048700BE0222A02DB0120487006E00F2A4E
:10BE300002DB0020487001E00020087070BC7047F1
:10BE400010B504469FED9C0A002008E000EB40017D
:10BE500004EB8101D1ED090A00EEA00A401C032881
:10BE6000F4DB04F05BFC84ED1C0ADFED940AB4EE15
:10BE7000600AF1EE10FA05D5002211460846BDE829
:10BE80001040B3E010BD000000401C4670B50C46E9
:10BE900004F59B65E97BAA7B121992F8E124891AC3
:10BEA000E973A97B091990ED1C0ADFED850AB4EE50
:10BEB000600AF1EE10FA03DB012081F8E10402E0F0
:10BEC000002081F8E104E87BA97B091991F8E114CD
:10BED0000818E873904E0022242106F50170F6F749
:10BEE000C7FA96F89A07042810D196F89B070028FD
:10BEF0000CD0E87B022803DA94F8D804002805D196
:10BF0000002204210220BDE870406FE070BD0000F7
:10BF1000CDCC4C3E30B591B07F4C04F5F2718878B1
:10BF2000401C88704A78002A0BD194F8E421002A3A
:10BF300002D1012284F8E42140B2072801D1012274
:10BF40004A7040B2072290FBF2F2C2EBC202801AA2
:10BF500088708888401C8880B4F86012491CA4F856
:10BF6000601280B2322190FBF1F1322202FB11010A
:10BF700031290BD194F88617491CC9B2052291FBCF
:10BF8000F2F202EB8202891A84F88617B0F5FA7F82
:10BF900024D104F518754022294600A8F6F7A6FA20
:10BFA0000022B82104F5F470F6F762FABDF800003B
:10BFB00040F2DC51884204D0402200A92846F6F71E
:10BFC00095FA04F28670C17C491CC9B20A2291FB21
:10BFD000F2F202EB8203A1EB4301C17411B030BD58
:10BFE000002240F29C714C48F6F742BA2DE9F0412C
:10BFF00006460C461546484F97F8990709300A211E
:10C0000090FBF1F101EB8102A0EB420800220A2132
:10C0100007F28F70F6F7A6FA5FFA88F808EB0700C8
:10C0200080F88F6707F2997044708570BDE8F081E1
:10C03000002803D03849B1F89A17018070470000F2
:10C040009A99993EF8B5344C01462046FFF794F989
:10C0500004F5F47504F52876324629462046FFF7A4
:10C06000E3FCB4F8E80140F2F31188420DD1284610
:10C07000FFF796FC04F28C7739462846FFF77AFEE4
:10C0800004F29A713846FFF7AAFEB4F8E8013221AB
:10C0900090FBF1F1322202FB1100312808D1284631
:10C0A000FFF7CEFE04F28C7231462846FFF7EEFE13
:10C0B000BDE8F1402EE700000000000052499D3924
:10C0C0000100C04085EB51B81E85F73FD7A3703DF6
:10C0D0000AD71540CDCCCCCCCCCC0040000054408D
:10C0E000000004C09A99999999991B400000F8BFE3
:10C0F0008DEDB5A0F7C6B03E0AD7E33FE17A14AEA6
:10C1000047E1BA3FC976BE9F1A2FAD3FEC51B81E2A
:10C1100085EBA13F9999E93F948A03000000000054
:10C12000FDF881C0232FE340DA1ED9C0F3456E40ED
:10C13000EDE88DBF0B030F3E2D8AE038A267283A49
:10C140008A81D23A5C560C3B8A81D23AA267283A5D
:10C150002D8AE03800000000AD9D27C0EE695740F1
:10C16000790B1FC088848C3F61738ABE9135EC3C8B
:10C1700061A1F13A0939353C4B87E23CDD04173DBA
:10C180004B87E23C0939353C61A1F13A00000000DF
:10C190001D1073BE20794C3FAE63E7BD2813F53DFB
:10C1A0005676F9BB3631F43A42CE113D63B55ABEEC
:10C1B0005EB1083FD24136BF5EB1083F63B55ABE9B
:10C1C00042CE113D10B588B0044600A81421F6F700
:10C1D000C5F905A800210A460B460EC00D222146CE
:10C1E00000A8F6F773F904F10D00CDF80D009DF8E5
:10C1F0000010062904DB0FF24010FAF775FF63E028
:10C200009DF80000002801D0022910D1BDF80300DC
:10C2100000280CD00422DDF80D1006A8F6F756F918
:10C220000422DDF80D00011D07A8F6F74FF99DF86F
:10C230000000042848D8DFE800F0030B132637007D
:10C24000DDF80D2005A99DF80100F8F7E1FD3BE0C0
:10C25000DDF80D2005A99DF80100F8F735FE33E063
:10C260009DF80100F9F7D3F800282DD09DF80100C2
:10C27000F8F7F1FE406A00F1080205A99DF80100F7
:10C28000F8F76EFE20E09DF80100FF2803D100A81A
:10C29000FAF742F918E0DDF80D30BDF803209DF8FB
:10C2A0000210F8F7ADFE0FE09DF80100FF2803D162
:10C2B00000A8FAF7ACF907E0DDF80D30BDF803206F
:10C2C0009DF80210F8F7AEFE08B010BD00B591B0B1
:10C2D00000A84021F6F742F900A9144804F08EFAAC
:10C2E00000A8FFF76FFFF7E710B584B0104C2346A6
:10C2F0001022402104F2344004F07AF90220029026
:10C300004FF49660019004F24C400090094B5A2281
:10C310000FF23C0104F5806004F076F91FBD80B592
:10C320000146024804F0A2F940B202BD4C7D030070
:10C3300018790300CDD200005B4552525D206F7624
:10C34000657220434D44204D41582025780000005F
:10C35000636D645F7461736B0000000030B4544916
:10C3600082680B6A9A188260012202744A692AB9AB
:10C37000026048610FF23100C8610CE001F1140362
:10C3800084689568651B012D03DB13461A68002A33
:10C39000F7D10260186048694A6A8068821A48BF0B
:10C3A000486230BC7047000010B5044610E0A06140
:10C3B0000168616100210174A069816081F31188C5
:10C3C000A06940688047802080F3118800BF00BFCB
:10C3D000606928B18168226A8A1A012AE7DB6162F2
:10C3E00010BD30B4002300241D4638C018C01438D6
:10C3F000C2608260416030BC704710B5802181F31B
:10C40000118800BF00BF017C294CC1B104F11401A7
:10C4100000E011460A6892B182420ED011460A68C5
:10C420006AB1824209D011460A6842B1824204D000
:10C4300011460A681AB18242EBD102680A60C168EB
:10C440008160FFF78BFF607808B980F3118810BD19
:10C45000802181F3118800BF00BF027C14490AB318
:10C460000022027482680B6AD21A826001F11402FF
:10C4700000E01A46136893B183420ED01A4613683F
:10C480006BB1834209D01A46136843B1834204D08A
:10C490001A4613681BB18342EBD1006810604869EB
:10C4A00000B9C861487808B980F311887047000066
:10C4B000C86703000EB400B582B003A9009102461C
:10C4C00000AB0121034878440A3004F0BDF906BCF2
:10C4D0005DF810FBF7980100010040F10980F44677
:10C4E000404200F005F851F000416047010000BFF4
:10C4F00009D0B0FA80F18840C91CC1F584610905F2
:10C5000001EBD0214005704780B54FF0FF3251EC70
:10C51000100B05F06FF841EC100B01BDF446400D17
:10C5200040EAC120490006D200F014F8004248BF9A
:10C530006FF00040604700F00DF84FF00041884276
:10C540008CBF084640426047400D40EAC120490088
:10C5500080F00D8040F00040490DA1F58061491C3C
:10C5600005D4D1F11F0154BFC840C01770474FF028
:10C5700000007047000000002DE9F8452DED088B04
:10C580000FB486B040F2FF7107989DED080B8DED5A
:10C59000040BC0F30A50884208D107980024000316
:10C5A00005BF069800280225012512E0012807DAB8
:10C5B00006A805F0CFF9012802DB0024002508E0D9
:10C5C000079A40F2FE3161F31E520792441A4FF06F
:10C5D000FF35002104A805F0DEF91A9F06460FB1C9
:10C5E0000020388036B9DDE908230020002105F05D
:10C5F00011FA12D0002D13D524B2012C15D1DDE98A
:10C6000006230020DFF88C1305F004FA05D0012E74
:10C610000BD1DF4905F0FEF93ED10AB0CD49E8E182
:10C62000022D04D1DDE90601E2E1012E6FDB022ECD
:10C6300008BFDDE9080100F0DB81012D2AD1079850
:10C640000028099806D4002854BF9FEDD50B9FED14
:10C65000D60BCBE100280ED456B94FF0FF3104A819
:10C6600005F099F9002848BF9FEDD10B00F1BE817C
:10C670009FEDCB0BBAE156B94FF0FF3104A805F09E
:10C680008AF9002848BF9FEDB40B00F1AF819FED00
:10C69000C60BABE1012E11D10998002824B206D4B3
:10C6A000012CACBF9FEDBE0B9FEDBF0B9EE1012C9B
:10C6B000ACBF9FEDBD0B9FEDBA0B97E10998002829
:10C6C00010D466B94FF0FF3104A805F064F90028D2
:10C6D00042BF079800289FEDA00B00F187819FEDD6
:10C6E000B20B83E100F0F2FC2221016066B94FF049
:10C6F000FF3104A805F04FF9002842BF0798002831
:10C700009FEDAB0B00F172819FEDA50B6EE10798D9
:10C71000002848BF002E0CD500F0D8FC2121016074
:10C720000AB04FF0FF30BDEC088B6FF00041BDE860
:10C73000F485DDE906010022002304F047F838BF44
:10C74000002509D381F00041CDE906014FF0FF310A
:10C7500004A805F020F90546012C13D1DDE90601F6
:10C760007F4A804B04F01AF80CD2DDE9062300263C
:10C770009FED7D8B00204FF08041FAF7ABF8CDE9BB
:10C7800006011CE0DDE906239FED798B00207A4944
:10C79000FAF7A0F853EC182BFAF710FCFFF7BEFEDF
:10C7A000A0F120063046FFF797FE0022734BFAF700
:10C7B00091F853EC182BFAF701FC41EC180B0FF22F
:10C7C000582000EB461ADDE9060153EC182BFAF766
:10C7D00035FBDDE9062341EC190B51EC180BFAF798
:10C7E000EDFB02460B4651EC190BFAF703FA41EC4C
:10C7F0001A0B53EC1A2BFAF76DF841EC1B0B8DED6D
:10C80000069B05F029F853EC1B2BFAF763F8DDE9DA
:10C810000623FAF713FB0646884600204D4953ECE1
:10C82000182BFAF70BFB00224FF08043FAF752F86F
:10C8300032464346FAF7C2FB53EC1A2BFAF74AF892
:10C84000DDE90623FAF7BAFB41EC180B4C4A4D4BD5
:10C85000FAF7D0F9CDE904012046FFF73DFE41EC9F
:10C86000190BDAE9000153EC192BFAF7A7FBDDE904
:10C870000423FAF7A3FBCDE90401DDE90823FAF765
:10C8800029F80022404BCDE9020103F087FFC0F0F8
:10C89000938001223D4B03F099FF40F291800022EA
:10C8A000002303F07BFFDDE9022339BF0020384974
:10C8B00000203849FAF782FBFFF730FE0446DDE935
:10C8C000080153EC182BFAF705F8CDE90201DAE973
:10C8D0000223DAE904019FED308BFAF76FFBDDE903
:10C8E0000823F9F7F7FF53EC182BF9F7F3FFDDE90D
:10C8F0000223FAF763FBCDE90201DAE9002351ECE8
:10C90000190BFAF75BFBDDE90823F9F7E3FF0646AD
:10C9100088462046FFF7E0FD02460B46304641467A
:10C92000FAF78CFA53EC182BF9F7D4FFDDE9022360
:10C93000FAF744FBCDE902010FB13C8000240094DA
:10C940000022044B02A805F075F8A8B3012837D0DF
:10C9500042E000BF0000F03F000000000000008047
:10C96000CD3B7F669EA0E63F000000000000F03F48
:10C97000000000000000E03F000050400000903F39
:10C98000EF39FAFE422EE63F0000E0C00000E04032
:10C990000000E0BF0000E03FEF39FAFE422EE63F24
:10C9A000000000000000F07F000000000000000018
:10C9B000000000000000F0FF0020CDE9020007E0C9
:10C9C0000020014902E000BF0000F07FCDE9020134
:10C9D00000F07CFB22210160002D1DBFDDE902017A
:10C9E00081F0004141EC100B9DED020B51EC100B5E
:10C9F0000AB0BDEC088BBDE8F48580B5002000903E
:10CA000053EC112B51EC100BFFF7B6FD41EC100B62
:10CA100001BD000000000000000000000000F0BFA9
:10CA20000000000000000080000000000000008006
:10CA30000000000000000000000000C05294EEBFA3
:10CA400000000048204E51BE000000F86467BCBCE6
:10CA50000000000000000000000000208133EDBF56
:10CA600000000080B3DB14BE000000506706A3BCCA
:10CA70000000000000000000000000D0E9DCEBBF77
:10CA800000000008C39259BE00000080B0D3B8BCBB
:10CA9000000000000000000000000070F98FEABFF5
:10CAA000000000C0A51028BE000000E8BFC0B0BC58
:10CAB000000000000000000000000070284CE9BFEA
:10CAC00000000060134B42BE000000C03D20B8BC17
:10CAD000000000000000000000000050FA10E8BF55
:10CAE000000000C05FF62BBE000000905C71A7BC88
:10CAF000000000000000000000000020FCDDE6BF98
:10CB0000000000C0F8F154BE00000018E9F6B9BCFE
:10CB10000000000000000000000000D0C3B2E5BF2C
:10CB200000000070E43254BE00000050DB06B4BCCC
:10CB3000000000000000000000000010EF8EE4BFC5
:10CB400000000020F36252BE000000C02A879ABC99
:10CB50000000000000000000000000B02272E3BFEF
:10CB6000000000F0E8E056BE00000028352DBDBCF6
:10CB70000000000000000000000000000A5CE2BFAE
:10CB8000000000B0FA8E41BE00000040AE6FBDBC98
:10CB9000000000000000000000000000564CE1BF53
:10CBA000000000F015CD5FBE00000000141C90BC1A
:10CBB000000000000000000000000040BD42E0BF97
:10CBC00000000030F93457BE000000E06C1E93BC3A
:10CBD0000000000000000000000000E0F57DDEBF66
:10CBE000000000B08A535EBE00000080DA77AABC65
:10CBF0000000000000000000000000C09D81DCBFBC
:10CC000000000000FFA226BE0000006057E2B0BC9A
:10CC1000000000000000000000000060F98FDABF93
:10CC2000000000580A8151BE000000F05F60B8BCEF
:10CC300000000000000000000000000098A8D8BF1D
:10CC4000000000607A7F45BE000000D05433A3BCD2
:10CC50000000000000000000000000600FCBD6BF05
:10CC6000000000D091CB40BE000000406D1BA0BC76
:10CC70000000000000000000000000A0FBF6D4BF90
:10CC800000000098C5CE52BE000000003A397EBCBC
:10CC90000000000000000000000000E0FE2BD3BFF9
:10CCA0000000004073872BBE00000000926879BC32
:10CCB000000000000000000000000040C069D1BF7B
:10CCC00000000058F16353BE00000080438D7CBC1F
:10CCD000000000000000000000000080D85FCFBF0F
:10CCE000000000181F8354BE000000B03F42A2BCE9
:10CCF00000000000000000000000008067FCCBBFC7
:10CD000000000060FAFF53BE00000050E00DB8BC08
:10CD100000000000000000000000000098A8C8BF4C
:10CD2000000000607A7F35BE000000C0543393BC21
:10CD3000000000000000000000000000DC63C5BF30
:10CD400000000058D6FF54BE00000000396490BCBB
:10CD50000000000000000000000000C0AD2DC2BFB8
:10CD600000000080A45915BE000000E0484BABBC99
:10CD70000000000000000000000000801A0BBEBF91
:10CD800000000050BF3C5ABE000000A0B364B6BC17
:10CD900000000000000000000000008004D6B7BFC3
:10CDA00000000040BBCF36BE0000008076CEA8BC9D
:10CDB00000000000000000000000008032BBB1BF96
:10CDC000000000402A0043BE00000028C60CBDBC85
:10CDD0000000000000000000000000009473A7BFE6
:10CDE000000000182B3B59BE000000C0E55DA5BC4B
:10CDF000000000000000000000000000EE4397BFAC
:10CE0000000000A0E6C340BE00000020958DB5BC28
:10CE10000000000000000000000000000000008092
:10CE20000000000000000080000000000000008002
:10CE300000000000000000000020704730B58BB0FB
:10CE4000040001D102204BE005A80FF25C112CC9AF
:10CE50002CC000210A460B460EC000A81421F5F78D
:10CE60007DFB1122214600A8F5F730FB9DF801401B
:10CE7000082C1FD19DF8000000280BD12320F8F7C3
:10CE8000C6FA002806D0002205A9CC20F7F7C0FF7B
:10CE9000012025E09DF8000001280BD1CC20F8F7F7
:10CEA000C2FA012806D1002205A9CC20F8F70CF817
:10CEB000012015E0232C12D19DF8000000280ED18E
:10CEC0000820F8F7A4FA002809D0002208A90820B1
:10CED000F7F7FAFF002205A9CC20F7F799FF002009
:10CEE0000BB030BD30B58BB0050001D102204AE057
:10CEF0000020029001902C780422691C02A8F5F70A
:10CF0000E5FA0422691D01A8F5F7E0FA21460FF2BF
:10CF1000A400FFF7CFFA2046F8F79DF800281DD0AF
:10CF20000025406A00280DD103A829460A460B4671
:10CF30000EC0029804900198059003A92046F7F7C7
:10CF400067FF0125F9F7BEF9012803D10820F9F799
:10CF500099F90125002D01D0002014E006A80FF258
:10CF600068011422F5F7C2FA00A80FF270010A68EE
:10CF700002608DF802400320ADF81B0000A906A84E
:10CF8000FAF7B0F902200BB030BD002803D0022818
:10CF900005D002D305E0084650E70846A2E7084658
:10CFA0004AE7002070470000010000000000000078
:10CFB0000000000023234548206E6F206576656ED3
:10CFC00074282564290A0000050000000000000004
:10CFD0000000000000000000000000000A1A00002D
:10CFE00010B52DED028B044682B094ED008A9FEDC2
:10CFF0002D0A28EE000AB5EE400AF1EE10FA8DED8A
:10D00000000AACBFF6EE000AFEEE000A30EE200A7F
:10D010008DED000A002100A804F06FFE9DED000ACE
:10D02000B5EE400AF1EE10FA17D0DFED1F0A20EE40
:10D03000200ADFED1E0A00EE608ADFED1D0A00EE19
:10D04000608ADFED1C0A00EE608ADFED1B0A00EE4D
:10D05000608ADFED1A0A00EE608A84ED008ADFED57
:10D06000180A9DED000AB4EE600AF1EE10FA06D43B
:10D07000DFED140AB4EE600AF1EE10FA05DBDFED25
:10D08000120A04F063FE8DED000A9DED000A02B065
:10D09000BDEEC00A10EE100ABDEC028B00F00300DA
:10D0A00010BD000083F9223F000080380000C9460F
:10D0B00000A0FD400020A23A000034330030C22E10
:10D0C000000000CF0100004F0000004F014804F0B5
:10D0D000DBBE0000000003001AA210EE101ADFF8F9
:10D0E00060C0F2EC060A614509DB00EE803A70EEA2
:10D0F000800A83EE200A40F0020010EE101A21F0A0
:10D10000004CDCF1665C0BD860EE000A20EE203AA1
:10D1100003EE010A01EEA02A42EE202A80EE220A46
:10D12000400810F0020F18BFB1EE400A02EB800277
:10D13000D2ED000A30EE200A28BFB1EE400A704757
:10D14000A430893ED7B3DD3F6AD5033F2B94A93D78
:10D15000B82A593F0000803F000080BF0000000057
:10D16000920A063FDB0FC93F920A863FDB0FC93F99
:10D17000920A0640DB0F4940368D2740DFED4A0A10
:10D1800060EE200A10B5B0EEE01ADFED481AB4EEFA
:10D19000611AF1EE10FA82B0044629D5F5EE400A84
:10D1A000F1EE10FAACBFB6EE001ABEEE001A70EE49
:10D1B000810AFDEEE00A10EE900AA8B1FAEEC90A63
:10D1C0009FED3B1A00EEC10A9FED3A1A00EEC10A2C
:10D1D0009FED391A00EEC10A9FED381A00EEC10A20
:10D1E0009FED371A00EEC10A00F00300041921E098
:10D1F0008DED000A0098C0F3C750FF2808D088B909
:10D20000009840020ED1002C4CD0B7EE000A13BD9E
:10D210000098400246D1FFF759FF212101609FEDA0
:10D22000290A13BD8DED000A00A8FFF7D9FE0419E5
:10D230009DED000ADFED240AB4EE600AF1EE10FA6B
:10D240000BDBDFED220AB4EE600AF1EE10FA04D532
:10D25000E00723D5B7EE000A20E0E00760EE000A01
:10D260000ED59FED1B0A9FED1B1A00EE801ADFED15
:10D270001A1A41EE201AB7EE000A01EEA00A0DE0DC
:10D28000DFED161A9FED162A00EEA12ADFED151A22
:10D2900020EE201A42EE201A01EE210AA00748BF14
:10D2A000B1EE400A13BD000083F9223F0000004F99
:10D2B0000000C94600A0FD400020A23A000034331F
:10D2C0000030C22EFFFFFF7FFEFF7FB900008039D4
:10D2D0009349B2BA36A02A3DDFFFFFBE6E8C4CB92F
:10D2E0004283083CA1AA2ABE1FB5FFF7EFFE212109
:10D2F00001601FBD08B584B00023029311B90093EB
:10D30000019302E00090481E019004AB00A9074879
:10D310007844183003F098FA009911B1009A00216E
:10D320001170002858BF029805B000BD1752FFFFCA
:10D3300000F10103810704D010F8011B89B18107B6
:10D34000FAD10268B2F10131914311F0803F04BF7C
:10D3500050F8042FF6E710F8011B11B110F8011B6B
:10D36000FBE7C01A7047000050EA010200F00E808F
:10D37000094200BF0BD1B0FA80F18840C1F19D0194
:10D38000C905020672F1004241EB10207047B1FA64
:10D3900081F241409040C2F1200261FA02F181EA3B
:10D3A000000018BF40F0010002F19D01E8E7000015
:10D3B000F0B591B004460D46002600AF17E0DFF847
:10D3C000C405335D1B111B5C3B70335D03F00F0321
:10D3D000185C07F8010F761C002007F8010F491CA4
:10D3E0009142ECDB00A90FF27860FFF763F8AE42E0
:10D3F00005DAAA1B212A00DB20220021F0E711B068
:10D40000F0BD01684A1C02600878704701688A1CF8
:10D4100002600878497840EA0120704701680A1DD7
:10D42000026008784A7840EA02208A7840EA02409E
:10D43000C97840EA0160704781B001680A1D026046
:10D4400008784A7840EA02208A7840EA0240C9789F
:10D4500040EA016000909DED000A01B0704713B5ED
:10D460000446012201A92068F5F730F82068401C25
:10D470002060012016BD13B50446022201A92068D0
:10D48000F5F724F82068801C2060022016BD13B533
:10D490000446042201A92068F5F718F82068001D49
:10D4A0002060042016BD38B504460D460094297846
:10D4B00000A8FFF7D4FF697800A8FFF7D0FFA9788C
:10D4C00000A8FFF7CCFFE97800A8FFF7C8FF29798B
:10D4D00000A8FFF7C4FF697900A8FFF7C0FFA9798A
:10D4E00000A8FFF7BCFFE97900A8FFF7B8FF297A89
:10D4F00000A8FFF7B4FF697A00A8FFF7B0FFA97A88
:10D5000000A8FFF7ACFFE97A00A8FFF7A8FF297B86
:10D5100000A8FFF7A4FF697B00A8FFF7A0FFA97B85
:10D5200000A8FFF79CFFE97B00A8FFF798FF297C84
:10D5300000A8FFF794FF697C00A8FFF790FFA97C83
:10D5400000A8FFF78CFFE97C00A8FFF788FF297D82
:10D5500000A8FFF784FF697D00A8FFF780FFA97D81
:10D5600000A8FFF77CFFE97D00A8FFF778FF297E80
:10D5700000A8FFF774FF697E00A8FFF770FFA97E7F
:10D5800000A8FFF76CFFE97E00A8FFF768FF297F7E
:10D5900000A8FFF764FF697F00A8FFF760FFA97F7D
:10D5A00000A8FFF75CFFE97F00A8FFF758FF95F898
:10D5B000201000A8FFF753FF95F8211000A8FFF7EF
:10D5C0004EFF95F8221000A8FFF749FF95F82310A9
:10D5D00000A8FFF744FF95F8241000A8FFF73FFFCD
:10D5E00095F8251000A8FFF73AFF95F8261000A837
:10D5F000FFF735FF95F8271000A8FFF730FF95F8E3
:10D60000281000A8FFF72BFF95F8291000A8FFF7B6
:10D6100026FF95F82A1000A8FFF721FF95F82B1098
:10D6200000A8FFF71CFF95F82C1000A8FFF717FFC4
:10D6300095F82D1000A8FFF712FF95F82E1000A8FE
:10D64000FFF70DFF95F82F1000A8FFF708FF95F8DA
:10D65000301000A8FFF703FF95F8311000A8FFF77E
:10D66000FEFE95F8321000A8FFF7F9FE95F833108A
:10D6700000A8FFF7F4FE0098001B32BD38B5044641
:10D680000D460094296800A8FFF701FF297900A83A
:10D69000FFF7E5FEE98800A8FFF7EDFE298900A85D
:10D6A000FFF7E9FEA97A00A8FFF7D9FEE97A00A8FA
:10D6B000FFF7D5FE297B00A8FFF7D1FE697B00A804
:10D6C000FFF7CDFE0098001B32BD10B582B00446B6
:10D6D0000094097800A8FFF7C2FE0098001B16BD51
:10D6E00038B504460D460094297800A8FFF7B7FE28
:10D6F000697800A8FFF7B3FE0098001B32BD10B593
:10D7000082B004460094097800A8FFF7A8FE0098AC
:10D71000001B16BD38B504460D46009500A8FFF75E
:10D7200070FE207000A8FFF76CFE607000A8FFF785
:10D7300068FEA07000A8FFF764FEE07000A8FFF785
:10D7400060FE207100A8FFF75CFE607100A8FFF783
:10D750005DFEE08000A8FFF761FEA06000A8FFF773
:10D760005DFEE06000A8FFF759FE206100A8FFF70A
:10D7700055FE606100A8FFF749FE208300A8FFF76F
:10D7800045FE608300A8FFF741FEA08300A8FFF7D5
:10D7900038FEA0770098401B32BD38B504460D46D0
:10D7A000009500A8FFF72DFE207000A8FFF729FEC6
:10D7B000607000A8FFF725FEA07000A8FFF73CFEF0
:10D7C00084ED010A00A8FFF737FE84ED020A00A8E5
:10D7D000FFF732FE84ED030A00A8FFF72DFE84ED6B
:10D7E000040A0098401B32BDF8B505460C460026D9
:10D7F0003746009400A8FFF704FE287000A8FFF742
:10D8000000FE687000A8FFF7FCFDA87000A8FFF7F5
:10D81000F8FDE87000A8FFF7F4FD287195F9040001
:10D82000412810DBA0F14007402028710BE000994F
:10D8300006EB860005EB80000830FFF7AEFF00998D
:10D8400040180090761C95F904008642EFDB002F0B
:10D8500003D0009800EB071000900098001BF2BD69
:10D8600038B504460D46009500A8FFF7CAFD2070A4
:10D870000098401B32BD38B504460D46009500A8FF
:10D88000FFF7BFFD207000A8FFF7BBFD6070009898
:10D89000401B32BD38B504460D46009500A8FFF781
:10D8A000B0FD20700098401B32BD70B59CB004469E
:10D8B0000E4602A86421F4F751FE00250FF218204D
:10D8C000D0E90023CDE900232046ADF80400E43878
:10D8D0000CD040F26131401A20D020380CD0AB3847
:10D8E00010D040F2C711401A12D01DE0314604A8F2
:10D8F000FFF7D9FD05461EE0314604A8FFF7BEFE3E
:10D90000054618E0314604A8FFF7DFFE054612E0A1
:10D91000314604A8FFF7E4FE05460CE0314604A8B2
:10D92000FFF7EDFE054606E022460FF24C110FF21E
:10D930005410FEF7BFFD2846ADF80000A0208DF87A
:10D94000080002ACA3206070062200A90DF10A00B5
:10D95000F4F7BCFD05F10800B0210155B32102AA7E
:10D9600082185170841C08480078002803D0214692
:10D9700002A8FFF71DFD214602A800F051F91CB0D6
:10D9800070BD0000CC6E0300F46F030070B5ADF500
:10D99000FD6D04460E46002500A840F2E471F4F740
:10D9A000DDFD06F1120100A800F0DAF8082851DBCD
:10D9B0009DF80000A0284ED100A84178A3294AD1A3
:10D9C0008188090401D5042100E02946BDF8022020
:10D9D00011FA82F10831BDF80650085CB0283AD13E
:10D9E00000A808184078B32835D1284640F24531C0
:10D9F000401A0ED04FF48071401A1ED0CB3812D08E
:10DA000040F2C711401A13D046F63321401A05D010
:10DA100018E002A92046FFF77DFE1CE002A920467F
:10DA2000FFF7E2FE17E002A92046FFF719FF12E018
:10DA300002A92046FFF71FFF0DE002A92046FFF7CD
:10DA400029FF08E02A460FF260010FF26C00FEF792
:10DA500031FD00E0054628460DF5FD6D70BD000066
:10DA60005B495D5B20676E737350726F746F636F99
:10DA70006C205D2025730A006265747057726170B6
:10DA8000706572005B495D5B202573205D20556EDB
:10DA900068616E646C6564206D6573736167652091
:10DAA000256C750A0000000062657470556E77720F
:10DAB00061707065720000005B495D5B202573201A
:10DAC0005D20556E68616E646C6564206D6573736E
:10DAD0006167652025690A0000000200000000005F
:10DAE00010F0030001D0C0F1040080B2704738B5D7
:10DAF000744C0020E060A060606020600120206124
:10DB000060610FF2E825E3686F4A29460FF2E820CA
:10DB1000FEF7D0FCA3686D4A29460FF20430FEF7E9
:10DB2000C9FC63686A4A29460FF21C30FEF7C2FC42
:10DB30002368224629460FF23830FEF7BBFC2369E2
:10DB4000644A29460FF25030FEF7B4FC6369624A1A
:10DB500029460FF2703001B0BDE83040FEF7AABC94
:10DB60002DE9F04188B004460D46002604A80FF2C6
:10DB700080318CC98CC059484088ADF812002846C5
:10DB8000ADF81600514F78680090386801904FF456
:10DB9000006002904FF47D30039000980199884214
:10DBA0003AD00C2204A900A800F09AF80C282FD132
:10DBB000BDF810004AF6CD31884229D1BDF8168053
:10DBC0004046FFF78DFF10FA88F0A0F10C08BDF871
:10DBD0001400C10BC0F3803090EA010F05D06FF044
:10DBE000010601984044386016E0A84502D34FF082
:10DBF000FF3611E04246214600A800F071F840458A
:10DC00000AD101983860BDF81600A0F10C0603E0B7
:10DC10006FF0020600983860304608B0BDE8F08129
:10DC20002DE9F04188B004460D4605A80FF2CC213D
:10DC30004CC94CC0294E7088ADF8160005F10C0097
:10DC4000ADF81A0030888DF81D000027DFF87480C9
:10DC5000D8F804000190D8F8000002904FF47A70D0
:10DC600003904FF47F3004900C2205A901A800F026
:10DC70007BF80C2822D12A46214601A800F074F82E
:10DC8000A8421BD100A839460160284680B2FFF7A0
:10DC900027FF0446224600A901A800F065F8A0422B
:10DCA0000CD17088401C70803088401C30800198F6
:10DCB000C8F80400022004F0F7F82F46384608B0F0
:10DCC000BDE8F081E8FF0300F4FF0300F0FF03006C
:10DCD000ECFF0300F8FF0300FCFF030040D9030042
:10DCE0002DE9F84F04460D4616462768D4F804B0CF
:10DCF000A0685F4503D23918A1EB0B0801E0A7EB40
:10DD00000B085F4502D2A0EB0B0901E0A7EB0B0962
:10DD1000CA46B14500D9B2465246E0680BEB000155
:10DD20002846F4F7D3FBD344A068834501D14FF0D4
:10DD3000000BB1450ED2C1450CD2A6EB0A008742BA
:10DD400000D90746BB465A46E1680AEB0500F4F7DE
:10DD5000BDFBDA44A068834501D14FF0000BC4F845
:10DD600004B05046BDE8F28F2DE9F04704460D4659
:10DD70001646E768D4F800806068804503D2A0EBBF
:10DD80000801491E04E0A1684118A1EB0801491EE1
:10DD9000B14201D2002027E0804504D2A0EB080068
:10DDA000A0F1010902E0A068A0EB0809CA46B1454C
:10DDB00000D9B2465246294608EB0700F4F786FB25
:10DDC000D044B14508D2A6EB0A0842460AEB050149
:10DDD0003846F4F77BFBC244A068804501D14FF080
:10DDE0000008C4F800805046BDE8F08773686D698C
:10DDF00070635F696E6974005B495D25733A4348DF
:10DE000055425F53484D4950435F52585F48454122
:10DE100044283078257829203D20307825780A005C
:10DE20005B495D25733A434855425F53484D49501D
:10DE3000435F52585F5441494C2830782578292057
:10DE40003D20307825780A005B495D25733A4348C8
:10DE500055425F53484D4950435F54585F484541D0
:10DE600044283078257829203D20307825780A000C
:10DE70005B495D25733A434855425F53484D4950CD
:10DE8000435F54585F5441494C2830782578292005
:10DE90003D20307825780A005B495D25733A434878
:10DEA00055425F53484D4950435F54585F49504372
:10DEB0005F4D5347283078257829203D203078253C
:10DEC000780A00005B495D25733A434855425F5329
:10DED000484D4950435F52585F4950435F4D534747
:10DEE000283078257829203D20307825780A0000D0
:10DEF000CDAB0000C000000000000000CDAB000072
:10DF0000C000000000000000012100F01F0291404D
:10DF1000DFF84C21400942F820107047012100F041
:10DF20001F029140DFF83C21400942F82010704761
:10DF300080B50FF24810FEF7BDFADFF82C01002182
:10DF4000016041610161BDE8014004F02AB87047F9
:10DF50007CB504F032F804460D46444ED6E9002361
:10DF60009D4208D801D3944205D2CDE900450FF275
:10DF7000B010FEF79FFAC6E90045204629467CBD51
:10DF800080B504F01AF84FF47A72BDE8084004F046
:10DF90007BB9F8B504460D4616461F4645EA04000F
:10DFA00030430FD121460FF2BC10FEF783FA4FF435
:10DFB000AD720FF2E4010FF2D400FEF77BFA0020FD
:10DFC000C046C046B6F57A7F08D34FF47A70B6FBE8
:10DFD000F0F045194FF47A7101FB1066B5F57A7FC0
:10DFE00008D34FF47A70B5FBF0F004194FF47A714E
:10DFF00001FB105500F025F81B4A069810701C48CC
:10E000006421694300FB041030180021C2E90201B9
:10E01000380000D0176132462946204603F0F7FF4A
:10E02000BDE8F14002E010480078704780B501205B
:10E0300004F0F7F801200C4988701420BDE8024074
:10E0400062E780B5002004F0ECF8074800218170F9
:10E05000C078002803D11420BDE802405EE701BD6E
:10E0600000E100E080E100E0C8D7030020D9030010
:10E0700040420F0000200146704700005B495D727E
:10E080007463496E69742E2E2E0A00005B455D256F
:10E09000732C2025640A0000443A5C576F726B5C55
:10E0A00050345C53454E534F525F43483932344BE2
:10E0B000494D5F53454E534F524855425F4D415372
:10E0C000535F313731365C4D4153535F50524F4AA5
:10E0D0004543545C50524F445C4D3331535C535C68
:10E0E000706C6174666F726D5C6578796E6F733990
:10E0F0003631305C6669726D776172655C6F735C36
:10E10000706C6174666F726D5C6578796E6F735C4C
:10E110007372635C7274635C7274632E63000000DC
:10E120005B455D4F6F7073212C206C6173745F735E
:10E13000797374656D5F74696D655F6E7365632077
:10E1400028256C6C75292C2073797374656D5F7448
:10E15000696D655F6E7365632028256C6C75290A8F
:10E16000000000005B455D7274635365745469631D
:10E170006B54696D652829202D20736563282564FB
:10E180002920697320696E76616C69640A00000059
:10E1900035488168002904BF08B008E0EFF3098220
:10E1A000A2F12802036882E8F84F83685A60FCF7FE
:10E1B000EFF8816879B14A6892E8F84F036002F19C
:10E1C000280282F3098890692849814202D013F419
:10E1D0007F4F43D07047264826490968401A80F38C
:10E1E00008884FF08071C161234981617FF0060E7C
:10E1F000704701BC2046DFF884E000BDFEE7204800
:10E2000000681C490968401A203820F0070080F394
:10E2100008884FF000011448417081F3118862B6FC
:10E2200000F018F8FEE703680CB44FF000014170ED
:10E230004FF0000181F311881249134A0A604FF030
:10E24000800181F311880CBC036070470D490E4AB0
:10E250000A6070470B490C4A0A6070474FF0000192
:10E2600081F3118870470000C867030042F2000084
:10E27000E81F030074D50000010E0200FDF100004C
:10E280000010000004ED00E00000001004F030B8C1
:10E2900080B521280BDB25220FF2C4110FF2B41038
:10E2A000FEF708F90020BDE8024004F0FDBFBDE81C
:10E2B000044004F02DB880B521280CDB2E220FF28B
:10E2C000A0110FF29010FEF7F5F80020C046C046EE
:10E2D0004FF0FF3002BDBDE8024004F037B880B512
:10E2E00021280BDB39220FF278110FF26810FEF7AC
:10E2F000E1F80020BDE8024004F0D6BFBDE80440CC
:10E3000004F041B880B521280CDB45220FF25011F2
:10E310000FF24010FEF7CEF80020C046C0464FF086
:10E32000FF3002BDBDE8024004F04BB880B52128A3
:10E330000BDB51220FF228110FF21810FEF7BAF87A
:10E340000020BDE8024004F0AFBFBDE8044004F087
:10E3500057B880B521280BDB5E220FF204110FF2B3
:10E36000F400FEF7A7F80020BDE8024004F09CBFCF
:10E37000BDE8044004F062B880B521280BDB6A22B6
:10E380000FF2DC010FF2CC00FEF794F80020BDE89C
:10E39000024004F089BFBDE8044004F06DB880B5C8
:10E3A00021280BDB76220FF2B8010FF2A800FEF74E
:10E3B00081F80020BDE8024004F076BFBDE80440CB
:10E3C00004F078B838B521280BDB85220FF29001D4
:10E3D0000FF28000FEF76EF80020BDE8324004F036
:10E3E00063BF05290BDB8A220FF274010FF2640070
:10E3F000FEF760F80020BDE8324004F055BF012A66
:10E400000DD1802B0BD38F220FF254010FF2440059
:10E41000FEF750F80020BDE8324004F045BF049CF0
:10E42000250002D0009404F053FF31BD80B52128AF
:10E430000CDB4FF487720FF228010FF21800FEF781
:10E4400039F80020BDE8024004F02EBFBDE80240CC
:10E4500004F0E0B85B455D25732C2025640A0000BC
:10E46000443A5C576F726B5C50345C53454E534F6B
:10E47000525F43483932344B494D5F53454E534FF9
:10E48000524855425F4D4153535F313731365C4DF1
:10E490004153535F50524F4A4543545C50524F448E
:10E4A0005C4D3331535C535C706C6174666F726D9C
:10E4B0005C6578796E6F73393631305C6669726D80
:10E4C000776172655C6F735C706C6174666F726D9E
:10E4D0005C6578796E6F735C7372635C6770696F8B
:10E4E0005C6770696F2E630080B504F0E2FF0D4930
:10E4F000086001BD80B500F025F80B4805F010FF5D
:10E50000012005F02CFFFFF7C1FE05F091FF05F09B
:10E51000A3FFFFF70DFD0FF21400BDE80240FDF769
:10E52000C9BF0000F06F030000EA3206537973742C
:10E53000656D20626F6F7420646F6E6520212121EC
:10E540000A00000080B506F08AF806F06DF906F0C2
:10E55000EAF9BDE8014003F0D5BCF8B504460D4624
:10E5600016461F46002C0DD10FF2F000FDF7A2FF5A
:10E5700036220FF218110FF20810FDF79BFF002052
:10E58000C046C046002D0DD10FF29010FDF792FF4E
:10E590003B220FF2F8010FF2E800FDF78BFF00209D
:10E5A000C046C04606F002FA002805D13A46314678
:10E5B0000FF28810FDF77EFF29462046BDE8F440A3
:10E5C00006F02CB9F8B504460D4616461F46002C39
:10E5D0000DD10FF28410FDF76DFF49220FF2AC014F
:10E5E0000FF29C00FDF766FF0020C046C046002DDC
:10E5F0000DD10FF28410FDF75DFF4E220FF28C015A
:10E600000FF27C00FDF756FF0020C046C0463000E8
:10E610000DD10FF28410FDF74DFF53220FF26C0164
:10E620000FF25C00FDF746FF0020C046C0463B46A7
:10E6300032462946204601B0BDE8F04006F0E8B871
:10E6400010B5044606F05CF9012C04D02046BDE864
:10E65000104006F03AB910BD000000005B455D6D4A
:10E6600061696C626F7857726974652829202D2062
:10E67000627566206973204E554C4C0A00000000FC
:10E680005B455D25732C2025640A0000443A5C57E5
:10E690006F726B5C50345C53454E534F525F43482E
:10E6A0003932344B494D5F53454E534F52485542D2
:10E6B0005F4D4153535F313731365C4D4153535FAA
:10E6C00050524F4A4543545C50524F445C4D333195
:10E6D000535C535C706C6174666F726D5C657879C5
:10E6E0006E6F73393631305C6669726D7761726551
:10E6F0005C6F735C706C6174666F726D5C65787969
:10E700006E6F735C7372635C6D61696C626F785C71
:10E710006D61696C626F782E630000005B455D6D12
:10E7200061696C626F7857726974652829202D20A1
:10E7300073697A6520697320300A00005B495D6D5A
:10E7400061696C626F7857726974654576743A20B6
:10E750002573282564290A005B455D6D61696C623B
:10E760006F78526561642829202D206275662069C2
:10E7700073204E554C4C0A005B455D6D61696C62BF
:10E780006F78526561642829202D2073697A65208D
:10E79000697320300A0000005B455D6D61696C6241
:10E7A0006F78526561642829202D2063616C6C624A
:10E7B00061636B206973204E554C4C0A00000000C9
:10E7C00010B5044606F0DAFA01200549605410BD80
:10E7D000002106F042BB06F08CBC06F0E3BC000052
:10E7E00028D903000C2802D36FF400407047854AF3
:10E7F00042F8201006F05BBE2DE9F84F04460C2CC1
:10E8000080F0898006F0C6FF05467F4810F8146046
:10E8100000EB440047783046FFF74DFD8046384610
:10E82000FFF749FD8146204606F07DFE3846FFF79A
:10E8300069FD83463046FFF765FD824652465946DC
:10E840000FF2C810FDF736FEBBF1010F63D0BAF12D
:10E85000000F1AD14FF0000B04E00A2004F012FD63
:10E860000BF10A0BBBF5FA7F08D23046FFF74AFDE1
:10E870008246BAF1000FF0D14FF0000BBBF1000F50
:10E8800003D00FF2A810FDF715FE3846FFF73AFD4A
:10E890008346BBF1000F2DD101213046FFF7F8FC74
:10E8A00000213846FFF7F4FC4FF0000A01E00AF1BE
:10E8B000010ABAF1640F16DA00213046FFF70FFDA6
:10E8C000052004F0CBFC01213046FFF708FD0520B0
:10E8D00004F0C4FC3846FFF715FD0128E7D10FF21C
:10E8E0006C10FDF7E7FDBAF1640F03D10FF2781059
:10E8F000FDF7E0FD41463046FFF7CAFC4946384681
:10E90000FFF7C6FC204606F0D9FC29462046BDE8A4
:10E91000F44F06F0CCBDBDE8F18FF0B587B00446EA
:10E920001D460C2C01D2080602D56FF400401CE0F5
:10E9300001910D9E03960C9805900495069201A9ED
:10E94000204606F0D3FE070004D02046FFF754FF10
:10E9500038460AE00E98010006D0002100913346A7
:10E960002A460F9907F01EF8002007B0F0BD39E7DE
:10E970001FB5069C002C01D0002B02D16FF4004083
:10E9800009E0227000220392029201930094012375
:10E990002246FFF7C2FF04B010BD2DE9FF47054630
:10E9A0000E4690469946DDF830A0BAF1000F02D02D
:10E9B000B9F1000F02D16FF4004020E009F1010726
:10E9C0003846FAF7AFFF040002D14FF0FF3016E0EF
:10E9D0004A465146601CF3F779FD84F80080002018
:10E9E00003900290019000903B4622463146284613
:10E9F000FFF793FF05462046FAF7ACFF284604B020
:10EA0000BDE8F0871CD50300586E03005B495D53D9
:10EA10004441206C696E653A25642C2053434C2098
:10EA20006C696E653A25640A000000005B455D5321
:10EA3000434C206C696E65206973207374696C6C3B
:10EA4000204C4F572121210A000000005B495D53F3
:10EA50004441206C696E65206973207265636F762E
:10EA6000657265640A0000005B455D534441206C9B
:10EA7000696E65206973206E6F74207265636F76AE
:10EA8000657265640A00000070B504463748384E68
:10EA90000568B5B1287A88B16868A0420ED1012016
:10EAA00028723078401C3070287A401E2872C0B21C
:10EAB00010B9284606F07EFFFBF7F8FCED68002D44
:10EAC000E8D170BD2B492C4A0A60002100220B4678
:10EAD0008C46A0E80E101038802181F3118800BF09
:10EAE00000BF22490A68C26008602148407808B91E
:10EAF00080F31188704730B51D4D04462878401CBE
:10EB0000287081B0A868217A39B960600125257222
:10EB1000FBF7CCFC284601B030BD6168814208D0CB
:10EB20001021204606F05CFF207A0028F8D1A86862
:10EB30006060207A451C2572FBF7B8FC284601B0BE
:10EB400030BD0B490A78521C0A70017A491E0172C5
:10EB5000C9B2002918BFFBF7A9BC00B581B006F007
:10EB600029FF01B05DF804EBFBF7A0BC58D9030006
:10EB7000C867030038D9030089FA000000F5E07087
:10EB80000268914203D343689A18914202D3806885
:10EB90000028F5D17047DFF86007016891B94FF49C
:10EBA000803181604FF4805141604FF0FF31C1608E
:10EBB00001610421DFF844274161C2F8BC11DFF88C
:10EBC000401701600120704701F1080313F00703AB
:10EBD00005D001F10803C3F1080303F00703591836
:10EBE000D21A8161C26042F001034B6051182823A0
:10EBF0004B60DFF804170969C16170472DE9F04FD8
:10EC0000064601F1080010F0070083B008BF8846EF
:10EC100007D001F10800C0F1080000F0070000EB88
:10EC2000010802F1080010F0070006D002F1080008
:10EC3000C0F1080000F0070082181546A5EB080097
:10EC4000A0EB030943F0030003EB080BC8F8040032
:10EC5000AB4528BF06F0E2FE2879C00758BF06F092
:10EC6000DDFEB9F1100F38BF06F0D8FEB06985425D
:10EC700009D1F0684844F060C6F818B040F00100CF
:10EC8000CBF804006DE1706985420BD1B06848444F
:10EC9000B060C6F814B040F00101CBF8041040F8A1
:10ECA0000B005EE1686800F00301012940F0AD80CF
:10ECB000C008C0000190C00820283AD2D5F808A0AA
:10ECC000EF680090BD4208BF06F0A8FE554508BF9A
:10ECD00006F0A4FE68680099C008C000B0EBC10F40
:10ECE00018BF06F09BFE009806EBC00000F128015B
:10ECF0008A4507D031698A45C0F08280DAF80C1065
:10ED0000A9427DD1574506D1009A30680121914032
:10ED10008843306076E02830874205D030698742EA
:10ED20006ED3B868A8426BD1CAF80C70C7F808A0B7
:10ED300068E0EF68D5F818A0AF420CD0A868316938
:10ED4000884223D3C168A94204BFB968A9421DD132
:10ED5000C760B8601CE005F11400076837B905F119
:10ED600010000768A7B101E00846076807F1140121
:10ED70000A68002A02BF07F110010A68002AF3D1CD
:10ED80003169884202D30021016001E006F046FEAD
:10ED9000BAF1000F36D0E86906EB800000F59870F4
:10EDA00001688D4208D10760A7B9EA69706801213E
:10EDB00091408843706025E03069824508D3DAF8D5
:10EDC0001000A84214BFCAF81470CAF8107001E00D
:10EDD00006F024FEB7B13069874211D3C7F818A0F6
:10EDE000296929B1814226BF39618F6106F016FE7B
:10EDF000686938B13169884202D37861876101E07E
:10EE000006F00CFE019845198144686840084000EE
:10EE100068604FEAD90549F00100CBF8040049F8D1
:10EE20000B90202D23D206EBC50000F12807B9F185
:10EE3000100F38BF06F0F2FD306820FA05F1C9075F
:10EE4000BA4604D40121A9400843306006E0B868FE
:10EE5000316988422CBF824606F0E0FDC7F808B051
:10EE6000CAF80CB0CBF808A0CBF80C7079E05FEAD8
:10EE7000192108BF002023D0B1F5803F28BF1F20F3
:10EE80001ED2A1F58070000C00F008008140A1F5B1
:10EE90008052120C02F004029140A1F580431B0C39
:10EEA000C0F10E0003F00203801AC01A994000EB73
:10EEB000D130C11D29FA01F202F0010101EB40003D
:10EEC000CBF81C000022CBF81420CBF8102006EB66
:10EED0008001726822FA00F3DB0701F5987107D40C
:10EEE000012303FA00F010437060C1F800B01DE088
:10EEF0001F2809680EBF00204008C0F1190009FA58
:10EF000000F000E011464A68D208D2004A4514D009
:10EF1000C20F01EB820202F1100340001A68002ABE
:10EF2000F0D1306983421AD3C3F800B0CBF818107F
:10EF3000CBF80CB0CBF808B013E032698868914286
:10EF400028BF90420BD3C0F80CB0C1F808B0CBF882
:10EF50000800CBF80C100020CBF8180001E006F0F8
:10EF60005DFD08F1080000F005BE2DE9FA4D0546EB
:10EF7000DFF88403006884B008B9FFF70CFEDFF8FF
:10EF800078030499806841182F31401E21EA00005F
:10EF90000499814280F0AB8105F5D876B16841B122
:10EFA000D5F8B0218018824280F0A1818142C0F062
:10EFB0009E8106F037FD00281EBF0446D0F8008071
:10EFC00014F1010F00F09381D5F8B0014044C5F869
:10EFD000B0017168814238BF01467160A86980BB89
:10EFE000286908B1844200D22C613461C6F81480CB
:10EFF0000020F06105F12801BF48006868624FF009
:10F00000FF3028620020C960896001F10802801C7D
:10F010001031D26020289260F5D3B848854203D1E0
:10F02000A8F12802214629E055F8040CC00805EB98
:10F03000C000A0F1080108EB0400401AA0F128026A
:10F040001CE005F5E071084600E08068D0B1026878
:10F0500043689A189442F8D1027B120712D4AA6925
:10F0600003689A420ED347683B449A420AD208EB9F
:10F0700007014160E868A96908EB00022846FFF72C
:10F08000A3FD1EE128698442084638BF2C6108EBC5
:10F09000040100E0806880B102688A42FAD1017BF5
:10F0A00009070AD404604168414441602146049B39
:10F0B000284606B0BDE8F04DA0E5AF6939462846C0
:10F0C000FFF75CFD01684068401802902F3800F19E
:10F0D000080111F0070105D000F10801C1F1080194
:10F0E00001F00701081807F11001884234BF0097AA
:10F0F000009000980830019004F10801009800F198
:10F10000180A11F007014FF0000BA8F1280005D0F4
:10F1100004F10801C1F1080101F007010A19401AC0
:10F12000AA61E86040F00101516080182821416027
:10F1300071480069E861019810F0070018BF06F0F7
:10F140006DFC00991B20486005F5E071B1E80C509A
:10F150000198A0E80C503461C6F81480C6F81CB0C1
:10F160000198B061029800E08A460722CAF804209C
:10F170000AF104010A1D82420BF1010BF4D3BBF129
:10F18000020FB8BF06F04AFC0098B84200F0998020
:10F19000C01BC119C4084A68520852004A6040F0B6
:10F1A00001017960C051202C20D205EBC40101F18E
:10F1B0002806102838BF06F031FC286820FA04F130
:10F1C000C907B04604D40121A1400843286006E0E5
:10F1D000B068296988422CBF804606F01FFCB760E2
:10F1E000C8F80C70C7F80880FE606AE0010A08BF22
:10F1F000002223D0B1F5803F28BF1F221ED2A1F5E7
:10F200008072120C02F008029140A1F580531B0C91
:10F2100003F004039940A1F58044240CC2F10E02CE
:10F2200004F00204D21A121BA14002EBD131CA1D14
:10F2300020FA02F303F0010202EB4102FA6100231B
:10F240007B613B6105EB82016B6823FA02F4E40702
:10F2500001F5987105D401209040184368600F6053
:10F260001CE01F2A09680EBF00225208C2F11902D1
:10F2700000FA02F200E019464B68DB08DB0083422B
:10F2800010D0D30F01EB830303F110045200236865
:10F29000002BF0D12869844211D32760B961FF6047
:10F2A000BF600EE02A698868914228BF904206D369
:10F2B000C7608F60B860F9600020B86101E006F0B7
:10F2C000ADFBE8680499814211D2401AE860A9694F
:10F2D000049A5218AA6140F001005060049840F06E
:10F2E0000300486006B001F10800BDE8F08D002081
:10F2F00006B0BDE8F08D0000F8D7030018BB03008E
:10F300006859883C2DE9F04D0446884600265FEA9E
:10F310001820C8F1000B08BF002123D0B0F5803FB2
:10F3200028BF1F211ED2A0F58071090C01F0080131
:10F330008840A0F58052120C02F004029040A0F523
:10F3400080431B0CC1F10E0103F00203891AC91A94
:10F35000984001EBD030C11D28FA01F202F0010102
:10F3600001EB400104EB8100D0F8300128B31F29E4
:10F370000EBF00224A08C2F1190208FA02F2002365
:10F3800000E052004768FF08FF00A7EB08075F4551
:10F3900003D25FEA070B06460BD04769D50F00EB97
:10F3A0008500002F00691CBF87423B460028E8D13A
:10F3B000184600283CD1002E3CD101208840400056
:10F3C000414208436168084000F0678141420840BB
:10F3D000411E080B00F0100021FA00F2510901F063
:10F3E000080122FA01F39A0802F00407FB405A08C8
:10F3F00002F00205081823FA05F23844C2F340036C
:10F400002818181822FA03F1081804EB8000D0F825
:10F4100030010DE008464168C908C900A1EB0801A8
:10F4200059453CBF8B46064601690029F2D1406927
:10F430000028F0D1002E00F03081A068A0EB080079
:10F44000834580F02A8120698642C0F0248170685B
:10F45000C008C00008EB0B01884208EB060518BF86
:10F4600006F0DCFAAE4280F01681F768D6F818A0F4
:10F47000B7420CD0B0682169884223D3C168B14239
:10F4800004BFB968B1421DD1C760B8601CE006F185
:10F490001400076837B906F110000768A7B101E04A
:10F4A0000846076807F114010A68002A02BF07F13D
:10F4B00010010A68002AF3D12169884202D3002191
:10F4C000016001E006F0AAFABAF1000F38D0F06945
:10F4D00004EB800000F5987001688E4209D1076046
:10F4E000380014D1F269606801219140884360605E
:10F4F00026E02069824508D3DAF81000B04214BF34
:10F50000CAF81470CAF8107001E006F087FABFB1AB
:10F510002069874212D3C7F818A0306930B1216939
:10F52000884226BF3861876106F078FA706938B181
:10F530002169884202D37861876101E006F06EFAA2
:10F54000BBF1100F0CD208EB0B0040F00300706011
:10F5500008EB0B008019416841F00101416096E021
:10F5600048F0030070604BF0010068604FEADB0078
:10F570004BF805B020281DD204EBC00101F128078B
:10F58000216821FA00F2D207BB4605D4012202FA13
:10F5900000F00843206006E0B868216988422CBF6B
:10F5A000834606F03BFABD60CBF80C50C5F808B0B6
:10F5B000EF606CE05FEA1B2108BF002023D0B1F5AB
:10F5C000803F28BF1F201ED2A1F58070000C00F0E4
:10F5D00008008140A1F58052120C02F00402914013
:10F5E000A1F580431B0CC0F10E0003F00203801A4A
:10F5F000C01A994000EBD130C11D2BFA01F202F084
:10F60000010101EB4000E86100226A612A6104EB1C
:10F610008001626822FA00F3DB0701F5987106D4D5
:10F62000012303FA00F0104360600D601CE01F2806
:10F6300009680EBF00204008C0F119000BFA00F065
:10F6400000E011464A68D208D2005A4510D0C20FD5
:10F6500001EB820202F1100340001A68002AF0D187
:10F660002069834211D31D60A961ED60AD600EE099
:10F6700022698868914228BF904206D3C5608D6098
:10F68000A860E9600020A86101E006F0C7F906F172
:10F690000800BDE8F08D06F0C1F90020BDE8F08D4E
:10F6A0002DE9F84F04468846606841420840411EF3
:10F6B000080B00F0100021FA00F2510901F00801D6
:10F6C00022FA01F39A0802F0040223FA02F56B0809
:10F6D00003F00203081825FA03F61018C6F34005D4
:10F6E0001818284426FA05F1081804EB8000D0F811
:10F6F00030014168C908C9000646A1EB080A09E0C3
:10F7000008464168C908C900A1EB080151453CBF42
:10F710008A46064601690029F2D140690028F0D1E5
:10F7200020698642C0F0C4807068C00808EB0A09EE
:10F73000C000484508EB060B18BF06F06FF95E45A0
:10F7400080F0B680F768B569B7420CD0B06821691F
:10F75000884223D3C168B14204BFB968B1421DD108
:10F76000C760B8601CE006F11400076837B906F1FD
:10F7700010000768A7B101E00846076807F1140107
:10F780000A68002A02BF07F110010A68002AF3D1B3
:10F790002169884202D30021016001E006F03EF9B0
:10F7A000002D34D0F06904EB800000F598700168FA
:10F7B0008E4209D10760380011D1F26960680121D9
:10F7C00091408843606022E02069854205D3286922
:10F7D000B04214BF6F612F6101E006F01FF9B7B1AD
:10F7E0002069874211D3BD61306930B121698842F7
:10F7F00026BF3861876106F011F9706938B1216957
:10F80000884202D37861876101E006F007F9BAF116
:10F81000100F09D249F00300706009EB060041683F
:10F8200041F0010141603FE048F0030070604AF0A0
:10F830000100CBF804004AF80BA0D4F808804FEA86
:10F84000D805202D28BF06F0E9F8B8F1000F27D021
:10F85000D4F81490009504EBC50000F12805B8F128
:10F86000100F38BF06F0DAF82068009920FA01F28C
:10F87000D1072F4605D4009A01219140084320600A
:10F8800006E0A868216988422CBF074606F0C6F842
:10F89000C5F80890C7F80C90C9F80870C9F80C5062
:10F8A000C4F808A0C4F814B006F10800BDE8F28F4F
:10F8B00006F0B4F80020BDE8F28F2DE9F04F83B0D8
:10F8C0000546C046C046F52DDFF8C04780F00781E9
:10F8D0000B2D31BF102705F10B00C008C7002168B0
:10F8E000FE0821FA06F010F0030F42D0C04300F0EA
:10F8F0000100861904EBC60000F12808F700D8F8CB
:10F9000008506868C008C000B84218BF06F086F802
:10F91000D5F80890454508BF06F080F84D4508BF6A
:10F9200006F07CF86868C008C000B84218BF06F04E
:10F9300075F8C84505D120680121B1408843206091
:10F940000DE02069814508D3D9F80C00A84204D104
:10F95000C8F80890C9F80C8001E006F05FF847F09D
:10F960000300686078190835416841F00101416081
:10F97000FDE0A168B94280F0C480002800F0A680B4
:10F98000012505FA06F149004A42B04011430840FA
:10F9900041420840411E080B00F0100021FA00F21D
:10F9A000510901F0080322FA03F18A0802F0040267
:10F9B00021FA02F6710801F00208181826FA08F177
:10F9C0001018C1F340064044301821FA06F202EB49
:10F9D000000804EBC80000F128094FEAC80AD9F86A
:10F9E00008607068C008C000504518BF06F016F8DF
:10F9F000D6F808B04E4508BF06F010F85E4508BFBF
:10FA000006F00CF87068C008C000504518BF06F03A
:10FA100005F8D94505D1206805FA08F1884320602A
:10FA20000DE02069834508D3DBF80C00B04204D117
:10FA3000C9F808B0CBF80C9001E005F0EFFF47F0F3
:10FA400003007060AAEB0708B819019048F00100A4
:10FA500001994860019848F80080A7684FEAD70AE2
:10FA6000BAF1200F28BF05F0D9FF47B3CDF800A0A9
:10FA700004EBCA00D4F8149000F1280A102F38BF04
:10FA800005F0CCFF2068009920FA01F2D107D34697
:10FA900005D4009905FA01F10843206007E0DAF87F
:10FAA0000800216988422CBF834605F0B7FFCAF8D9
:10FAB0000890CBF80C90C9F808B0C9F80CA0C4F8AD
:10FAC000088006F108050198606150E06068C0B3E5
:10FAD00039462046FFF7E4FD050012D047E015F156
:10FAE000400F28BF4FF0FF370BD205F10B00C008C5
:10FAF000C700606828B139462046FFF703FC0500BF
:10FB000035D1A068B8421CD3C11B626910290AD341
:10FB1000B8186061A16041F001034360095047F0EB
:10FB2000030050600AE00021A160616140F0030120
:10FB300051608018416841F00101416002F10805FF
:10FB400015E0E06887420DD2C01BA169E0607A1819
:10FB5000A26140F00100506001F1080547F0030088
:10FB6000486004E039462046FFF7FFF90546C046E5
:10FB7000C046284603B0BDE8F08F00B970472DE9B4
:10FB8000F047A0F10804C046C046DFF800552869D8
:10FB90008442C0F07482616801F00302012A00F01F
:10FBA0006E82CA084FEAC208CA0708EB040936D4B5
:10FBB000226811F0030F00F06482A41A844290447A
:10FBC000C0F05D8269698C4200F0D880D608202E92
:10FBD00070D2D4F80CA0A768544508BF05F01EFFEA
:10FBE000BC4208BF05F01AFF6068C008C000B0EB57
:10FBF000C60F18BF05F012FF05EBC60000F1280183
:10FC00008F4205D029698F4251D3F968A1424ED164
:10FC1000BA453DD128680121B140884328604C4550
:10FC200080F02D82D9F80400C10740F128828107B5
:10FC300000F17A81A969894540F0B580E868AC6136
:10FC40004044E86040F00101616069698C4202D182
:10FC500000216961A960E969814280F01282DFF8C0
:10FC60003004006808B9FEF796FFA969002900F082
:10FC70000882E868292824BF2846FEF77FFFE86944
:10FC8000E968884280F0FD814FF0FF30E861F8E1DB
:10FC90002830824506D02869824508D3DAF8080062
:10FCA000A04204D1C7F80CA0CAF80870B7E705F065
:10FCB000B5FEB4E7E768A669A7420BD0A168814208
:10FCC00022D3C868A04204BFB868A0421CD1CF604C
:10FCD000B9601BE004F114010F6837B904F1100199
:10FCE0000F689FB101E011460F6807F11402136815
:10FCF000002B02BF07F110021368002BF3D18142E1
:10FD000002D30020086001E005F088FE002E86D0B6
:10FD1000E06905EB800000F5987001688C4209D11C
:10FD20000760380011D1E269686801219140884379
:10FD3000686074E72869864205D33069A04214BF21
:10FD40007761376101E005F069FE002F3FF467AF8E
:10FD500028698742ABD3BE61216929B1814226BFA0
:10FD600039618F6105F05AFE606900283FF457AF92
:10FD7000296988429BD37861876150E799F804002C
:10FD800000F0030003287FF44AAFC5F80880D9F8D3
:10FD9000040040084000C9F8040048F00100606019
:10FDA00048F804806DE16969894508D1A8686C61EB
:10FDB0004044A86040F001016160005161E1C00869
:10FDC000C0004FEAD00ABAF1200F804436D2D9F8E9
:10FDD0000C70D9F80860B94508BF05F01FFEB145A1
:10FDE00008BF05F01BFED9F80400C008C000B0EB46
:10FDF000CA0F18BF05F012FE05EBCA0000F128017A
:10FE00008E4206D029698E42C0F08180F168494552
:10FE10007DD1B74206D12868012101FA0AF1884351
:10FE2000286076E02830874205D0286987426ED363
:10FE3000B86848456BD1F760BE606AE0D9F80C70CD
:10FE4000D9F818604F450DD0D9F8080029698842C3
:10FE500023D3C168494504BFB96849451DD1C7606E
:10FE6000B8601CE009F11400076837B909F1100007
:10FE70000768A7B101E00846076807F114010A689E
:10FE8000002A02BF07F110010A68002AF3D129698C
:10FE9000884202D30021016001E005F0BFFD002E81
:10FEA00037D0D9F81C0005EB800000F59870016888
:10FEB00089450AD10760380012D1D9F81C2068683A
:10FEC000012191408843686023E02869864205D378
:10FED0003069484514BF7761376101E005F09EFD48
:10FEE000BFB12869874212D3BE61D9F8101029B179
:10FEF000814226BF39618F6105F090FDD9F8140069
:10FF000038B12969884202D37861876101E005F040
:10FF100085FD48F00100606048F80480686984420B
:10FF20000BD1C5F80880ACE040084000C9F80400D7
:10FF300048F00100606048F804804FEAD807202F9D
:10FF400022D205EBC70000F12809B8F1100F38BF25
:10FF500005F064FD286820FA07F1C9074E4604D46D
:10FF60000121B9400843286007E0D9F80800296951
:10FF700088422CBF064605F051FDC9F80840F460E0
:10FF8000A660C4F80C907CE05FEA182008BF00214E
:10FF900023D0B0F5803F28BF1F211ED2A0F580716D
:10FFA000090C01F008018840A0F58052120C02F003
:10FFB00004029040A0F580431B0CC1F10E0103F038
:10FFC0000203891AC91A984001EBD030C11D28FAE2
:10FFD00001F202F0010101EB4001E16100226261E6
:10FFE000226105EB81006A6822FA01F3DB0700F564
:10FFF000987006D4012303FA01F11143696004608B
:020000021000EC
:100000001CE01F2900680EBF00214908C1F1190139
:1000100008FA01F100E010464268D208D2004245D9
:1000200010D0CA0F00EB820202F1100349001A68D7
:10003000002AF0D129698B4211D31C60A061E460D1
:10004000A4600EE02A698168904228BF914206D3DD
:10005000CC608460A160E0600020A06101E005F058
:10006000DDFC286A401E28620BD1D5F8C80100E0EB
:1000700080680028FCD14FF0FF30286201E005F0D5
:10008000CDFCC046C046BDE8F087000018BB0300A9
:10009000F8D7030038B50C46082820D1854DE8680C
:1000A0008DF8000000AA012149206B691B6998475F
:1000B0002078002813D000EE100AB8EE400ADFEDD9
:1000C0007C0A80EE200A85ED040A10EE100AF6F78D
:1000D000D9FB02460B460FF2E810F7F705F80020AF
:1000E00032BD10B50020734C00E00120002806D17D
:1000F000A06980470028F8D104F1180060616369A5
:10010000002B05D10FF2C410F6F7EEFF032010BD4F
:1001100004F10802002147205B699847002010BDC8
:1001200010B5044664490820FAF74CF820466149A6
:1001300049694968BDE81040084713B586B002A870
:100140001021F2F70BFA00A800210A4606C0594C0C
:10015000616989688847002801D001206AE0062289
:1001600002A900A8F2F7C2F9F6F7B4F801284ED1B7
:10017000E06801284BD194ED040AF7EE000A70EE16
:10018000C00ABDF9000001EE100AB8EEC11A21EE56
:10019000001AB4F9000001EE900AF8EEE11A00EE40
:1001A000A11ABDEEC11A11EE100AADF8000000A8A8
:1001B000B0F9021001EE101AB8EEC11A21EE001AC1
:1001C000B4F9021001EE901AF8EEE11A00EEA11A4D
:1001D000BDEEC11A11EE101A4180B0F9041001EE03
:1001E000101AB8EEC11A21EE000AB4F9041001EE9B
:1001F000101AB8EEC11A00EE810ABDEEC00A10EE68
:10020000101A8180062200A902A8F2F76FF9BDF842
:100210000000208000A8418861808088A08008229A
:1002200006A90DF10E00F2F751F902A90120F9F724
:10023000A3FB002008B010BD10B504461E490820DD
:10024000F9F7E0FF20461B494969C968BDE810403D
:100250000847F8B504460D461646164F252C05D11D
:100260003178F9600FF26C00F6F73EFF324629460E
:1002700020467B691B6901B0BDE8F04018470D4B73
:100280005B695B6918470B4890ED020A70470B49A0
:1002900001F11002C26101220270042242700622A2
:1002A0008270012202820E22428241610020704748
:1002B0000000C8421869030095100100CC690300D2
:1002C00041434F45464620252E3266004143432098
:1002D000504600004C5046207374617475732020A2
:1002E0003A20256400000000024601214820884B86
:1002F0005B6A5B69184770B50024854D00E0641C9B
:10030000012C0ADA04EB440005EBC006B06A804712
:100310000028F4D106F1280068626B6A002B05D131
:100320000FF2F410F6F7E0FE032070BD05F1200295
:10033000002147205B69984705F1180202214720F8
:100340006B6A5B699847002070BDF8B50446F6F704
:100350000EF86F4DC5E9020100222A70D5E9062387
:10036000002B01D1002A14D0D5E90467002F01D158
:10037000002E0ED0801BB9418B420AD301D8824295
:1003800007D30FF29C10F6F7AFFE01202870002073
:10039000F2BD2046696A49688847002801D00120DB
:1003A000F2BD002205F14001A120F4F731FD002843
:1003B00001D00320F2BD54A0F6F796FE0020F2BD56
:1003C000D3B586B001A81021F2F7C8F8504C2078B8
:1003D000002820D0D4E90601DDE90623D4E904672A
:1003E000921BBB41994214D801D3904211D20020F4
:1003F0008DF800000FF23410F6F776FE0020FFF7BC
:10040000A4FF00AA03214920636A1B6998470020C2
:100410002070012012E001A8616A896888470028DD
:1004200001D001200AE0082206A90DF10A00F2F726
:100430004DF801A90420F9F79FFA002008B0D0BDBB
:1004400038B50546324C2078002805D00FF2EC0074
:10045000F6F74AFE002032BD002204F14001A1203F
:10046000F4F732FD002805D12846616AC96888473B
:10047000002801D0032032BDD4E90601002901D1B2
:10048000002803D0F5F773FFC4E904011FA0F6F7B5
:100490002BFE002032BD1E4B5B6A5B69184780B59E
:1004A00003463D3B022B09D8194B1B78002B05D086
:1004B0000FF29400F6F718FE002002BD144B5B6AA1
:1004C0001B69BDE80050184710B5114C04F14C02EF
:1004D00001214720636A5B69984704F14C0010BD15
:1004E0000B4890ED080A70470A4901F11002C261F9
:1004F00004220270427006228270012202820E22C1
:10050000428241610020704747594F0047594300DC
:10051000286603001C6A030047594F20504600001C
:1005200047594F20534B4950000000004759524F44
:1005300020535441525421210000000047594320C8
:10054000534B495000000000534F445220534B4935
:1005500050212100802282F3118800BF00BFC160BA
:100560000248407808B980F311887047C8670300D3
:1005700000B581B0802282F3118800BF00BF83687C
:10058000094A33B9507808B980F31188012001B0C5
:1005900000BD13785B1C137005F07DFAF9F786FF38
:1005A000002001B000BD00BFC867030010B50F4CAC
:1005B0002178491C2170802181F3118800BF00BF80
:1005C000A1688A69024205D1C861082008742046E2
:1005D000FDF729FEA168886900228A612178491EF9
:1005E0002170617809B981F3118810BDC8670300D3
:1005F00070B400240025264670C070C018384360CF
:10060000C260818270BC70472DE9F0470E46089F9A
:10061000099DDDF828900446924698463421F1F76A
:100620009DFF1049C4F814A0207C09780843207469
:1006300084F8299006B16662E819C008C00000215C
:1006400040F8501D4FF08071416407490164C0F8C3
:100650004C806FF00201416260602046BDE8F047C7
:10066000F9F77CBF71D90300F3F1000030B50D4DEF
:100670002A78521C2A7081B00124802282F31188CA
:1006800000BF00BF8268C3689A4202D205F0E0F959
:100690000024687808B980F31188F9F707FF20462D
:1006A00001B030BDC867030000B581B0802282F37D
:1006B000118800BF00BF8A69104388610A7C02F07C
:1006C000F802082A05D1CA6902421CBF0846F9F798
:1006D00009FF0348407808B980F3118801B000BDD4
:1006E000C867030010B5EFF3108072B60A4C21689A
:1006F00041F47F01216080F31088A06E10F4700F28
:1007000004BFA72005F0F4F94FF00070C4F81C02F4
:100710000020C4F8140210BD20ED00E0B5EEC00AC0
:10072000F1EE10FA02D4B1EEC00A70476FF0004C3F
:1007300000EE10CAFCF7D8BD10EE101A04204FF0DE
:100740007E5C01EE90CA49004FEA510100EE101A9A
:1007500088BF0820B1F17E5F13D871EEC00ADFF8C0
:1007600038C031EE801A61EE200AF1EEE00A6145F0
:1007700086BF80F0040080EE800A80EE200AFCF73D
:10078000ABBC490011F1807F9CBF6FF0004100EECF
:10079000101A7CF6A9AD7047F404353F4FF4001CE5
:1007A0001CEB410F94BF1CEB430F09E041EA030C23
:1007B00050EA4C0C52EA0C0C03D2994208BF90420A
:1007C000704714BF8B428242704700004FF4001CF8
:1007D0001CEB410F94BF1CEB430F09E041EA030CF3
:1007E00050EA4C0C52EA0C0C03D28B4208BF8242F6
:1007F000704714BF994290427047000030B50446DC
:1008000010480D460178491C017081B0802080F3AA
:10081000118800BF00BFA06858B94021204605F0EC
:10082000DFF8802080F3118800BF00BFA068002897
:10083000F3D02946204605F02EF901B0BDE830403E
:10084000F9F734BEC86703002DE9F04FA1B0824626
:10085000002017461D4602910B900DF1440B6FF0DE
:1008600000490AE017F8011B0298D04702900028BF
:1008700000F0A8820B98401C0B90387808B90B98B0
:10088000A2E22528EED1002005900690079008905E
:1008900009900A9001E040F0010017F8011F20299B
:1008A000F9D023290DD02B2904D02D2906D03029A9
:1008B0000AD00CE040F0020080B2EEE740F0040005
:1008C000FAE740F00800F7E740F01000F4E72A29C3
:1008D0000ED12968296051F8042B2960002A0D9255
:1008E00004D5514240F004000D9180B27F1C11E00C
:1008F00000210D9109E00D99494505D001EB8103D7
:1009000002EB430130390D917F1C3A78A2F130019E
:100910000A29F0D339782E2903D04FF0FF310C91FA
:100920001DE017F8011F2A2907D1296829607F1CBB
:1009300051F8042B29600C9211E000210C9109E080
:100940000C99494505D001EB810302EB4301303995
:100950000C917F1C3A78A2F130010A29F0D3ADF84E
:1009600038000FF67440397805F0D6F808B117F85A
:10097000010B8DF83A009DF83A00682802BF3978DB
:100980006829622005D06C2804BF38786C2803D110
:1009900071208DF83A007F1C11A8049017F8014BC4
:1009A000B4F125002AD01C3800F0CC80001F0228AA
:1009B00040F2C880133800F0EE80093800F0C280A1
:1009C000801E00F04F81401E00F02481401E02284E
:1009D00040F2B880001F00F01D81401F00F08380AE
:1009E000401E00F0D880401E29D0C01E0CD0801EB2
:1009F00000F0D180C01E00F0CE803DE101200590C6
:100A000025208DF8440043E12868286050F8044B05
:100A100028600394DDF83080B8F1000F04D520463B
:100A2000FCF786FC804607E042460021204605F0A0
:100A30007FF808B1A0EB0408CDF8188028E12968F8
:100A400029604FF03C0851F8040B29600021CDE9E2
:100A5000000111A80390DDE90001049C11B908B957
:100A60000C9AC2B10206120FA0EB02123032D2B2BF
:100A70003A2AA8BF27320009A8F1010340EA017011
:100A800009091A5508BF0028984604D0039A08EBB4
:100A900004039A42E6D308EB04000390C8F13C013A
:100AA0000C980691814209DA401A08904FF6EF71CE
:100AB000BDF838000840ADF83800E9E0002840F102
:100AC000E7809DF8380000F01400102840F0E08026
:100AD0000D98059A801A089A801A401A0128C0F2C7
:100AE000D7800890D4E09DF83A0062281AD0682890
:100AF00006D06A280CD06C281CD0712808D019E0C8
:100B00002868286050F8041B28600B980880BFE014
:100B10002868286050F8042B28600B98C117C2E998
:100B20000001B5E02868286050F8041B28600B9885
:100B30000870ADE02868286050F8041B28600B9806
:100B40000860A5E02868C01D20F007022A60D2E9ED
:100B5000000108322A60CDE90001002903D50120F7
:100B600005902D200CE0BDF83800810703D5012049
:100B700005902B2004E0C00704D50120059020201B
:100B80008DF84400059911A808180390214600A883
:100B900000F0D8F97CE09DF83A206C2A0DD0712A3B
:100BA00018BF6A2A09D12868C01D20F007032B60EE
:100BB000D3E9000108332B6005E02968296051F86A
:100BC000040B29600021CDE90001682A08BF80B22A
:100BD00007D0622A08BFC0B203D0742A18BF7A2A8D
:100BE00002D10021CDE900019DF83800000730D581
:100BF000DDE90001002908BF00282AD044F02000C8
:100C0000782826D130208DF844008BF8014002204E
:100C100005901EE09DF83A00294600F0D8F8CDE98D
:100C20000001002904DA0598411C05912D210EE0F0
:100C3000BDF83800810704D50598411C05912B218A
:100C400005E0C00705D50598411C0591202100F855
:100C50000B10059911A808180390214600A800F070
:100C6000EDF815E0012005902868286050F8041B75
:100C700028608DF844100BE0012005902520002C01
:100C80008DF8440004D00598411C059100F80B40F4
:100C90000D980599401A0899401A0699401A099921
:100CA000401A0799401A0A99A0EB01089DF83800EC
:100CB00040070FD420208DF84000002408E00123D5
:100CC00010AA00A9504600F070FC00287AD1641CDC
:100CD0004445F4DB059C11AE0AE016F8011B0298AE
:100CE000D047029000286DD00B98401C0B90641EDA
:100CF000002CF2D130208DF840000026089C08E03E
:100D0000012310AA00A9504600F04FFC002859D139
:100D1000761CA642F4DB069C039E0AE016F8011B33
:100D20000298D047029000284CD00B98401C0B90A2
:100D3000641E002CF2D130208DF840000026099C62
:100D400007E0012310AA00A9504600F02EFCC8BB02
:100D5000761CA642F5DB03980699079C0E1809E05D
:100D600016F8011B0298D047029058B30B98401C0C
:100D70000B90641E002CF3D130208DF8400000262B
:100D80000A9C07E0012310AA00A9504600F00DFCC0
:100D9000C0B9761CA642F5DB9DF8380040077FF508
:100DA0006CAD20208DF84000002400E0641C444518
:100DB000BFF663AD012310AA00A9504600F0F5FB71
:100DC0000028F3D04FF0FF3021B0BDE8F08F62284B
:100DD00026D068281DD06A2808D06C2827D0712812
:100DE00004D0742823D07A280CD020E00868C01DD5
:100DF00020F007000860D0E9002308300860194699
:100E0000104670470A680A6052F8040B0A60002115
:100E100070470A680A6052F8040B0A6000B20BE0DF
:100E20000A680A6052F8040B0A6040B204E00A68DB
:100E30000A6052F8040B0A60C11770472DE9FA4E98
:100E400005460A462F696F2A08BF082405D041F0DD
:100E50002000782814BF0A2410243C26D5E900017C
:100E6000642A18BF692A81468A4605D1002903DA17
:100E7000D9F100096AEB4A0ABAF1000F08BFB9F1CB
:100E8000000F0CD1286B50B9082C36D195F83800DA
:100E9000000732D530203B2687F83B002DE0E317D2
:100EA00048465146224604F06FFEA4FB0023A9EBFE
:100EB00002023032D2B2A6F1010B3A2A5E4603DBBF
:100EC0009DF80030513B9A1881465FEA010A0BF801
:100ED000072008BFB9F1000F03D0E868F119884274
:100EE000DDD3082C09D195F83800000705D5F05D51
:100EF000302802D0761E3020F055C6F13C00A861A3
:100F0000F119E960296B884208DA081A28624FF65D
:100F1000EF71288F08402887BDE8F38E00290ED591
:100F200095F8381001F01401102908D1696B6A692D
:100F3000891A2A6A891A081A0128A8BF2862BDE8F6
:100F4000F38E00002DE9F24F04468EB0D4E9000183
:100F5000CDE9020104AF9DF8380040F0200BBBF151
:100F6000610F0AD0206B002848BF062004D408BFB8
:100F7000BBF1670F01D1012020636168C1F30A5002
:100F800040F2FF7290421CD1080304BF2068002881
:100F900009D10320A0619DF8380061381A2836D3A2
:100FA0000FF2486108E00320A0619DF83800613825
:100FB0001A2829D30FF22C61E0680322F1F786FA90
:100FC000BEE1012816DA204600F0C4FC012811DB3E
:100FD00000250020BBF1610F20D1E168302201F82B
:100FE000012B4A1CE2609DF83820612A0CBF782250
:100FF00058220FE0626840F2FE3161F31E52451A3A
:1010000062604FF0FF30E5E70FF2D451D4E70FF202
:10101000D851D1E70A706169891C616110B9002655
:10102000002584E1BBF1610F40F09780206B002820
:101030004CBF2126461CDDE90201D4E900AB0022A9
:101040000023FFF7ABFB36B23ABF8BF00040CDE98F
:1010500002A0CDE902AB06F101082D1F8DF810208A
:101060000DF1110700E0C71DB8F1010F33DBDDE919
:10107000020100220023FFF7A9FB2CD21C2102A8A9
:1010800004F0FAFDDDE90201FBF748FAA8F10708D0
:10109000B8F1010F814609DBFBF71EFA02460B4649
:1010A000DDE90201F5F7CAFECDE90201F81D0721CD
:1010B00005E009F00F0200F8012D4FEA2919B9F1F6
:1010C000010F01DB491EF4D5491E5CBF002200F868
:1010D000012DF9D5C7E70DF11100391AB142B8BF9A
:1010E0000E4636B230000DF111072FD4884206DAD1
:1010F00004A9411849780829A8BF0F2100DA002166
:1011000004AA821800E0761E12F80139401E8B42B4
:10111000F9D00F2904D104A941184A78521C4A7009
:10112000002802D504AF761C2D1D36B2701E0DD4DA
:10113000C1190A783032D2B23A2A03DB9DF838302E
:101140003A3B9A18401E01F80129F2D5206B00287D
:1011500040F1ED80701E2063E9E0DDE9020100222C
:101160000023FFF71BFB3CBF81F00041CDE90201EA
:101170002DB247F2975068434B49DFF8309190FB0E
:10118000F1F52DB2C5F1070ABAF1010F90461CDB4B
:10119000DDE902675FEACA7007D542464B46304632
:1011A0003946F5F797FB06460F464FEA6A0A40466E
:1011B000494642464B46F5F78DFBBAF1000F804693
:1011C0008946E7D1CDE9026724E0CAF1000A00268A
:1011D000374F14E05FEACA7007D542464B463046A7
:1011E0003946F5F777FB06460F464FEA6A0A40464E
:1011F000494642464B46F5F76DFB80468946BAF1B3
:10120000000FE7D1DDE9020132463B46F5F7F2FC7B
:10121000CDE90201BBF1660F216BDFF898900CBF9E
:1012200005F10A0006204618142EA8BF1326302008
:101230008DF810000DF11107012E3DDBDDE90201F3
:10124000FBF782F907F1080104220A23B0FBF3F34C
:1012500003EB8307A0EB4700303001F8010D0A20B3
:10126000B3FBF0F000EB8007A3EB47033033521ED3
:1012700001F8013DE9D1083E012E01F10807DBDB51
:10128000DDE90201FBF760F9FBF730F902460B4696
:10129000DDE90201F5F7D2FD00224B46F5F71AFB16
:1012A000CDE90201CAE700BFA0860100000024408A
:1012B0000000F03F84D797410DF11100381A0DF16D
:1012C000110702E0401E6D1E7F1C39783029F9D0CD
:1012D000BBF1660F02D12DB2691C04E0BBF1650FB2
:1012E0000CBF01210021226B8E1836B2B042B8BF6C
:1012F000064636B231001AD4814204DAC85D352878
:10130000A8BF392000DA3020CA19521E00E0761E2C
:1013100012F80139491E8342F9D0392802D1C85D3B
:10132000401CC855002902D57F1E761C6D1C2DB2AD
:101330009DF83810009533B23A46204600F003F885
:101340000FB0BDE8F08F2DE9F043054685B01E468D
:10135000D5F83080012E8946174602DA01260FF2B1
:10136000902749F02000BDF93040662808BF641C72
:1013700017D0672840F0828014F1040FC0F28480F7
:10138000444580F2818095F83800641C000702D43F
:101390004645B8BFB04624B2B8EB040848BF4FF08A
:1013A000000824B2E868A969012C25DA4A1C302318
:1013B0000B54B8F1010F03DA95F83810090702D57C
:1013C0002E211154521C18EB040FB8BFC8F10004B1
:1013D00024B26142A044B045AA61B8BF46466962E2
:1013E00036B2EE613246AB6939461818F1F76EF83D
:1013F000A8EB0600A862C1E00818A64218DA324637
:101400003946F1F763F8A9697118A01BA961B8F111
:10141000010F686203DA95F83800000705D5EA681D
:101420002E208854E869401CE861C5F82880A5E0B2
:1014300022463946F1F74AF8A8692018361BB8F158
:10144000010F03DA95F83810090703D5EA682E2151
:101450008154401CA86136B2B045B8BF4646E86822
:10146000AB6936B23246E1191818F1F72FF8A869BE
:101470003018A861A8EB060068627FE0B9F1610F3F
:1014800016D14FF0700918E0464504DA95F8381087
:10149000090758BFB046B8F1010848BF4FF000082F
:1014A000B9F1670F14BF4FF045094FF0650904E02B
:1014B000B9F1410F08BF4FF05009A969E86817F862
:1014C000013B0B544A1CB8F1010F05DA95F83810AE
:1014D000090758BFAA6117D52E211154531CB8F122
:1014E000010FAB6110DB761E36B2B045B8BF464681
:1014F00036B2324639461818F0F7E8FFA8693018B6
:10150000A861A8EB06006862E868A9690F182000C6
:1015100007F8019B03D42B2007F8010B03E02D21D2
:1015200007F8011B644200260DF1080808E00A22B2
:1015300000A804F02DFC019808F8010B761C009C13
:1015400021B20129F3DA022E06DA49F020006528DB
:1015500004BF302007F8010B4EB9302007F8010B0B
:1015600007E0761E02A8305C303007F8010B012E30
:10157000F7DAE868A9690818381AE86195F83800B8
:1015800000F0140010280DD16869A9690818696A6B
:101590000818E9690818A96A0818696B8842BCBF6D
:1015A000081A286205B0BDE8F083F8B504460D4678
:1015B00016461F46002004E0E86A401CE8627F1ED1
:1015C000002047B116F8011BA868A047A8600028B2
:1015D000F2D14FF0FF30F2BD686A6C747A4C0000B3
:1015E0006E616E004E414E00696E6600494E4600C7
:1015F000300000002DE9F84C2DED068B154603B4A4
:10160000C1F30A5040F2FF7188420CD101980024C6
:10161000000304BF0098002802D1019800281BD4C1
:10162000DDE9000113E101280FDA00A800F092F9CA
:1016300001280ADBFBF74AFD2221016002B00020ED
:10164000BDEC068BA249BDE8F48C019A40F2FE3154
:1016500061F31E520192441A019800280CD5FBF741
:1016600035FD2121016002B04FF0FF30BDEC068B4B
:101670006FF00041BDE8F48CDDE90001954A964B1E
:10168000FFF78CF809D2DDE9002300204FF08041FC
:10169000F5F720F9CDE90001641EDDE90023002003
:1016A0008E49F5F78BFCDDE9002341EC180B002097
:1016B0008B49F5F783FC02460B4651EC180BF5F706
:1016C00099FA41EC190B53EC192BF5F703F941EC9E
:1016D0001A0B53EC1A2B83488349F5F7FBF8834A1E
:1016E000834BF5F76BFC53EC1A2BF5F7F3F8814AB3
:1016F000814BF5F763FC53EC1A2BF5F7EBF87F4AB7
:101700007F4BF5F75BFC53EC1A2BF5F7E3F87D4ABA
:101710007D4BF5F753FC53EC1A2BF5F7DBF87B4ABE
:101720007B4BF5F74BFC53EC1A2BF5F7D3F8794AC2
:10173000794BF5F743FC53EC1A2BF5F7CBF802463F
:101740000B4651EC180BF5F779FB53EC192BF5F719
:10175000C1F841EC190B20B2FAF7BEFE41EC1A0BAE
:10176000CDB953EC1A2B6D486D49F5F7B3F853EC2E
:10177000192BF5F763FB53EC182BF5F71FFC044608
:101780000D4653EC1A2B4FF040406649F5F7A2F88E
:1017900022462B4659E0012D53EC182B34DB002058
:1017A0006149F5F797F882468B4653EC182B5F4852
:1017B0005F49F5F78FF806460F4653EC1A2B5D4844
:1017C0005D49F5F787F804460D4653EC192B5B4845
:1017D0005549F5F77FF802460B4620462946F5F7AE
:1017E0002DFB32463B46F5F7E9FB52465B46F5F7E3
:1017F000E5FB04460D4653EC1A2B00205049F5F743
:1018000069F822462B4620E04FF0C0404D49F5F7DD
:1018100061F804460D4653EC182B4B484B49F5F73D
:1018200059F806460F4653EC192B49484549F5F738
:1018300051F802460B4630463946F5F7FFFA224684
:101840002B46F5F7BBFB53EC1A2BF5F7B7FB02B0B1
:10185000BDEC068BBDE8F48C80B52DED028B41EC20
:10186000180B53EC182B1F481F49F5F733F81F4A84
:101870001F4BF5F7A3FB53EC182BF5F72BF81D4A7C
:101880001D4BF5F79BFB53EC182BF5F723F81B4A80
:101890001B4BF5F793FB53EC182BF5F71BF8194A84
:1018A000194BF5F78BFB53EC182BF5F713F8174A88
:1018B000174BF5F783FB53EC182BF5F70BF8154A8C
:1018C000154BBDEC028BBDE80050F5F777BB00006F
:1018D0000000F0FFCD3B7F669EA0E63F0000F0BF1A
:1018E0000000F03FF7DE29BFD8F8C23FF4B3FECCCA
:1018F0001A99C33F62CB68D96F46C73FC6C912DA8F
:10190000C471CC3F4AE98A942449D23FF75F979942
:101910009999D93FBC5555555555E53F9EBC9AF709
:101920001C7D7F3E422EE63F7BCBDB3FABA6320EDB
:10193000E526553E7CC4BC7FDE27743E0EE52615A9
:101940001344D33F4715F73F44DF5DF80BAE543ED9
:10195000FE822B6530B4436803F0004201211B0373
:101960001B0B436004BF0368002B08D10DE0036824
:10197000DD0F45EA440444605B000360491E44688F
:10198000E302F4D523031B0B436043681A43426010
:10199000084630BC70474268C2F30A5240F2FF73F7
:1019A0009A4209D14168090304BF0068002801D1A7
:1019B000012070470220704743685B0004BF036842
:1019C000002B25D040F233439A1A521A012A1FDB0A
:1019D000352A06DB416801F00041416000210160C9
:1019E00013E0012102F01F039940491E920607D51A
:1019F000426811404A40426002681143002202E0FE
:101A0000026811404A40026011B14FF0FF30704748
:101A10000020704790420CD141EA030C50EA4C0C74
:101A200007D0994205D14FF4001C1CEB410F38BF81
:101A3000894270472DE9704C04462DED088B94EDDA
:101A4000009B43EC182B51EC190B04F0A8F9064647
:101A500051EC180B04F0A3F931000E9D06D50028B7
:101A60004DD4022805D184ED008B42E1022EF8D13D
:101A700021E050B951EC190B0022344BFFF7CAFF9B
:101A80000FD084ED008B002033E1012818D151ECF8
:101A9000190B00222E4BFFF7BDFF18BF84ED008B02
:101AA00051D1FBF713FB212101604FF0FF306FF0A4
:101AB0000041C4E90001BDEC088B0220BDE8708C38
:101AC0007EB984ED008B2946204604F0D5F8040049
:101AD00018BF012C40F00C81FBF7F8FA22210160BD
:101AE00006E151EC190B0022184BFFF793FF0DD1C3
:101AF00051EC180BF4F7EEFEC4E9000123E051ECC1
:101B0000190B0022134BFEF749FE0BD251EC180BB8
:101B10000023F4F7DFFEC4E90001BDEC088B0020D0
:101B2000BDE8708C01220C4BFEF750FE16D851EC2C
:101B3000180B0022054BF4F7CDFEC4E90001FBF7BA
:101B4000C5FA222101600120D3E000BF0000F07F30
:101B50000000F0FF00C89CC000C89C40384A394BC8
:101B6000F4F7B8FE00220023FEF718FE34BF9FED05
:101B7000360B9FED370B53EC102BF5F71FFAFAF7E6
:101B8000CDFC0646FAF7A8FC41EC1A0B4FF0784260
:101B9000314BF4F79FFE02460B4651EC190BF5F75B
:101BA0004DF982468B4653EC1A2B2C482C49F4F7FE
:101BB00091FE02460B4650465946F5F73FF96FF045
:101BC0000102284BFEF702FE41EC190B05D800225A
:101BD000254BFEF7E3FDC0F07D8053EC192BF4F7A5
:101BE00079FE41EC1A0B214A214BF4F773FE214A8E
:101BF000214BF5F7E3F953EC1A2BF4F76BFE1F4A70
:101C00001F4B41EC1B0B51EC1A0BF4F763FE1D4A02
